:10000000004000205D7000009D7000009F700000A7
:1000100000000000000000000000000000000000E0
:10002000000000000000000000000000A1700000BF
:100030000000000000000000A3700000A570000098
:10004000A7700000E5510000D9740000A7700000FF
:10005000A770000000000000A7700000A77000005B
:10006000A7700000A977000055310000A7700000BC
:10007000A7700000A7700000A7700000A770000024
:10008000A770000041790000A7700000A770000071
:10009000A7700000A7700000A7700000A770000004
:1000A000A7700000A7700000000000000000000022
:1000B0000000000000000000000000000000000040
:1000C00010B5064C2378002B07D1054B002B02D02E
:1000D000044800E000BF0123237010BD640200202B
:1000E0000000000070E30000044B10B5002B03D0AB
:1000F0000349044800E000BF10BDC04600000000F6
:100100006802002070E30000164B002B00D1144B56
:100110009D46402292029A1A924600218B460F4633
:100120001348144A121A0BF0B3F90F4B002B00D0EE
:1001300098470E4B002B00D0984700200021040068
:100140000D000D48002802D00C4800E000BF0BF065
:100150005FF92000290007F0DDF90BF033F9C04604
:100160000000080000400020000000000000000027
:1001700064020020B82F00200000000000000000F2
:1001800002000120104011D1042A0ED91368180969
:1001900080B2002809D001388000031D11180979A8
:1001A000002902D001309842F8D170470020FCE7C6
:1001B0000378002B03D05AB2002A01DB01307047CC
:1001C0003F229343C03B59424B41C01803789343AD
:1001D000802BF4D10130F9E710B500240378002B0F
:1001E00001D1200010BDFFF7E3FF0134F6E770B541
:1001F000002204000D00411C092003F0C7FA00286A
:1002000006D001236200134343600023A34200DBB6
:1002100070BD9A00A958821891600133F6E770B555
:10022000012803DC1C2001F047F870BD01230D6894
:1002300011201D42F7D04868184206D1042804D97D
:100240000F2302681340042B01D00E20EBE703F0CC
:10025000FBF86D100400002D03DDFFF7BDFFA84281
:1002600006DA1220DFE72000FFF7A2FF0400013DBD
:10027000012DF8D120787F2809DDDF280BDCF82359
:100280003F22DB00800118406378134018430123AC
:1002900040001843C9E7EF280BDCFC226378120109
:1002A0009B0113403F220007000C0343A07810403D
:1002B000ECE7F72812DCFC22637892021B03134060
:1002C000E0228004520310403F221843E378134099
:1002D000FC220343A07812018001E8E7012040429C
:1002E000D5E7F8B54D680F00EB0706D4042D04D907
:1002F0000F232E683340092B03D00B2000F0DCFFC6
:10030000F8BD6B683609B6B25C10731EA3420FD8F5
:100310000321200008F078FF6421642803DC010039
:10032000032800DA03212800891903F061FA050087
:100330002B6800201B099BB2013B9C42E0D23A682B
:10034000A31C9B005A510123013464001C436C60C0
:10035000D6E7F0B585B0012803DC1C2000F0ACFF27
:100360002CE001274B683A000093022806D08B68E6
:100370003B4203D05F10002F00DC17000124009BDC
:10038000234200D0B2E0042B00D8AFE01B680D6818
:100390000F2619003140042925D1254205D1042D0D
:1003A00003D92B681E40042E01D00E20D6E70098FA
:1003B000FFF7E6FEB84203DA0120404205B0F0BD87
:1003C000009803F041F80600280003F03DF8010012
:1003D000781E30180BF012FC0028EDD0801B013085
:1003E00040002043EAE709293DD1009B5B685B1090
:1003F00001939F42E0DC25422CD1042D2AD92B68A1
:100400003340042B26D1280003F01EF803960290F7
:100410007E1C009AB300D058854201D17800E0E7F5
:1004200020420ED104280CD90368039A1340042BF0
:1004300007D103F009F8010002980BF0A9FB00288E
:10044000ECD0019B37009E42E2DDB5E71F00019B27
:100450009F42B1DC7B1C00999A008A58AA42F5D1D0
:1004600078000124BDE7032940D11A0992B25B0F3D
:1004700092000B40D31A01939F429DDC254229D163
:10048000042D27D92A681640032E19D1100980B2ED
:10049000520F800032402C1D801A019B26181B1A17
:1004A0000193009B781E0433019A904200DD83E79C
:1004B00022001918B2420FD316D101304000D0E704
:1004C000042E07D1280002F0BFFF04002800FFF728
:1004D00057FEE2E70F2041E70D78AC461578AC45B2
:1004E00002D101310132E5E70130DDE7212035E7B6
:1004F00010B502F08DFF43000120184310BD00002D
:10050000C30711D404280FD90F2302681340032B0B
:100510000AD119400133591AC0234907DB05194094
:10052000024B1A40114301607047C046FFFFFF9F16
:10053000F7B507000E001C20012F06DD4C680123D3
:1005400022001A40009203D10D2000F0B5FE53E0C6
:10055000022F02D08A681A42F6D0012335681D4264
:1005600000D0A9E0042D00D8A6E01C41002C00DC3E
:100570001C000F2029680840092828D16B685B10EF
:100580000093022F05D0B368009A5B109A4200DDF9
:100590000093009B01221D1B0135EB43DB171D401F
:1005A000691C092003F0F2F8071E09D001236D0031
:1005B0001D4303003268083345600099A14201DA07
:1005C0003800FEBD0134A100515802C3F5E70428EC
:1005D00045D1280002F038FFFFF7FEFD0190022F01
:1005E00004D0B3685B10984200DD0193019BA342E5
:1005F00004DA002003F03CF90700E1E7280002F0EC
:1006000023FF0700009BA34221DB2800009702F094
:100610001BFF05003800FFF7CBFD019B01340700ED
:10062000A342F7DA009BC41A200003F021F9071E49
:10063000C6D002F009FF0190306802F005FF2200E9
:10064000009B591B411801980AF006FFB8E73800D3
:10065000FFF7AEFD009B070001330093D2E70328AC
:100660002AD10B099BB2490F9B000140591A022F56
:1006700004D0B2685210914200DD1100A14205DAA7
:1006800000220320110003F081F8B5E703200E1BC0
:10069000331DD9170140C9188910002203F076F8DC
:1006A000071E00D18CE7013631000334FFF728FF25
:1006B000381D29193200C7E7212046E7F8B5002880
:1006C00005DC1C2000F0F8FD05002800F8BD01261F
:1006D0000C6826400FD06410E343DB171C40E11C7C
:1006E00089100022032003F051F8051EEDD02100EF
:1006F000FFF706FFE9E7042C01D80025E5E70F2303
:1007000022681340042B1BD12000FFF739FDC31CC6
:1007100007000320D9170140C9188910320003F0DF
:1007200035F8051ED1D03900FFF7EAFE200002F0AF
:100730008BFE2B1D01003A0018000AF08DFEC4E765
:10074000092BDAD10320636832005F10FB1CD91734
:100750000140C918891003F019F8051ECDD03900E1
:10076000FFF7CEFEFF20BE42AFDA0122B300E3184E
:100770009B68134208D01341FF2B00DD0300D943CF
:10078000C917AA190B4013710136ECE710B57F2980
:1007900002DC0170013010BD1A4B99420CDC402381
:1007A0008A115B42134303703F230B40802149426F
:1007B000194341700230EEE7134B994210DC2023BD
:1007C0000A135B4213433F24802203708B11524271
:1007D0002340214013430A43437082700330DAE719
:1007E0000A4B9942D7DCF0230370603B4370113B06
:1007F0008A11FF3B1A4382703F2211401943C17096
:100800000430C8E7FF070000FFFF0000FF0F0100F2
:10081000F0B50D0085B0002803DC1C2000F04CFD75
:100820000DE009680122080010400AD002AC114115
:100830002000FFF7ABFF011B200003F025F80400A8
:100840001AE004293FD90F230C682340092B3AD121
:100850004B685B10019303239C46019B9A420EDD7B
:1008600003F006F8041E07D02E68012502F0ECFD07
:100870002F00019B9D421DDD200005B0F0BD01321F
:100880009300CC580123234001D10D20C6E764100A
:100890007F2C0DDD0D4E0223B44209DD0C4E634664
:1008A000B44205DD00270B4EE30FA6427B419B00BF
:1008B000C018D2E70135AB00F1583942E5D04910F4
:1008C000FFF764FFD5E72120A8E7C046FF07000037
:1008D000FFFF0000FF0F010010B5040001200840D9
:1008E00010D104290DD90F230A681340042B08D115
:1008F000080002F0A9FD010020000BF049F9434275
:10090000584110BD0020FCE7F7B50F00012803DCBB
:100910001C2000F0D1FCFEBD01264D682E4006D102
:10092000042D04D90F222B681A40092A01D00B206C
:10093000EFE76A681B099BB25410A34200D85C1E03
:1009400039681E48FFF7C8FF01230190002813D122
:1009500039681B48FFF7C0FF002811D0002C0DD0CC
:100960000123621C013C9C409200535123436B6065
:1009700004E00136B200AB50B442FADA0020CAE714
:100980003B680D20DA07C4D55B10002B11DD9C42BB
:100990000FDB9B00A200291DEB1889180433994234
:1009A00009D10123013C9C40AA181C4353606C6090
:1009B000E4E71220ADE758681860EFE723CB0000AA
:1009C00027CB0000002310B50C000B70C30705D522
:1009D0000D49421020000BF09FF808E00B49002859
:1009E00002D0042804D10A4920000BF0B5F810BD4C
:1009F0000428FCD90F2302681340042BF7D102F01E
:100A000023FD04490200E5E720D500002CCB0000BF
:100A100032CB000037CB0000F0B593B00600029156
:100A20001C20012E1DDD029B01251B681C002C4093
:100A300000D0ADE0042B00D8E6E01A680F231A407E
:100A4000092A4AD10394039A029992008A581700FE
:100A50002F4005D1042A03D910681840092806D070
:100A6000222000F029FC0190019813B0F0BD5268DB
:100A70005210A418039A013203929642E3D1611CEA
:100A8000012202F083FE0190002802D1002301938D
:100A9000EAE7019B6400190025435D600831029A72
:100AA000BB00D05802684368120992B25B109A42A8
:100AB00000D8531E0022934209DCDA43D2171340B8
:100AC0009B00C918039B01379F42E8DBCCE79400E9
:100AD0000519AD6801320D51EDE72700032A59D100
:100AE0000193029ABB00D3582B42B9D1042BB7D93A
:100AF000186801990140032939D1020992B2430FC4
:100B000092000B40D31A1C190137BE42E9D10320D1
:100B1000E31CD9170140C9188910002202F036FEE3
:100B200001900028B2D000252100FFF7E9FC019BCD
:100B30001E1D029AAB00D45801231C421FD1042C65
:100B40001DD90F2123681940032918D1180980B233
:100B50005B0F80000B40C01A0023834213DBC343AA
:100B6000DB17184001353618BD42E2DB7CE704296B
:100B700000D075E71800FFF703FB2418C4E7200036
:100B8000FFF7FEFAE8E7E2181279F2540133E4E7DE
:100B900000273C000F25029ABB00D35801221342C4
:100BA00034D1042B32D9186801002940042935D1E9
:100BB0001800FFF7E5FA24180137BE42EBD12000F8
:100BC00002F056FE0190002800D15FE7029FB600B8
:100BD000BB19041D029301233D681D4229D1042D38
:100BE00027D90F262B681E40042E37D12800FFF787
:100BF000C7FA0600280002F027FC0100200032009E
:100C00000AF02AFCA41922E02700C3E7180005A96E
:100C1000FFF7D8FE05A80AF0C5FFCCE7032900D0EE
:100C20001EE7020992B2430F92000B40D31A1C191F
:100C3000C2E705A92800FFF7C5FE05A80AF0B2FF24
:100C400005A90500020020000AF006FC6419029BB9
:100C50000437BB42BFD10023237005E7032EF6D132
:100C60001A0992B25B0F92001E40961B291DC5E720
:100C7000F0B50D0095B0002806DC1C2000F01CFB30
:100C80000400200015B0F0BD0C68012123000B40CA
:100C9000009306D1042C04D922680F331A40092A84
:100CA00001D00B20EAE7626852100392002A03DCAD
:100CB000009802F0DDFDE3E73F4A019201280BD0E6
:100CC0006868084208D1042806D902681340042B3A
:100CD00002D102F0B9FB019001980AF063FF06000F
:100CE0000F27039B0834013B04935E43039B029050
:100CF0009B001B19059301232068184251D1042839
:100D00004FD903683B40042B52D1FFF739FA059BBA
:100D100004343618A342EED1300002F0A9FD041EBF
:100D2000AFD02B680593029B002B03D0686802F0BC
:100D30008BFB0190200002F087FB0500009B059AC9
:100D40009B00D3189F68380002F07EFB0123060049
:100D50001F4201D1042F04D807A93800FFF732FE43
:100D600007AE30000AF01EFF070002003100280025
:100D70000AF072FB029BED19002B0AD0049B009A2B
:100D8000934206DD2800029A01990AF065FB029B56
:100D9000ED18009B01330093009A039B9342CDD141
:100DA0006FE707A9FFF70EFE07A80AF0FBFEAEE704
:100DB00002F04AFBF9E7C046C4CF000010B500249A
:100DC000A04207DD0B6801341C4003D05C10E343F4
:100DD000DB171C40611C0122092002F0D7FC00280F
:100DE00003D0012364001C43446010BD0A6870B541
:100DF00010000125284034D1042A32D90F24136869
:100E000049681C40092C17D154681B099BB22C411E
:100E1000A34200D85C1E844205DC022001339842C4
:100E200006DB00200FE085005519A9600130F2E7CC
:100E3000840011510130F2E7032C12D1294203D171
:100E4000132000F039FA70BD4910FF29F8D81B09AA
:100E50009BB204329B00D3189342E2D91170013245
:100E6000FAE70B2000F028FADBE700000123F7B5D2
:100E700000254E680F0033400093AB420ED11D0099
:100E8000042E0BD90F2233681A40092A10D1726838
:100E90001B099BB25510AB4200D85D1E3968CB07C9
:100EA00017D54C10002C01DDA5421DDA122032E0CE
:100EB000042A04D13000FFF763F90500EEE7009D36
:100EC000032AEBD11D09ADB25B0FAD001340ED1A43
:100ED000E4E72E48FFF700FD002814D00AF0B8FD23
:100EE000290008F077FA4C1C009B002B4CD1042EF3
:100EF0004AD932680F331340092B10D10134A400B2
:100F0000A4592000FEBD39682148FFF7E5FC2C00FC
:100F10000028E9D1113000F0CFF90400F1E7042BEB
:100F20002AD1300002F090FA0500FFF755F9A042EF
:100F3000BCDB012C1ADC300002F086FA009028009D
:100F4000FFF736F9461B300002F092FC041ED8D0A1
:100F500002F07AFA0190786802F076FA009B32008B
:100F6000E91A411801980AF077FACAE72800FFF752
:100F70001FF9013C0500DCE7032B05D13419E478A7
:100F8000023B64001C43BCE70B20C4E71CCB000001
:100F900027CB0000F7B54D680F002A0001210A4059
:100FA0002FD1042D2DD90F242B68BE681C40092C8D
:100FB00014D169681B099BB24C100192A34200D85E
:100FC0005C1E39682A48FFF787FC00282DD00F23C4
:100FD0002A681340092B1DD1012317E0032C10D1DF
:100FE0000E4203D1132000F067F9FEBD721001928A
:100FF000FF2AF7D81A0992B25B0F92001C40141B0B
:10100000DFE70B20EFE701339A00AE509C42FADA9B
:101010000020EAE7032BFBD12B0001335A1BA2422D
:10102000F6DC6A461279DA70F7E73968CB0706D53D
:101030004910002901DD8C4209DA1220D3E70D485E
:10104000FFF74AFC2100002801D11130CBE70F2324
:101050002A681340092B03D1013189004E51D7E78B
:10106000032BD5D16B461B796D18EB70D0E7C046CA
:1010700023CB000027CB000010B5012408682042D4
:101080001AD1042818D90F2102681140092901D169
:10109000406810BD032908D113099BB2500F9B0073
:1010A0000840181A40002043F3E7042904D102F055
:1010B000CBF9FFF791F8F5E70B2000F0FDF8E8E732
:1010C00010B5034A0B21034804F084F910BDC04653
:1010D000C4CA0000BCCA000000207047042070474A
:1010E0000120704710B5002002F0C2FB10BD0020A7
:1010F0007047002070470020704700207047002094
:1011000070470020704700207047002070470000A3
:1011100010B5034A0C21034804F05CF910BDC04629
:10112000ACCB00000CCC000010B50124044002D070
:101130004410200010BD042810D90F23026813406A
:10114000042B07D102F080F921000A220AF0F2FDF7
:101150000400EEE7032B01D10430F5E70D22014B2B
:101160001A70E6E7A4020020012210B5024018D14F
:10117000042802D903681A0992B201230B4012D144
:10118000042902D90B681B099BB20024934206D1A3
:1011900004309B000431C318984206D30124200078
:1011A00010BD0022E9E70023EFE704780A78002C5D
:1011B00001D1002AF2D0013001319442ECD0002458
:1011C000EDE70000F7B50700009101933049314B7E
:1011D000002A02D002220A70013A00261A601B6817
:1011E000CE54BE4200DBF7BD009AB300D058294B65
:1011F000274D1C68C8239B0065191C1B012318423E
:1012000006D0254A4310210028000AF053FC09E0CB
:10121000224A002802D004281BD1214A210028009C
:101220000AF048FC1A4C20000AF0BCFC194A019B49
:101230001060002B0BD07B1EB34208DD194B984287
:1012400005D8431C1360202222540022E2540136A8
:10125000C7E7042819D90F2301680B40042B04D1D8
:1012600002F0F2F8104A0300CDE7092B03D14368DE
:101270000E4A5B10C7E7032B08D10A0992B2490F47
:1012800092000B40D31A0A4ABDE70123094ABAE784
:10129000A5020020C805002020D500002CCB0000AE
:1012A00032CB00001F0300004BDB00007CCE0000AF
:1012B0008BCE000096CE0000014B187000207047C6
:1012C000A402002070B501F033FE094C0100251D79
:1012D0001F2228000AF07EFC28000AF063FC042389
:1012E00004308008000118432060200070BDC04613
:1012F00080020020C368F0B59D00836889B05D1945
:101300000300183306930369069A9F00069B029018
:10131000DF19436901939B00D3180393CD4B1B78CE
:10132000002B26D17F222B68CB491C1213409B0037
:101330005B58043501929F46029B587804F066FC86
:101340000023029A137027E0C24B1B78002B10D1A8
:101350002B68019A1C121340BF4A9B009B5804350E
:10136000E9E7069B3A1DD11ABA4BD82928DD1A2283
:101370001A70029BB74C9B6821780193EA1A029B72
:1013800092109B7812021A43029B587804F046FC94
:101390000023029A23701370029B069A9B680193A4
:1013A000ED1A029BAD10DD60069BFE1A029BB61083
:1013B0001E61039B9B1A029A9B10536109B0F0BDFA
:1013C0001B783C60002B01D01700D2E72B680199F5
:1013D0001C120B40A0499B005B5817000435AAE77C
:1013E000069B3A1DD11A9B4BD82902DD1A221A708E
:1013F000BFE728681B78291D3860002B02D0170032
:101400000D00B6E76B6801991C120B4092499B00D6
:101410005B58170008358EE7069B3A1DD11A8D4B95
:10142000D82902DD1A221A70A3E7A4001B782C1910
:101430003C60002B01D017009BE72B6801991C1220
:101440000B4085499B005B581700043573E7069BEA
:101450003A1DD11A7F4BD82902DD1A221A7088E76B
:101460007E49A40061581B783960002B01D0170019
:101470007FE72B6801991C120B4077499B005B5852
:101480001700043557E7043F744B3A68A400E25054
:10149000704B1B78002B00D06BE72B68019A1C1255
:1014A00013406D4A9B009B58043544E76B4BA400E6
:1014B000E058FFF739FE043F06003868FFF734FEB6
:1014C00036180120654B76000643E650614B1B78C9
:1014D000002B00D04DE72B68019A1C1213405E4A86
:1014E0009B009B58043526E7069B3A1DD11A594BA1
:1014F000D82902DD1A221A703BE70698039C0121C5
:10150000A04202D221000C3909681B783960002BF7
:1015100001D017002DE72B6801991C120B404E4992
:101520009B005B581700043505E7069B3A1DD11A4E
:10153000484BD82902DD1A221A701AE70699039837
:1015400081420FD203000C3B1B6845495B106418B5
:10155000E41AA40023583B603E4B1B78002B05D0B7
:10156000170006E7182119700023F4E72B6801998A
:101570001C120B4038499B005B5817000435DAE613
:10158000069B039A934219D213000C3B1B68344A02
:10159000043FA4185B10E31A039A39689B00995022
:1015A0002C4B1B78002B00D0E3E62B68019A1C1211
:1015B0001340294A9B009B580435BCE61822254B52
:1015C0001A70EDE7069B039A93422DD2244B3E1FDF
:1015D000E31814000C3C04932368049A5B10D31A9C
:1015E000039A9B009858FFF79FFD07903068FFF71C
:1015F0009BFD2468049B64101C1B079BA4001F1800
:1016000001207F00039B0743E7503700114B1B78F5
:10161000002B00D0ADE62B68019A1C1213400E4A35
:101620009B009B58043586E618220A4B1A70EDE79A
:10163000069B3A1DD11A074BD82902DD1A221A70CF
:1016400097E60399A40061581B783960002B09D0F4
:1016500017008EE6A40200207CCC0000842D002020
:10166000FDFFFF3F2B6801991C120B40D9499B00DD
:101670005B58170004355EE6043F039B3A68A400FC
:10168000E250D54B1B78002B00D072E62B68019AF4
:101690001C121340CF4A9B009B5804354BE6039B1A
:1016A000A4001C192368043F38685E10FFF73CFD56
:1016B00036180120C84B76001B7806432660002BA5
:1016C00000D056E62B68019A1C121340C14A9B00B9
:1016D0009B5804352FE6069BA4003F1BBE4CBB4223
:1016E0000CD82378002B00D043E62B68019A1C12FB
:1016F0001340B84A9B009B5804351CE6B74801F0DC
:1017000093FE2378002B00D033E62B68019A1C123D
:101710001340B04A9B009B5804350CE6A300ED181B
:10172000002C00DA38E6AC4B1B78002B00D020E60A
:101730002B68019A1C121340A64A9B009B58043543
:10174000F9E5043F3B68042B04D1A300ED18002CFD
:1017500000DA21E6A04B1B78002B00D009E62B68AD
:10176000019A1C1213409B4A9B009B580435E2E5EA
:10177000043F3B68042B04D0A300ED18002C00DAD2
:101780000AE6954B1B78002B00D0F2E52B68019AF6
:101790001C1213408F4A9B009B580435CBE53A1F1F
:1017A00013685B10013B06D401215B00A4000B43CE
:1017B0002D191360F0E5884B17001B78002B00D023
:1017C000D7E52B68019A1C121340824A9B009B5854
:1017D0000435B0E53A00069B0C32D31AD82B03DD52
:1017E0001A227D4B1A70C4E5FF2361005B0019408B
:1017F000FE3BFF3B19433960029906988968241221
:1018000004916D1A0299AD1089782D020D43039948
:101810009D40091A891099401D430B43BB60029BF0
:101820007D609C70E4B26E4BE4000392E358029A30
:101830009360694A1278002A03D008331D00039F81
:1018400097E51D00019A9B680C351C121340614AF4
:101850009B009B58039F6EE53B1F1C68039A069BE9
:1018600093422DD10A20E3070CD4042C13D90F2363
:1018700022681340042B11D1200001F0E5FD0AF08D
:1018800091F90630643003F0DFFD00280FD1043DEC
:10189000069B039380E50720042CF3D02000431E11
:1018A0009841FA234042FF3318400730EAE7029B91
:1018B0002100587804F0C4F90023029A1370E7E776
:1018C000039B039A0C3B1B6802995B109B00D31A85
:1018D0000C3B1C601F1D1300083B1B685A108A70CC
:1018E000D2B23F49D2005B0055589B0A029A9B0036
:1018F0009560ED18039B069A043B1B685B109B00E8
:10190000D3180393344B1B78002B00D031E52B68A0
:10191000019A1C1213402F4A9B009B5804350AE57C
:101920003B1F1868FFF700FCA40006003F1B1E28A1
:1019300027DC00280DDC284B1B78002B00D018E595
:101940002B68019A1C121340224A9B009B580435B5
:10195000F1E401F0DBFA033E361801F0D7FA214B2F
:10196000801B9842F9D81C4B1B78002B00D000E557
:101970002B68019A1C121340164A9B009B58043591
:10198000D9E40123029A137001F0C0FA029B0A38CD
:1019900086195E6000E53B1F1868FFF7C5FBA400D1
:1019A00006003F1B00280DDC0B4B1B78002B00D0E2
:1019B000DFE42B68019A1C121340064A9B009B58D7
:1019C0000435B8E4084B984210DD1D22024B1A7012
:1019D000CFE4C0467CCC0000A4020020A8CE0000CA
:1019E0008C2500203F420F0080EE36000123029A32
:1019F000137001F08BFAFA239B005E43029B0A3EB0
:101A000030185860C8E4A300FF1A002320001A0011
:101A10003900FFF7D7FBD44ED44C3168200001F0D9
:101A200033FFD34B31681860200003F0BDFF3168ED
:101A3000200004F00CF9CF4B1B78002B00D098E469
:101A40002B68019A1C121340CB4A9B009B5804350B
:101A500071E4C84BA4001B783F1B002B00D088E426
:101A60002B68019A1C121340C34A9B009B580435F3
:101A700061E4029803F04CFDBE4B1B78002B00D0B4
:101A800077E42B68019A1C121340BB4A9B009B58B9
:101A9000043550E43B1F1B68002B3ED13B000C3B40
:101AA0001B68DA072CD5390001225B105800083971
:101AB00002430A60002B44DD012259001143381F04
:101AC00001603900083909681141CB1A39000C3915
:101AD0000968114224D09B189340A4001343039A31
:101AE000A350A44B1B78002B00D042E42B68019A32
:101AF0001C121340A04A9B009B580435FFF71BFCA7
:101B0000042B06D90F211A680A40092A01D15B6803
:101B1000C9E71922974B1A702BE45B10013BC9E708
:101B2000042909D90F200A680240092A04D1023386
:101B30009B005B58A400D2E719228E4B1A70FFF766
:101B400018FC0435CDE7A300069AFB189B1AD82B86
:101B500013DC0122631E002C14DC864B1B78002B47
:101B600001D0FFF706FC2B68019A1C121340824A31
:101B70009B009B580435FFF7DEFB1A227D4B1A7041
:101B8000FFF7F7FB3A601C000437E3E7069A3B1DBA
:101B90009B1A784ED82B03DD1A233370FFF7E9FB2D
:101BA000069B039AA40093422AD23B1F1868FFF7B2
:101BB000BBFA011E21DD039B0C3B1A6852108242C6
:101BC0001BDB9007801A6D4B4018C018039B8000E8
:101BD000C2583B1B1A60674B3F1B1B780437002B16
:101BE00001D0FFF7C6FB2B68019A1C121340624A12
:101BF0009B009B580435FFF79EFB20233370EAE7D8
:101C00001823FBE75A4BA4001A683B1B1F001A60FD
:101C1000584B04371B78002B01D0FFF7AAFB2B6829
:101C2000019A1C121340544A9B009B580435FFF73D
:101C300082FB3B1F1A68042A11D1A4002D194D4BB9
:101C40001B78002B01D0FFF794FB2B68019A1C1224
:101C50001340494A9B009B580435FFF76CFB1F005B
:101C6000EDE73A1F1368042B04D0002313603A00F9
:101C7000A4002D193F4B1B78002B02D01700FFF753
:101C800078FB2B6801991C120B403B499B005B5869
:101C900017000435FFF74FFBA3009C46FE1A002CEB
:101CA00017DC1C22334B1A70002333606346FF1A83
:101CB000304B04371B78002B01D0FFF75AFB2B6801
:101CC000019A1C1213402C4A9B009B580435FFF7C5
:101CD00032FB002033685A108300F15801230B4077
:101CE00003D10D21234A1170DFE749108A4200DD3C
:101CF0000A0001308442EFDC012352001343D4E791
:101D0000A3009C46FE1A002C17DC1C22194B1A70EB
:101D1000002333606346FF1A164B04371B78002BF1
:101D200001D0FFF726FB2B68019A1C121340124AC0
:101D30009B009B580435FFF7FEFA002033685A10C9
:101D40008300F15801230B4003D10D21094A117082
:101D5000DFE749108A4200DA0A0001308442EFDCF2
:101D6000012352001343D4E7C8050020A502002038
:101D700008000020A40200207CCC0000FCFFFF3FF4
:101D80003B00083B1868FFF7CFF93B1F06001868B7
:101D9000FFF7CAF90023864200DA0433A4003A1B95
:101DA00017001360E54B04371B78002B01D0FFF7B9
:101DB000E0FA2B68019A1C121340E14A9B009B58E1
:101DC0000435FFF7B8FA3B00083B1868FFF7ACF999
:101DD0003B1F06001868FFF7A7F9F30FC217B042C0
:101DE0005341A4003A1B17009B001360D34B0437E8
:101DF0001B78002B01D0FFF7BCFA2B68019A1C124C
:101E00001340CF4A9B009B580435FFF794FA3B00E0
:101E1000083B18683B1F1968A600BE1B04238142BB
:101E200002D0042802D80023336018E001239C4626
:101E30001842F8D10F2302681A40042AF3D16346EE
:101E40001942F0D10429EED90B680B321340042B50
:101E5000E9D1FFF789F9431E984180003060B74B04
:101E6000A4001B783F1B0437002B01D0FFF781FA39
:101E70002B68019A1C121340B14A9B009B580435F1
:101E8000FFF759FA3B00083B18683B1F1968A6008A
:101E9000BE1B0023814202D0042802D804233360F1
:101EA00018E001239C461842F8D10F2302681A401B
:101EB000042AF3D163461942F0D10429EED90B6804
:101EC0000B321340042BE9D1FFF74EF9434258413E
:101ED00080003060994BA4001B783F1B0437002B17
:101EE00001D0FFF746FA2B68019A1C121340944A5E
:101EF0009B009B580435FFF71EFA3B00083B18680F
:101F0000FFF712F93B1F06001868FFF70DF9F317EA
:101F1000C20F86425341A4003A1B17009B00136076
:101F2000864B04371B78002B01D0FFF722FA2B6871
:101F3000019A1C121340824A9B009B580435FFF7FC
:101F4000FAF93B00083B1868FFF7EEF83B1F060064
:101F50001868FFF7E9F80023864200DD0433A40087
:101F60003A1B17001360754B04371B78002B01D008
:101F7000FFF7FFF92B68019A1C121340704A9B006F
:101F80009B580435FFF7D7F93B1F1B68A400043B9F
:101F90005A1E93413A1B17009B001360674B04378E
:101FA0001B78002B01D0FFF7E4F92B68019A1C1273
:101FB0001340634A9B009B580435FFF7BCF93B0074
:101FC000083B1868FFF7B0F83B1F06001868FFF7DA
:101FD000ABF832180120A4003B1B1F005200024343
:101FE0001A60564B04371B78002B01D0FFF7C1F95C
:101FF0002B68019A1C121340514A9B009B580435D0
:10200000FFF799F93B00083B1868FFF78DF83B1F75
:1020100006001868FFF788F8321A0120A4003B1B5D
:102020001F00520002431A60444B04371B78002BF8
:1020300001D0FFF79EF92B68019A1C121340404A09
:102040009B009B580435FFF776F93B00083B186866
:10205000FFF76AF83B1F06001868FFF765F80200F3
:102060000120A4003B1B1F007243520002431A6070
:10207000324B04371B78002B01D0FFF77AF92B681D
:10208000019A1C1213402E4A9B009B580435FFF7FF
:1020900052F93B1F1868FFF747F8061E17D11F2398
:1020A000264A1370A4003B1B1F001E60234B0437FD
:1020B0001B78002B01D0FFF75CF92B68019A1C12EA
:1020C00013401F4A9B009B580435FFF734F93B002F
:1020D000083B1868FFF728F8310007F095F801264B
:1020E00040000643DEE73B1F1868FFF71DF8061E99
:1020F00017D11F23114A1370A4003B1B1F001E6041
:102100000E4B04371B78002B01D0FFF732F92B68F8
:10211000019A1C1213400A4A9B009B580435FFF792
:102120000AF93B00083B1868FEF7FEFF310007F094
:1021300051F9012649000E43DEE7C046A402002003
:102140007CCC00003B1F1868FEF7EEFFC21780181A
:1021500050400122A4003B1B1F00400010431860A8
:10216000F14B04371B78002B01D0FFF702F92B68E5
:10217000019A1C121340ED4A9B009B580435FFF74F
:10218000DAF8A300FE1A3068012C24D1FEF7CCFF48
:102190000494079009F05CFC0799002900DC0121F8
:1021A00007F018F9049BA400C9180123490019433A
:1021B000DD4B3F1B1B7831600437002B01D0FFF74C
:1021C000D8F82B68019A1C121340D84A9B009B58E0
:1021D0000435FFF7B0F8FEF7A7FF04907068FEF72C
:1021E000A3FF049B0130C31A0793D3E7A300FE1A91
:1021F00031002000049301F0CDFC049B3060FF1AF5
:10220000C94B04371B78002B01D0FFF7B2F82B68BD
:10221000019A1C121340C54A9B009B580435FFF7D6
:102220008AF83B00083B1868FEF77EFF3B1F06005C
:102230001868FEF779FF02000120A4003B1B1F0075
:102240003240520002431A60B74B04371B78002B10
:1022500001D0FFF78EF82B68019A1C121340B34A85
:102260009B009B580435FFF766F83B00083B186855
:10227000FEF75AFF06003B1F1868FEF755FF3200B5
:1022800002430120A4003B1B1F00520002431A60BE
:10229000A54B04371B78002B01D0FFF76AF82B6899
:1022A000019A1C121340A14A9B009B580435FFF76A
:1022B00042F83B00083B1868FEF736FF06003B1F5C
:1022C0001868FEF731FF320042400120A4003B1B9A
:1022D0001F00520002431A60934B04371B78002BF7
:1022E00001D0FFF746F82B68019A1C1213408F4A61
:1022F0009B009B580435FFF71EF83B1F1868FEF73C
:1023000013FFC0430122A4003B1B1F0040001043E9
:102310001860854B04371B78002B01D0FFF729F894
:102320002B68019A1C121340804A9B009B5804356D
:10233000FFF701F83B00083B1868FEF7F5FE0600C2
:102340003B1F1868FEF7F0FE320082405100012268
:10235000A4003B1B1F000A431A60734B04371B7811
:10236000002B01D0FFF705F82B68019A1C121340CF
:102370006E4A9B009B580435FEF7DDFF3B00083B8F
:102380001868FEF7D1FE06003B1F1868FEF7CCFE6A
:102390003200024151000122A4003B1B1F000A43EE
:1023A0001A60614B04371B78002B01D0FEF7E1FF68
:1023B0002B68019A1C1213405C4A9B009B58043501
:1023C000FEF7B9FF3B000C3B1868FEF7ADFE3B0083
:1023D000083B06001868FEF7A7FEF1170200C317B6
:1023E000300007F049F83B1F049005911868FEF78C
:1023F0009BFE02000498059906F0F2FF43000120BD
:10240000A4003E1B37001843474B30601B7804374D
:10241000002B01D0FEF7ADFF2B68019A1C12134070
:10242000424A9B009B580435FEF785FFA300FE1A25
:10243000310020000493FEF7C1FC049B3060FF1ABA
:10244000394B04371B78002B01D0FEF792FF2B6825
:10245000019A1C121340354A9B009B580435FEF725
:102460006AFFA300FF1A39002000FEF7BFFC2E4BC5
:102470001B78002B01D0FEF77CFF2B68019A1C1201
:1024800013402A4A9B009B580435FEF754FFA300D3
:10249000FE1A310020000493FEF7E8FC049B306034
:1024A000FF1A214B04371B78002B01D0FEF761FF88
:1024B0002B68019A1C1213401C4A9B009B58043540
:1024C000FEF739FFA300FF1A39002000FEF762FD76
:1024D000154B1B78002B01D0FEF74BFF2B68019AA0
:1024E0001C121340114A9B009B580435FEF723FF32
:1024F000A300FE1A310020000493FEF7BDFD049BEB
:102500003060FF1A084B04371B78002B01D0FEF710
:1025100030FF2B68019A1C121340044A9B009B5801
:102520000435FEF708FFC046A40200207CCC000062
:102530003B1F186800F088FF3A00083A1268030051
:10254000A400D10729D4042A0CD910680F22104006
:10255000013808280FD806F0B9FD052026220E0EF6
:102560000E0E2400EE49180009F012FB43425841B8
:102570003B1B80001860EB4B3F1B1B780437002B84
:1025800001D0FEF7F6FE2B68019A1C121340E64AB2
:102590009B009B580435FEF7CEFEE449E3E7E4498F
:1025A000E1E7E449DFE7E449DDE7069B3E1DF31A76
:1025B000DC4CD82B03DD1A232370FEF7DAFE00F083
:1025C000AFFC43000120184323783860002B02D071
:1025D0003700FEF7CEFE2B68019A1C121340D24A38
:1025E0009B009B5837000435FEF7A5FE069B3E1D59
:1025F000F31ACC4CD82B03DD1A232370FEF7B9FE57
:1026000000F084FCCD4B4000184001231843237890
:102610003860002B02D03700FEF7ABFE2B68019A22
:102620001C121340C04A9B009B5837000435FEF72C
:1026300082FE0123A600BE1B20001A003100FEF717
:10264000C1FDBF4C2068643002F0FEFE002802D1BC
:10265000043DFEF7A1FE029B21685A78B94803F0B9
:1026600004FB0123029A3700137000F04FFCB64BB5
:1026700022681B68063253431818029B5860FEF705
:102680008BFEA600BE1B2000012300223100FEF7B6
:1026900099FDAB4C2068643002F0D6FE0028D7D0FC
:1026A000A84803F071F8DCE7A4003E1BFEF70AFE21
:1026B00037009C4B30601B780437002B01D0FEF7AD
:1026C00058FE2B68019A1C121340974A9B009B5896
:1026D0000435FEF730FE934BA4001B783F1B002B04
:1026E00001D0FEF746FE2B68019A1C1213408E4A59
:1026F0009B009B580435FEF71EFEA4003E1B3000D5
:1027000000F03DFC3700874B30601B780437002B0E
:1027100001D0FEF72EFE2B68019A1C121340824A4C
:102720009B009B580435FEF706FEA4003E1B3000BC
:1027300000F027FC37007B4B30601B780437002B00
:1027400001D0FEF716FE2B68019A1C121340764A40
:102750009B009B580435FEF7EEFDA300FE1A3100E6
:102760002000049300F010FC049B3060FF1A6D4BB6
:1027700004371B78002B01D0FEF7FBFD2B68019A74
:102780001C121340684A9B009B580435FEF7D3FD8A
:10279000A4003F1B380000F029FC624B1B78002B83
:1027A00001D0FEF7E6FD2B68019A1C1213405E4A29
:1027B0009B009B580435FEF7BEFDA300FE1A3100B6
:1027C0002000049300F03AFC049B3060FF1A554B44
:1027D00004371B78002B01D0FEF7CBFD2B68019A44
:1027E0001C121340504A9B009B580435FEF7A3FD72
:1027F000A4003F1B380000F063FC4A4B1B78002B01
:1028000001D0FEF7B6FD2B68019A1C121340464A10
:102810009B009B580435FEF78EFD0121200000F03F
:1028200037FC404B1B78002B01D0FEF7A2FD2B6834
:10283000019A1C1213403C4A9B009B580435FEF73A
:102840007AFD0021200000F023FC364B1B78002B82
:1028500001D0FEF78EFD2B68019A1C121340324AFC
:102860009B009B580435FEF766FDA4003E1B30001C
:1028700000F048FC37002B4B30601B780437002BEE
:1028800001D0FEF776FD2B68019A1C121340264AF0
:102890009B009B580435FEF74EFDA4003E1B300004
:1028A00000F044FC37001F4B30601B780437002BCE
:1028B00001D0FEF75EFD2B68019A1C1213401A4AE4
:1028C0009B009B580435FEF736FDA4003F1B3800E3
:1028D00000F006FC134B1B78002B01D0FEF749FDDE
:1028E0002B68019A1C1213400F4A9B009B58043519
:1028F000FEF721FDA4003F1B380003F0D1FC094B7B
:102900001B78002B01D0FEF734FD2B68019A1C12B6
:102910001340054A9B009B580435FEF70CFDC0464A
:10292000B8CE0000A40200207CCC0000C0CE000085
:10293000C7CE0000CECE0000D3CE0000FEFFFF7F4A
:10294000C8050020A502002004000020A4003E1BB2
:10295000300003F03FFD3700CD4B30601B7804376B
:10296000002B01D0FEF705FD2B68019A1C121340C5
:10297000C84A9B009B580435FEF7DDFCA4003F1BB2
:10298000380003F03DFCC24B1B78002B01D0FEF752
:10299000F0FC2B68019A1C121340BE4A9B009B5806
:1029A0000435FEF7C8FCA4003E1B300003F03EFCDB
:1029B0003700B74B30601B780437002B01D0FEF78F
:1029C000D8FC2B68019A1C121340B24A9B009B58FA
:1029D0000435FEF7B0FCA300FF1A3900200001F017
:1029E000F7FBAB4B1B78002B01D0FEF7C2FC2B682A
:1029F000019A1C121340A74A9B009B580435FEF70E
:102A00009AFCA300FF1A3900200001F017FAA04B2E
:102A10001B78002B01D0FEF7ACFC2B68019A1C122E
:102A200013409C4A9B009B580435FEF784FCA3008E
:102A3000FF1A3900200001F003FB954B1B78002B97
:102A400001D0FEF796FC2B68019A1C121340914AA4
:102A50009B009B580435FEF76EFCA300FF1A39005B
:102A6000200001F015FB8A4B1B78002B01D0FEF7EC
:102A700080FC2B68019A1C121340864A9B009B58CD
:102A80000435FEF758FCA300FE1A31002000049321
:102A900003F038FD049B3060FF1A7D4B04371B7830
:102AA000002B01D0FEF765FC2B68019A1C12134025
:102AB000784A9B009B580435FEF73DFCA300FE1AA4
:102AC00031002000049303F025FD049B3060FF1AC1
:102AD0006F4B04371B78002B01D0FEF74AFC2B68A4
:102AE000019A1C1213406B4A9B009B580435FEF759
:102AF00022FCA300FE1A31002000049303F012FD13
:102B0000049B3060FF1A624B04371B78002B01D006
:102B1000FEF72FFC2B68019A1C1213405D4A9B00A4
:102B20009B580435FEF707FCA300FE1A3100200075
:102B3000049303F01DFB049B3060FF1A544B0437D1
:102B40001B78002B01D0FEF714FC2B68019A1C1295
:102B50001340504A9B009B580435FEF7ECFBA30042
:102B6000FF1A3900200001F0A1F9494B1B78002B16
:102B700001D0FEF7FEFB2B68019A1C121340454A58
:102B80009B009B580435FEF7D6FBA300FF1A3900C3
:102B9000200001F0A5FA3E4B1B78002B01D0FEF778
:102BA000E8FB2B68019A1C1213403A4A9B009B5881
:102BB0000435FEF7C0FBA300FE1A31002000049389
:102BC00001F00AFA049B3060FF1A314B04371B787E
:102BD000002B01D0FEF7CDFB2B68019A1C1213408D
:102BE0002C4A9B009B580435FEF7A5FBA300FF1A57
:102BF0003900200001F0B8F9254B1B78002B01D0DB
:102C0000FEF7B7FB2B68019A1C121340214A9B0068
:102C10009B580435FEF78FFB069B029AFB1A9B100C
:102C20001361A300FF1A3900200002F0EBFD184BDE
:102C30001B78002B01D0FEF79CFB2B68019A1C121D
:102C40001340144A9B009B580435FEF774FB069B07
:102C5000029AFB1A9B101361A300FE1A3100200098
:102C6000049302F0CFFD049B3060FF1A084B043739
:102C70001B78002B01D0FEF77CFB2B68019A1C12FD
:102C80001340044A9B009B580435FEF754FBC04692
:102C9000A40200207CCC00000023F7B55A1E01924C
:102CA000002B07DA01F0AAFA02F0DCFE03F03CF890
:102CB0001923019300263000194B1968B14212DD27
:102CC000184B1A6801328A420FDAF0241A601D6824
:102CD000154F6C43E35D002B1FD0E419022B06D186
:102CE0002000FEF707FB019BD8E70022EDE7012B50
:102CF0000DD1002801D100F009F9F0226A43BB1878
:102D00005B680A49C31A8B4201D80223BB54F023E3
:102D10005D43054BEB5C022BE2D00136CCE7C046AD
:102D2000CC050020000000202C1C00203F420F009A
:102D3000012200210A4B0B481A6119500430195026
:102D4000A2210420C9005850C121C020890080025E
:102D500058501A60044BFC311960044B1A707047CC
:102D600000A000400405000000E100E0F3050020A1
:102D700004207047F8B550C9012322001A40101EE4
:102D80002DD03340181E2AD0641000201C2C26D8C9
:102D90001D4B761035009E4200DD1D001B4F3B5D34
:102DA000012B05D00121200004F04AFD01233B55F1
:102DB000174B1B78002B01D1FFF7BAFF0023154AF0
:102DC0009E420DDCFF2514491448D65CB44202D162
:102DD0005E007052D5540133042BF6D10420F8BDA7
:102DE000D15C8C4203D10C4A5B009D52F6E7013363
:102DF000042BF5D10023D15CFF2901D1D454F2E793
:102E00000133042BF7D1E9E788130000D405002033
:102E1000F30500201C0000200E000020DC0500004F
:102E2000F8B530C9012623003340181E1BD02B00F3
:102E30003340181E17D0344100201C2C13D8174FD4
:102E40003B5DB34204D03100200004F0F9FC3E5554
:102E500069100800124A1038124B904204D901221E
:102E600052421A600420F8BD1C600F4806F0CCF9ED
:102E70000E4B18800E4B1B78002B02D1FFF758FF2A
:102E8000F0E701220B4B9A64A922D2009A588018CD
:102E9000A82280B2D2009850E4E7C046D4050020B2
:102EA000908601001800002020A107000C000020DF
:102EB000F305002000A00040030010B50120002B06
:102EC00002DC1B30FEF7F8F910BD0420704710B586
:102ED000002803DC1C20FEF7EFF910BD0B68002072
:102EE000DB07FAD40D30F6E701220020054B064936
:102EF0001A61585004310330585008318018585026
:102F00001A60704700800040040500000122034B56
:102F10001A64A822D20098587047C046008000402A
:102F200010B5FFF7F3FFFA21890006F0E3F810BDB2
:102F30000048704730CF00001D20704770B5054E27
:102F40000400335C0D008B4202D004F079FC35554F
:102F500070BDC046D405002070B50024064D635DE9
:102F6000012B05D10021200004F06AFC00236355E9
:102F700001341D2CF2D170BDD405002070470D2006
:102F800070473B2070470000F8B501240B6806002D
:102F90000D00234204D10D20FEF78EF92000F8BD6C
:102FA0005B102000052BFAD80E4A9B009C580E4F50
:102FB0003B5D002B05D00021200004F041FC0023E4
:102FC0003B55012E06DD6B68042B03D10221200046
:102FD00004F036FC200004F0E1FA01244000204314
:102FE000DDE7C04618CF0000D4050020F8B5012663
:102FF0000568354202D04468344203D10D20FEF703
:103000005BF9F8BD6D101C2DFBD80A4F7B5D012BC1
:1030100004D03100280004F013FC7E5506496410EA
:103020008C4202DCE143C9172140280004F03CFB3C
:10303000E7E7C046D4050020FF03000070B5012477
:103040000D68254204D10D20FEF736F9200070BD31
:103050006D101C2D17D80024012804DD4C68043C99
:1030600063425C416400094E735DA34204D02100B9
:10307000280004F0E5FB7455280004F015FC03005B
:103080000420012BE3D00020E1E7C046D405002056
:1030900070B504000D001C280ED8084E335C012BBF
:1030A00004D0012104F0CCFB01233355290020007A
:1030B0004D1EA94104F0E2FB70BDC046D4050020BE
:1030C000036810B5DA0703D40D20FEF7F5F810BD3C
:1030D0004168581004394A425141FFF7D9FFF6E7D9
:1030E00037B569460A00064B30CB30C20368022070
:1030F000042B02D100F0A4FF37BD00F0C9FFFBE7AD
:10310000E0CE000010B5084C6379002B05D00021FB
:10311000052004F095FB00236371052004F0C4FB37
:1031200043425841800010BDD405002010B5084C22
:10313000E37A002B05D000210B2004F081FB002353
:10314000E3720B2004F0B0FB43425841800010BDF5
:10315000D4050020F7B5304D304E6B6C002B15D0E8
:10316000A8240023E40037596B642D4B186800280D
:103170000CDB2C4B19784A425141C9B2197004F04A
:103180007DFB294B1B88DF19BFB23751AB6C002B7D
:1031900039D00021254B264FF458A9643A780C34D5
:1031A0000193244D8A4206D02B68032B03D8224A70
:1031B000D05C04F063FB2B68204A0133134004D534
:1031C0000422013B5242134301331B4900228C4627
:1031D0002B60042B18D06046C05C591CFF2802D11C
:1031E0000B000122F5E7002A00D02B60012104F03A
:1031F00045FB01233B702B68114A5B009B5AE41886
:10320000019BA4B2F450F7BD01235B422B60002365
:103210003B700C4BF3E7C046FCA0004000A0004010
:1032200018000020F20500200C00002044050000DA
:10323000F1050020D00500201C00002003000080C4
:103240000E00002050460000084B094AFF201A805B
:103250005A809A80DA800023064A07491370074A89
:10326000087048708870C870136070470E000020A6
:10327000DC050000F10500201C000020D005002026
:103280000122024B52421A607047C04618000020CB
:1032900010B5034A0621034802F09CF810BDC04651
:1032A000E8CE000052D60000E12170B54902144872
:1032B00003F06CFFFFF718FE0A2004F069F9002301
:1032C000FF21104A995401331D2BFBD1012200200C
:1032D0000D4B01001A6004230C4A0D4D1468002C9C
:1032E000FCD02C680002013B20431160002BF5D17B
:1032F0000122084B1A6004F005F901F0CBF870BD0B
:10330000B41B0020D405002000D0004000D10040B4
:1033100008D5004004D00040F8B50B4E070030003F
:103320000D0003F07BFF0400A84200DD2C003D00EF
:10333000EB1B9C4205DD300003F07AFF287001355D
:10334000F6E72000F8BDC046B41B002010B5010010
:10335000014803F023FF10BDB41B002010B5054C3D
:10336000200003F029FFE1212000490203F00EFFB5
:1033700010BDC046B41B0020C3070CD4064B1B680D
:10338000834208D8054B1B68984204D8031F1B686A
:10339000002B00D018007047FC050020F805002025
:1033A0000023012210B50A48990001334250642BD2
:1033B000FAD1084C084B00211A602000074A08F097
:1033C00067F8074B074A6360074B1A6010BDC04699
:1033D000842D00200006002008000020D4090000F1
:1033E0003027000004060020F405002010B5044B2F
:1033F000044A1A60044B054A1A60FFF7D1FF10BD5A
:10340000FC05002000060020F8050020D40F002055
:10341000044B1B681868000980B20238C343DB17ED
:1034200018407047F405002000B59BB00200054924
:1034300001A808F071FB01A802F0C2F902F074FCC7
:10344000FCE7C046B4CF00000B4BC20704D40428ED
:1034500004D80A4B00D00A4B180070470F220368AB
:103460001A40031D042AF7D0064B092AF4D0064B54
:10347000032AF1D0054BEFE78ECF000032CB0000DE
:103480002CCB000098CF0000A8CF00009FCF0000F9
:103490000020064A0649131F186013681B099BB2D7
:1034A00002339B00D2188A42F5D3704704060020ED
:1034B000D40F0020F7B50F240126314B314A19688B
:1034C000314B324D186813681F002740072F26D84C
:1034D00013681B099BB202339B00D218AA42F2D395
:1034E00000242B4EA500AD192868FFF745FF0134D5
:1034F0002860642CF6D1274C2068FFF73DFF206040
:10350000254C2068002802D0FFF736FF20600025F8
:10351000224B1B680093009B9D4214DBF7BD1B09E7
:103520009BB29B00D3189A42D2D01F68374208D171
:10353000B94206D2B84204D3043F3F68002F00D0FE
:103540001F60043BEFE7F0236B43154A9B181A7882
:10355000002A01D10135DEE71F693C2300266B43B9
:10356000DB199B0001930136BB1BF3D4019BB40014
:103570001C1B0B4B1C19A069FFF7FEFEA061F2E7B4
:10358000FC05002004060020F8050020D40F0020D0
:10359000842D002008000020D40F0020CC0500203E
:1035A0002C1C0020F7B50124204246D1234B1B6878
:1035B0009C46984241D3224B1B68019398423CD8C9
:1035C000031F1B68002B38D10200036800941B09FD
:1035D0009BB2002B0FD10099131F196090422CD081
:1035E00015682B1F1B68990069180C68013B146053
:1035F0000A602A00EDE79D0055192968009C2142C8
:1036000019D18C4517D8019C8C4214D30E1F3468F5
:10361000002C10D10F680F343C40072C08D92F60C4
:10362000151F2B600B680A601B099BB20A00D0E7CC
:1036300000993160CDE7013BCBE7F7BDFC050020E9
:10364000F80500200D4970B50A000D4D1368141FD0
:103650001B0926689BB2981C002E0BD000238A42BF
:1036600000D00B0023608300C91880001218AA4202
:10367000ECD370BD1B011360F7E7C04604060020C1
:10368000D40F0020F8B5124C27000F223B681D090B
:10369000ADB213420DD06E1CB600A74204D032006A
:1036A0003900200007F0E1FE0022A3190436A41916
:1036B0001A600235AD00074B7F199F42E5D31B1BF3
:1036C0009B10013B1B012360034B1C60F8BDC046EF
:1036D00004060020D40F0020F4050020F0B59BB0B4
:1036E000FFF714FC00240700214AA300D05801343E
:1036F000FFF758FF642CF7D11E4B1868FFF752FFF5
:103700001D4B1868002801D0FFF74CFF00261B4B0B
:103710001B689E4217DBFFF795FFFFF7CBFEFFF715
:10372000B1FFFFF7F3FB164BC21B1B6815491B6863
:1037300001A81B099BB2023B08F0EEF901A802F0B8
:103740003FF81BB0F0BDF02575430F4BED182B78FB
:10375000002B01D10136DAE72B695C1E002CF9DB66
:10376000A300EB189869FFF71DFF013CF6E7C04680
:10377000842D002008000020D40F0020CC0500205C
:10378000F40500206ECF00002C1C0020F7B5174D6B
:103790004F1C2B6806001B680C001B099BB2019292
:1037A0009F420BDBFFF79AFF2B681B681B099BB23C
:1037B0009F4203DB0A20FDF77FFDFEBD2868A71CA2
:1037C000BA00DB1B81181B010B6029600021031F5D
:1037D00019600F231E4003002401264340C3083A0A
:1037E0009A189A42E9D9019902C3FAE7F405002030
:1037F000F7B503000122134004000D000193002BD4
:103800002BD1174B1B68834227D8164B1B6883426A
:1038100023D90F23144F386000681840FFF7B6FF14
:10382000019B3C68061E3B6017D0236804301B09CF
:103830009BB29D4200DD1D00AA00211D251F07F03F
:103840000BFEFFF725FE2E60FFF734FE00232B60F2
:103850002268064B1340236034002000FEBDC046A2
:10386000FC050020F8050020D40F0020F0FF0F0019
:103870000323043010B5C11719400918891000221C
:103880000420FFF783FF10BD70B5050008000C0091
:10389000FFF7EEFF0023002804D170BDE95CC218D9
:1038A00011710133A342F9DBE343DB171C40002312
:1038B00004192371F1E7F0B50C009BB0022804DC79
:1038C0001C20FDF7F9FC1BB0F0BD0123086818426D
:1038D00006D1042804D90F2601683140042901D0FB
:1038E0000E20EEE761680D001D40F9D10429F7D9DB
:1038F0000A683240042AF3D1A2681A4201D10D208D
:10390000DFE7FFF7A1FD06006068FFF79DFDA768F0
:10391000010001AC7F103000257002F0E2FF390099
:103920006423220003F042F8200008F03BF9010074
:103930002000FFF7A9FFC6E710B51C4CA544041EE4
:1039400002D1FFF795FF0BE002F0E4FE01380628F4
:1039500028D805F0BBFB0909111829042400002010
:103960008023DB009D4410BD200002F04FFF011BAF
:103970002000FFF789FFF3E7200002F0F5FE430087
:1039800001201843ECE780226946D200200002F0B3
:1039900002FF684608F006F901006846E9E70421DD
:1039A0000348E6E70020CCE70420D9E700FCFFFF4E
:1039B000FCCF000070B50C00022803DC1C20FDF7D2
:1039C0007BFC70BD01230868184206D1042804D985
:1039D0000F2501682940042901D00E20EFE7616816
:1039E0001942FAD10429F8D90A682A40042AF4D1E4
:1039F000A2681A4201D10D20E1E7FFF725FD05007D
:103A00006068FFF721FDA46801006410280002F03F
:103A100068FF210002F0A5FFFFF78EFFD1E770B528
:103A20000D00012803DC1C20FDF746FC70BD0124BD
:103A30000868204206D1042804D90F2102680A40F0
:103A4000042A01D00E20EFE76A682242FAD1042A44
:103A5000F8D913680B40042BF4D1FFF7F5FC0600EE
:103A60006868FFF7F1FC0100300002F03AFF02F055
:103A7000BCFF40002043D9E7F8B507000C001C202C
:103A8000012F0BDD01250868284206D1042804D93E
:103A90000F2102680A40042A03D00E20FDF70CFC17
:103AA000F8BD62682A42F8D1042AF6D913680B409F
:103AB000042BF2D1FFF7C8FC06006068FFF7C4FCD6
:103AC0000100022F14D0A4682C4211D064103000E1
:103AD00002F007FF050002F01DFE012811D1002CA5
:103AE00002DD0135012C06D12800FFF725FFD7E7BD
:103AF00001246442EBE7280002F094FE013C05003B
:103B0000F0E70228F0D1002CEEDD0135012CEBD0DE
:103B100000222800110002F0B7FE02F083FE013CF3
:103B20000500F3E710B501240868044016D04410DE
:103B3000200005F0FDFD154905F0C8FC07F0AEFBBF
:103B400003F0F6FF0022124B06F062FD03F098FF2F
:103B500007F034FB43000120184310BD042810D99E
:103B60000F2302681340042B07D1FFF76DFC2100DF
:103B70000A2208F0DFF80400DAE7032B01D1043051
:103B8000F5E70D20FDF798FBD2E7C046D3023739A1
:103B90000000D040086870B501240500254006D11A
:103BA000042804D90F2302681340042B03D00E20ED
:103BB000FDF782FB70BDFFF747FC03782900233B2C
:103BC0005A4253411022C01808F0B4F880239B05D4
:103BD000C218044B9A4201D91420E9E7400020435F
:103BE000E8E7C046FFFFFF3F10B5034A0621034840
:103BF00001F0F0FB10BDC046CCCF0000C5CF0000E7
:103C00000020704710B51E20FDF756FB10BD10B503
:103C10001E20FDF751FB10BD10B51E20FDF74CFB1B
:103C200010BD10B51E20FDF747FB10BD10B51E20BE
:103C3000FDF742FB10BD10B51E20FDF73DFB10BD8A
:103C400010B51E20FDF738FB10BD10B51E20FDF786
:103C500033FB10BD10B51E20FDF72EFB10BD10B5B7
:103C60001E20FDF729FB10BD10B5034A0B210348A8
:103C700001F0B0FB10BDC04638D0000090D000006D
:103C80000120034B1860034B1B68834018437047A7
:103C9000F80F0020D80F0020F0B5EFF310810123BA
:103CA000194083F31088134C134AA4461268134E2C
:103CB000013A9340124F134A002B17D01468034265
:103CC0000FD03D682C60C046C046C046C046C046C6
:103CD000C046C046C0460C4C1568246825605B0889
:103CE000EAE765462C6014683460F8E781F31088D1
:103CF000F0BDC04608050050200000200C05005013
:103D0000E40F0020EC0F0020E00F002030B585B05C
:103D100001AD0C220649280007F09EFB0024285D17
:103D200001210134FFF70AF90C2CF8D105B030BDA0
:103D300025D10000F7B56A46394B01AD13801C232D
:103D40009370384B2B800A23AB70FFF7DFF8364BAC
:103D5000364CC0182368984201D20023236026689D
:103D6000002E3DD16B469F5D01213800FFF7E6F83C
:103D700001360021380003F081FD032EF2D1002628
:103D8000AF5D01213800FFF7D9F801360121380075
:103D900003F074FD032EF3D1C8200138C046C0469D
:103DA000C046C046C046C046C046C046C046C046E3
:103DB000C046C046F1D100212878FFF7BFF86878E7
:103DC0000021FFF7BBF8A8780021FFF7B7F8FFF74D
:103DD0009DF8FA2300251B01C01820602800FEBDB5
:103DE000FFF794F8236800259842F7D3032003F0E7
:103DF000D5FB0600042003F0D1FB36180A2003F09F
:103E0000CDFB0B4B9B1B181A0A4BA84206DB186014
:103E10000023094A236013600125DFE71D60F7E7EF
:103E20001A1B00000304000010270000F00F002000
:103E3000E3030000D80F0020F80F00200022054BFC
:103E400010B51A60044B1B68934201D002F002FCCB
:103E5000002010BDF40F0020D81A002010B5041E59
:103E600010DA00240A4BA400E25801239340094AC7
:103E700009491360094A1160094A0A4911600A4A4E
:103E8000136010BDFFF758F8A042EADDEAE7C0462C
:103E900028DE0000EC0F002008050050E40F002091
:103EA000E00F00200C050050180500502B4BF7B513
:103EB0001B680C00002B03D101204042FFF7CEFF0E
:103EC00024680126250035401AD0FF226310120213
:103ED00060121040DAB21043FF221B02120413409A
:103EE00018431F4B1B68202B06D1B4401D4BA40E5A
:103EF000A400E35800021843FFF7CEFE0020FEBDE9
:103F0000042CFBD90F2322681340092BF6D1FF277D
:103F100063683F025B100193019B9D42EEDAAB00A8
:103F2000E3189B68334216D05A105812D1B2384069
:103F30000843FF21120209040A401043084A12688C
:103F4000202A06D15B009B0E06499B0002025858AE
:103F50001043FFF7A1FE0135DEE7C046EC0F00205D
:103F6000200000200CD300000200086810B5C30731
:103F70000FD540101823012A03DD4A68042A00D116
:103F80000833054A1360FEF7F9FFFFF767FF0020CB
:103F900010BD01204042EDE72000002010B50124B3
:103FA000044002D04410200010BD042810D90F2373
:103FB00002681340042B07D1FFF746FA21000A22BA
:103FC00007F0B8FE0400EEE7032B01D10430F5E75B
:103FD0000D20FDF771F9E6E70868F8B5C3071AD5B3
:103FE000FFF7DCFF0300203B5E2B25D80520434371
:103FF00001221D180020114E9D4219D005211024C8
:10400000F75C3C4200D0801801395200641000294E
:10401000F7D10133F0E704280ED90F2203681A40C4
:10402000042A09D11B099BB2002B05D00379DAE7DA
:10403000012340001843F8BD0120FCE731D1000006
:1040400070B508680D00FFF7A9FF04006868FFF766
:10405000A5FF621E0100042A14D8451E042D11D8A4
:1040600005236B439B18012215009D402B00064839
:1040700005682B430360054B1B68002B02D0200012
:1040800002F0E9FA002070BDF40F0020D81A0020D9
:1040900070B508680D00FFF781FF04006868FFF73E
:1040A0007DFF621E0100042A13D8451E042D10D87E
:1040B00005236B439B1801229A40074803689343EA
:1040C0000360064B1B68002B03D00022200002F087
:1040D000C2FA002070BDC046F40F0020D81A00209C
:1040E000F0B5050089B008680C00FFF757FF06908F
:1040F000022D36DD6068FFF751FF0190A068FFF7E1
:104100004DFF04000127231D661E0793731C0293B5
:10411000079B9E4235D0052373430593019B019D68
:1041200005330493049BAB421ED0042E16D86B1E9D
:10413000042B13D80122059B2349013B5B199A40AC
:104140009446224A0B681068069A3A4003920DD0B2
:1041500062461A430A60012200280DD17F00013512
:10416000E0E701240194CDE7029ECFE76246934346
:104170000B600028F2D0039A0299280002F06BFA33
:10418000ECE7019B1E1D042E1AD8012C18D1002526
:1041900005273B0021006B439B1999400B000A4AFD
:1041A000013511689943094B11601B68002B05D03C
:1041B000019B0022581D290002F04DFA052DE8D17F
:1041C000002009B0F0BDC046F40F0020D81A00202E
:1041D000086810B5C30703D5FFF7E0FE054B18606C
:1041E000054B1B68002B03D0024B186802F034FA11
:1041F000002010BDF40F0020D81A00207FB5A04C7D
:104200002368002B0AD19F4A1268002A06D19E4BD0
:104210001B68002B01D0FFF78DFD7FBD9B4D2A68E9
:10422000002A26D1984A1268002A1BD0FFF782FD87
:104230000028F2D0FFF76AFD924B24681A681C60D0
:10424000002A16D0002C14D101AD0C229049280070
:1042500007F002F9285D00210134FEF76FFE0C2CF7
:10426000F8D1DAE7874A1268002AE5D1002BE3D0BB
:10427000E0E700211A2003F001FB00211B2003F0DE
:10428000FDFA00211C2003F0F9FA2E68012E5CD003
:10429000022E00D1A2E0002E50D101363100794C1F
:1042A00003202368994303F0E9FA042021680140C0
:1042B0004B42594103F0E2FA102123680A201940C9
:1042C0004B42594103F0DAFA802123680901194071
:1042D0004B425941062003F0D1FA8021236809029C
:1042E00019404B425941072003F0C8FA8021236846
:1042F000490219404B425941092003F0BFFA80217D
:104300002368890219404B425941192003F0B6FA3B
:1043100080212368C90219404B425941182003F0FB
:10432000ADFA802321681B0319404B4259411720E5
:1043300003F0A4FA31001A2003F0A0FA2B6803213D
:10434000581C05F047F8296067E702214D4C1720FB
:10435000236819404B42594103F090FA0821236821
:10436000182019404B42594103F088FA80212368F4
:10437000C90019404B425941042003F07FFA8021C3
:104380002368490119404B4259410A2003F076FA4B
:1043900080212368C90119404B425941032003F091
:1043A0006DFA80212368890319404B425941092045
:1043B00003F064FA802321681B0419404B425941E1
:1043C000192003F05BFA3100062003F057FA3100A0
:1043D000072003F053FA31001B20ADE72021294CC0
:1043E0001720236819404B42594103F047FA4021F6
:1043F0002368182019404B42594103F03FFA8021AD
:104400002368192019404B42594103F037FA8021A3
:104410002368490019404B425941092003F02EFA04
:1044200080212368890019404B425941072003F03D
:1044300025FA80212368890119404B425941062001
:1044400003F01CFA80212368490319404B4259416B
:104450000A2003F013FA80212368C90319404B4254
:104460005941032003F00AFA802321685B041940B4
:104470004B425941042003F001FA01211C205BE763
:10448000F40F0020E80F0020F80F0020DC0F0020C0
:1044900025D10000012010B54042FFF7DFFC10BD20
:1044A00010B5034A0921034800F094FF10BDC0462F
:1044B0000CD4000054D4000030B502248025094BF0
:1044C000094AED009C505C59002CFCD0A124E4006A
:1044D000884202D30021995030BD8025ED0018514B
:1044E0004019F5E700E001400405000010B5002880
:1044F00006D1C020B02140028902FFF7DDFF10BDC8
:10450000B02080218002C902F7E7000043425841F1
:10451000064B40421840B0239B02C018036800209D
:104520001A0E532A01D11B02180A704700C0FEFF61
:1045300030B501248025054B054AED009C505C599F
:10454000002CFCD001600021995030BD00E00140FA
:104550000405000043425841074B40421840B02335
:104560009B02C018A62310B50902DB05090A1943EE
:10457000FFF7DEFF10BDC04600C0FEFF70B501248E
:1045800080250D4B0D4EED009C515C59002CFCD04C
:10459000002902DC00229A5170BD557814782D0252
:1045A00025439478013924042543D4780432240621
:1045B0002C4310C0ECE7C04600E0014004050000B9
:1045C00070B505004B680A009C1C2100A400FFF791
:1045D000D5FF281970BD0000134B1B68002B0CD0B1
:1045E0008022B023D2029B0200280BD11A1D5B68E7
:1045F0001B0E522B00D110007047B022C023920234
:104600005B02F1E782420DD903681B0E522B09D1E0
:10461000436802339B00C018824203D903681B0E13
:10462000522BE9D00020E7E7FC100020F0B5002075
:10463000B7B00024FFF7D0FF270005002600002DAB
:104640002ED1284D2868FFF761FF32003B00019012
:104650000094254904A807F05FFA04A801F0B0F817
:10466000224B64201C682B68A0215A425341204AE7
:104670005B421340B02292029B18E41A6043490245
:1046800004F0C2FDA0225202030000921949220048
:1046900004A807F041FA04A801F092F837B0F0BD81
:1046A000FF226B6829689C460233FF180B12013603
:1046B00013409C4200DA1C00FF200A1402400392BF
:1046C0006246014001920091039A0B4904A807F049
:1046D00023FA04A801F074F82800FFF77DFF050015
:1046E000ADE7C046FC1000205ED5000000110020A0
:1046F00000C0FEFF08D500004AD5000070B50020BC
:10470000FFF704FF04000120FFF700FF844200DAF6
:1047100004000A4B1D686A42554128001D60FFF7DE
:10472000E5FEA0226B4252021340054A28009B1866
:10473000044A611C1360FFF70DFF70BDFC100020E0
:104740000480010000110020F8B50020FFF7DEFE14
:1047500007000120FFF7DAFE3E00204D0643204C03
:104760000DD18021C020C9024002FFF7A5FE012122
:104770003000FFF7EFFE1B4B2E6023601DE08742E9
:1047800009DD0023B0212B60164B890223602368CA
:104790000020012517E0012380212B60124BC90264
:1047A0002360F4E7120E522A08D0002800D02360BC
:1047B0000E4801F005F8FFF7A1FFF8BD28005A6880
:1047C000023292009B188B4205D21A68561CE9D11E
:1047D0000028F2D0D1E72160EFE7C046FC100020AE
:1047E000001100200480010004C0020023D5000055
:1047F00070B50020FFF7F0FEFF260500002801D16C
:10480000280070BD03681C143440FFF7E5FEDA2C65
:10481000F4D10500F2E700008022F0B55200A1B00B
:104820000021674806F034FE8022002152006548CE
:1048300006F02EFE644BFF271B681A0004935342B8
:104840005A4110000592FFF751FE049C0020631EA0
:104850009C415E4B64421C405D4BE418FFF7C8FF6F
:104860000600002E2DD10498FFF750FE411C05983C
:10487000FFF770FE059A574D534B2C601A60FEF7F8
:104880006DFD514B64201B68A0215A4253414F4A91
:104890005B421340B0222C6892029B18E41A6043DA
:1048A000490204F0B1FCA0225202030000924A49DE
:1048B000220007A807F030F907A800F081FF21B017
:1048C000F0BD3268131412123A403B4003921A00B2
:1048D0000A3A092A49D83A4B039A995C002931D1FE
:1048E00010223E4806F0D4FD35002B6803991A12B9
:1048F0003A40914209D11A143A400B2A27D0132A80
:104900002DD00A2A01D1354B1D602800FFF764FE27
:10491000051EEAD1314B196800290FD02000FFF79E
:104920004FFE04002D4B5B195968002903D020006D
:10493000FFF746FE040004350C2DF3D1204B012176
:10494000039A99543000FFF747FE060089E73B4081
:10495000022BDADC214A9B00D3185D60D5E71022D8
:1049600000211E4806F094FDCFE71A00153A082AE8
:10497000E8D8144A0399525C002AE3D13500152B7C
:1049800000D01500300003681A143A40152A0FD0E1
:104990001D2A00D10025FFF71FFE0028F3D1002DAE
:1049A00004D020002900FFF70BFE0400054BC6E7EA
:1049B000039A1B123B409A42EDD10500EBE7C0463B
:1049C000FC0F002004110020FC10002000C0FEFF9E
:1049D00004C0020000110020EDD40000142F0020BC
:1049E00010B5FFF719FF10BDF0B585B00392032293
:1049F0000333DC17294D1440E4182B68284F5A4222
:104A0000534180225B42D202A4103B409B18A21C5F
:104A10000291244E910000910190316800980A188B
:104A2000934215D2FFF7F8FE2B685A425341802279
:104A30005B421F40D202BF183368009A9B189F4206
:104A400006D2194800F0BCFE0025280005B0F0BDD4
:104A5000029B356819066B461A7BA423DB051343BA
:104A6000FF222F00090C1943019B12041B04134061
:104A700019432800FFF75CFD0837281D2100376027
:104A8000FFF756FD002C04D00A9A21003800FFF7EA
:104A900075FD009B083BFF183760D6E7FC1000202F
:104AA00000C0FEFF00110020C7D4000070B59AB00E
:104AB000FFF74AFEFF221E4CD2000021200006F024
:104AC000E7FCFF25FFF794FE0026002814D1020022
:104AD000C300E3580130591E8B41D218FF28F7D18B
:104AE000144901A807F018F801A800F069FE12485F
:104AF00000F066FE1AB070BD03681A142A400A2A34
:104B00000AD11A122A40FF2A03D0D200A1180B7131
:104B1000A050FFF761FDD8E7132AFAD11B122B40F2
:104B2000FF2BF6D0DB00E2181671E650F1E7C04625
:104B30008C25002093D50000A7D500000021094B4B
:104B4000094A59600131516059680029FCD000219F
:104B50001961012393600222044B8131FF315A50C5
:104B60001A607047FC1000400010004000E100E0B7
:104B70000222064B0121DA670022054B5A61054AE1
:104B800011615A69002AFCD07047C04604E100E078
:104B9000FC1000400010004010B5044C2378002B9E
:104BA00001D0FFF7E5FF0020207010BD05120020A6
:104BB000802301205B055B6E5B001843704700009B
:104BC0000120024B1B685B001843704788120020CD
:104BD0000120024B1B685B00184370472400002033
:104BE0000120024B1B685B00184370478C120020A9
:104BF00070B504000D001600FEF792F98023012124
:104C00005B055A6E2670002653006170E170627277
:104C1000010A5A0A6071A171A272010C5A0C000EAD
:104C20005B0EA6702571E1712072E272237370BD74
:104C300010B5044C200006F0B5FF01002000FEF77F
:104C400023FE10BD911200200E4B10B51B680E4CB8
:104C50005A1C0FD00D4C002B0CD00D4C012B09D041
:104C60000C4C022B06D0094C042B03D00A4C052B0C
:104C700000D1074C200006F095FF01002000FEF750
:104C800003FE10BD2800002038D60000C0CE000072
:104C900043D60000C7CE00003DD6000070B5214CC1
:104CA0002278002A3DD1204B01215A608022D20572
:104CB00011605A68002AFCD0002207201B4B1C49B7
:104CC00001255A500439585008315A5019481A4988
:104CD00058501A491A485A501A495A50A622D20016
:104CE0009D50082218495A50043158500220174943
:104CF0005850174917485850174804395850182029
:104D000016495850C12189005A500539FF39585861
:104D1000921802435A501249124A9950FFF70EFF57
:104D2000257070BD05120020FC00004000100040FE
:104D30000C050000746962751C0500002405000064
:104D4000200004022C0500001405000034050000BA
:104D50003C050000FFFF0000211001005405000089
:104D6000061200200405000070B50E4B06001B78EB
:104D7000002B01D1FFF792FF00200B4D2C788442CD
:104D80000ED00A4B202219780323091B1940084B27
:104D90004901C918300006F05FFB0120013C2C706E
:104DA00070BDC046051200209012002004120020A1
:104DB00006120020002370B588B0984235DD0D68DA
:104DC00001262C0034409C422FD12300042D2CD9E5
:104DD0000F222B681A402300092A26D16A683F2A2D
:104DE00023DD6846FFF7C0FF230000281DD06B4677
:104DF00019783300A14203DB6B461B5D5B00334334
:104E0000A200AA1801349360202CF2D10921694430
:104E10004A780B7812021A438B781B041A43CB781A
:104E20001B061343024A13600423180008B070BD28
:104E30008C12002070B5454B8AB01B78002B01D135
:104E4000FFF72CFF02AC2000FFF78EFF002802D1F5
:104E500000200AB070BD23780B2BF9D96378012BA1
:104E6000F6D1E378012BF3D100231120384E394DD0
:104E700033602B7068442379374A41781360027895
:104E800009021143827812041143C27812060A43C0
:104E900032490A60002B0ED1152169444A780B78FB
:104EA00012021A438B781B041A43CB781B06134358
:104EB0003360002318E0012B1AD1152169444A7888
:104EC0000B7812021A438B781B041A43CB781A21F1
:104ED0001B06134333600E23627C6944934200DD5A
:104EE000130000229A422CD100220420EA54B0E799
:104EF000022B03D1627B10331621EEE7042B0DD178
:104F0000152108226944684606F0A6FA009801991E
:104F100002F026FD06F052F93060CAE7052BC8D131
:104F2000152108226944684606F096FA009801990E
:104F300002F016FD06F042F93060627D0A231E2160
:104F4000CBE7885CA8540132CCE7C04605120020AC
:104F50008812002091120020280000208C120020CE
:104F600010B5134B04001B78002B01D1FFF796FE00
:104F7000FFF7FEFD00200F4A0F49104B54505860B8
:104F80000130106058680028FCD000201861013002
:104F9000906018690028FCD0094B0A481B785B0117
:104FA0001B185350FFF7E4FDFFF7C8FD10BDC046C6
:104FB000051200200010004004050000FC10004015
:104FC000041200200612002010B588B000281DDD54
:104FD0000A68012113000B4018D1042A16D90F20AA
:104FE00014682040092811D150683F280EDD980030
:104FF000101880680024084201D04010C4B26846EE
:10500000C4540133202BF2D1FFF7AAFF002008B0CF
:1050100010BD000010B5002813DD0C68E30710D5A3
:105020006410532C0DD8084B1B78002B01D1FFF7CF
:1050300035FEFFF79DFDA123044ADB00D450FFF7A6
:105040007DFD002010BDC04605120020001000406C
:1050500010B500280EDD0C68E3070BD56410FF2C9B
:1050600008D8054B1B78002B01D1FFF717FE034A28
:10507000034BD450002010BD05120020001000404A
:105080002405000013B5002814DD0C68E30711D5D2
:10509000094B64100093094B0193072C0AD8084B65
:1050A0001B78002B01D1FFF7F9FD6B46054A195714
:1050B000054BD150002016BDE2ECF0F4F8FC0004E2
:1050C00005120020001000400C05000070B588B0EB
:1050D000002820DD0124086804401CD104281AD9C6
:1050E0000F2302681340042B15D1FEF7ADF906001B
:1050F00006F058FD0500122800D912252A000221C9
:105100000D326846FFF774FD6B465D73A54205DC02
:105110006846FFF725FF002008B070BD2300325D10
:105120006B449A730134F1E7F0B50D008BB00128A0
:1051300032DD08680122040014402DD104282BD947
:105140000F2301680B40042B26D16B68134223D038
:10515000FEF77AF96E6807007310019306F022FDDE
:1051600005000E2800D90E252A000121113202A8BF
:10517000FFF73EFD6A46127902AB5A7302AA731218
:105180009373019B76141B0ED67313745574A5424A
:1051900005DC02A8FFF7E4FE00200BB0F0BD3A5D8D
:1051A00002A963189A740134F1E730B589B0002878
:1051B00014DD0C68E30711D5102268460021FFF7C3
:1051C00017FD6B466A4665105D73684663122D0EC7
:1051D00064149373D4731574FFF7C2FE002009B0F2
:1051E00030BD0000174B184A5968002903D0002130
:1051F000596001319160196900291FD000201861A0
:105200008023DB00D3581149012B18D1A923DB00DF
:10521000D3585B420B600E490B78032B01D8013346
:105220000B7003200B490B78013303400B700A49C4
:105230005B015B1809495350012393607047086074
:10524000FAE7C046FC100040001000402400002097
:105250009012002004120020061200200405000015
:1052600010B5034A1021034800F0B4F810BDC04641
:10527000B8D50000AFD50000044A05491368C854EA
:1052800001339B059B0D13607047C046C01600207C
:10529000C012002070B5114C114A2368834202DC11
:1052A0000023236016E0155C411C2E00FA3E012EFF
:1052B00005D899420FDA555C013D1F2D01D9080030
:1052C000ECE70100151A565C6E5401318B42FADC92
:1052D000181A206070BD1570FAE7C046CC1A00207D
:1052E000CC16002010B5FDF711FE064B1A6882425D
:1052F00001D900221A601B68C31A034898428041F2
:10530000404210BDBC120020204E000010B5094CD8
:10531000094A23681268934200D110BD074AD05C45
:10532000FEF714F80028F8D0236801339B059B0D85
:105330002360ECE7C4160020C0160020C012002035
:1053400010B50400064B074A1B6812689B1ADB4322
:105350009B059B0DA34200DB10BDFFF7D7FFF1E7D4
:10536000C0160020C4160020F7B50500566801914C
:10537000B000441C06301700FFF7E2FFFB20FFF7E8
:105380007BFF1C20FFF778FFE8B2FFF775FFE0B264
:105390002412FFF771FFE0B2FFF76EFF6B4618793A
:1053A000FFF76AFF0025AE4200DCF7BDAB00FB183B
:1053B0009C680135E0B2FFF75FFF2012C0B2FFF733
:1053C0005BFF2014C0B2FFF757FF200EFFF754FF1A
:1053D000E9E7000070B5074E33680B2B08DC0C259D
:1053E0005D43054C0133285164196160A26033604C
:1053F00070BDC046C8160020242F002010B5FBF752
:105400005FFEFFF74DF8FBF783FEFDF741FFFEF768
:10541000EBFBFEF729FCFFF723FF00F015FF01F07F
:105420001DF901F067FB10BD962210B51201002195
:10543000034806F02DF80022024B1A6010BDC0464A
:105440002C1C0020CC050020064B074A1B68126864
:105450009B1ADB439B059B0D0122834200DC00224B
:1054600010007047C0160020C4160020F8B50500D3
:105470000C0016001F1E0ED10320FFF7E5FF0028C9
:1054800008D0FA20FFF7F8FEE8B2FFF7F5FEE0B229
:10549000FFF7F2FEF8BD501DFFF7D6FF0028F9D048
:1054A000FB20FFF7E9FEE8B2FFF7E6FEE0B2FFF708
:1054B000E3FEF0B2FFF7E0FE3012C0B2FFF7DCFE11
:1054C0003C00E31B9E42E5DD2078FFF7D5FE01346A
:1054D000F7E7000070B50024F0250B4B1B68A342D2
:1054E00002DCFFF7A1FF70BD2B006343074A9B1846
:1054F0001A78002A05D05978002311201A00FFF7E6
:10550000B5FF0134E9E7C046CC0500202C1C002083
:10551000F8B507000024F0252B0063430C4A013442
:105520009E18B74211D0317800290BD00133D15CDD
:10553000002311201A00FFF799FF2A0000213000F4
:1055400005F0A6FF0A2CE7D1F8BD024B1C60F9E775
:105550002C1C0020CC050020F0B5150001222F00E6
:10556000754C1740A54401900291002F11D005AB56
:105570001A706A105A70120E1A7105226912997007
:105580006D140299DD70FFF771FFCF239B009D44DE
:10559000F0BD042D1ED90F202A681040042826D102
:1055A000022304AA28001371FDF74EFF040006F041
:1055B000F9FA624B984200D91800B84204DC421C48
:1055C00005AB02990198DEE701377B1EE35C05AA73
:1055D000D355F2E7042D00D0A9E0032304AA043D2B
:1055E00013716B425D4105AB55710222E9E7092851
:1055F0007ED1042205AB1A706A6851100091694689
:10560000521209789A70009A59701F2A01DD2022DF
:1056100000926A46127806ACDA70009BBB4202DC4C
:1056200005ABE21ACDE70126BB00EB1898680640EF
:1056300006D1042837D90F210368194002290CD15B
:10564000012323704310637042121B0E4014A2709A
:10565000E070237105340137DFE7042921D10223EB
:105660002370FDF7F1FE039006F09CFAA31C0C28B2
:1056700009D86070864201D19C19ECE7039A925DCB
:105680009A550136F6E70C226270039A925D9A559C
:105690000136092EF9D12E23E372237363730E347E
:1056A000D9E7012907D10323043823704342584125
:1056B00060700234CFE7092909D1042323704368BD
:1056C0005A1062705B12A370E6700434C3E70329BA
:1056D0000BD1052323700068020992B2430F920098
:1056E0000B40D31A63701B12EDE726700134B2E74A
:1056F000032800D049E7052105AB1970110989B2CB
:10570000520F890002408A1A111299705A701100C2
:10571000642A00DD64210420D970C9B2041FA142AB
:1057200001DC04324DE72C5C1C540130F6E7002DFF
:1057300000D02AE751E7C046C4FCFFFF2303000066
:1057400070B502000024F0210D4E0800604380195E
:105750004578954203D001340A2CF6D170BDF02271
:10576000002105F095FE074A1368013BA34200D1D2
:105770001460002329001A001120FFF777FEEDE7DF
:105780002C1C0020CC05002010B5B2B002236A46C4
:105790000400137006F006FAC72800D9C7200023BA
:1057A000984207DC421C6B46FE211420FFF75EFE88
:1057B00032B010BD694601335A1EA25CCA54EFE7ED
:1057C00030B5B3B002236A460500137006F0EAF95B
:1057D0000400C72800D9C72400239C420BDC20000A
:1057E0003230FFF7ADFD621C6B46FF211420FFF73E
:1057F0003DFE33B030BD694601335A1EAA5CCA541F
:10580000EBE70000F0B5BBB004900C00012803DC0E
:105810001B20FBF751FD51E02A4B08680293C30798
:1058200009D4042807D90F2302681340042B02D19E
:10583000FDF70AFE0290234B60680393C30709D467
:10584000042807D90F2302681340042B02D1FDF767
:10585000FBFD039000271C4B1B680693069BBB4275
:105860000BDC039B194A0093C821029B08A806F091
:1058700021F908A8FFF7A4FFCAE70C267E43144BC2
:105880000299F618306806F083F9051E05D1736891
:10589000B6680793079B9D4201DB0137DEE730685E
:1058A0000399059606F074F90836002808D12100FE
:1058B0000498059B083102385B6898473BB0F0BDFF
:1058C0000135E7E7C4CF0000C816002014D7000058
:1058D000242F0020F7B5234B06001B68F02100930E
:1058E0000023009A9A4211DC0024F0231A0062433C
:1058F000019201991C4A55182F78002F12D00134BB
:105900000A2CF3D11948FFF75BFF29E00A005A433C
:10591000154882185078B04202D11278002A1FD15F
:105920000133DEE7F0223900280005F0B1FD022343
:105930000D4A0199EB6053540D4AF1008A58009BBF
:105940006E70AE70AA602F616F61A34202DC054BDE
:1059500001341C60002331001A001020FFF786FD7F
:10596000F7BDC046CC0500202C1C00205DDB0000EC
:105970008C25002010B5FFF7ADFDFF24084AE30099
:105980005B429B18074AD35C043B012B03D8E043DE
:10599000C0B2FFF79FFF013C002CEFD110BDC04605
:1059A000FC0700008C250020F7B50F00FF247F25A1
:1059B00001901E4AE300D31A1D4A9A181278062A4B
:1059C00001D0032A20D1FF22D2009B1818688368D7
:1059D0002B401C2B18D1C3681A002A40042A13D16B
:1059E00002692A40192A0FD11B0A01339B000C308F
:1059F000C018FDF729FD03780600002B10D006F033
:105A0000D1F80023B84209D0013C002CD1D1F7BD18
:105A1000019AF15CD25C9142F6D101339F42F7DCEE
:105A2000E043C0B2FFF756FFEEE7C0468C250020EA
:105A3000FC07000070B50500FF24084AE3005B4244
:105A40009B18074AD35CAB4203D1E043C0B2FFF7D7
:105A500041FF013C002CF0D170BDC046FC070000A6
:105A60008C250020F7B5FDF751FA514B1A68824298
:105A700001D900221A601A684E49821A8A4200D857
:105A800083E01860FDF74CFA071E00D101370020B3
:105A9000FDF738FB01900020FDF748FB019B0090CB
:105AA000454C464D002B14D02368002B00D07AE0E3
:105AB0002B682760002B00D171E0414B01261B7839
:105AC000002B63D10920FFF7B5FF3E4B1E703C4B06
:105AD0001E70009B002B12D02B68002B0FD1236867
:105AE0002F60002B1ED0374B01261B78002B52D184
:105AF0000920FFF79FFF334B1E70314B1E70236848
:105B0000002B0FD02F4E3278002A0BD19F4200D2AB
:105B100027602368FB1A312B04D90720FFF78AFF7F
:105B2000012333702B68002B0FD0254E3278002ACA
:105B30000BD1BB4200D92F602B68FF1A312F04D93B
:105B40000820FFF777FF012333702368002B0CD068
:105B5000019B002B09D11B4E3378002B02D107206B
:105B6000FFF768FF0023236033702B68002B0CD0F5
:105B7000009B002B09D1124C2378002B02D1082066
:105B8000FFF758FF00232B602370F7BD0720FFF7B6
:105B900051FF0C4B9CE70820FFF74CFFADE7009B43
:105BA000002B9CD1ABE7009A002A95D1AAE7C0460A
:105BB000B81200200F270000A8120020B012002009
:105BC000B4120020AC12002037B500240500FFF706
:105BD00081FC01A80194FDF783FA21002000FEF763
:105BE0002DF9FEF70BFBFDF72FFBFDF749FBFEF749
:105BF00051FCFDF7B1F9A54204D0FDF7D1FB0248F5
:105C0000FFF7DEFD37BDC0464EDB0000002310B5B8
:105C100001001A001120FFF729FC10BD07B56B46E3
:105C2000197069465A7013128B701314120ECB70D0
:105C30000A716B46010005221320FFF717FC07BD10
:105C400010B50A0001001220FFF786FC10BD70B5E8
:105C5000050008000C003230FFF772FB2B00220019
:105C600000211B20FFF702FC70BD10B50C000300E3
:105C7000110014202200FFF7F9FB10BD012370B5BD
:105C8000FF24084A41185B42884201D3D84370BDC3
:105C900006781D0A234073409B009B5801306B40DF
:105CA000F2E7C04630D7000013B50400FE2813D831
:105CB0000A4BC200D05800280ED043680830990023
:105CC000FFF7DCFF01900920FFF73AFB01AB04224C
:105CD00021001720FFF7CAFB13BDC0468C2500200A
:105CE000F7B50190FEF784FD01250400FF276D4202
:105CF000002C01D12800FEBD266833143B40152B33
:105D00000DD121000198083105F042FF002801D192
:105D100035123D402000FEF75FFC0400E8E71D2B34
:105D2000F8D101256D42F5E7F0B580279DB0FFF76A
:105D3000EDFAA54CA54D2068FF00391A4019FDF772
:105D4000EBFA23680600C3182360002B0ED11DB0A8
:105D5000F0BD2068391A2818FDF7DEFA236806001E
:105D60001B182360FDF7D2F8994B1860002EF0DC69
:105D70002B78FA2B00D037E12368022B07DCFFF7E2
:105D8000B1FA0028E3D00120FFF784FADFE7687852
:105D9000AC78023818282BD803F0A2F919002C008F
:105DA00030003400370040002A004A007C008600A2
:105DB0008A00A000F10002012A002A002A002A001D
:105DC0002A002A002A002A002A002A001001FF2C9B
:105DD0000ED02000FFF7B4FC00227E4BE100CA5039
:105DE0005B181A712100009213001320FEF7FCFDCE
:105DF0000320C9E72000FFF76DFDF9E72000FFF75A
:105E00009FFCF5E7FFF7B6FDF2E7FFF763FB002025
:105E1000FFF7DAFE7048FFF7D3FCE9E7632CE7D819
:105E20006E4BA200D25821001520FFF795FBDFE74B
:105E3000FEF7DEFCFF270400002CD9D025682B14C8
:105E40003B40152B04D02000FEF7C6FB0400F3E70F
:105E50002000083005F0A6FE06000530FFF770FAB6
:105E6000FB20FFF709FA2D121D20FFF705FAE8B213
:105E7000FFF702FAF0B2FFF7FFF93012C0B2FFF7F6
:105E8000FBF925002B1B9E42DDDD287AFFF7F4F994
:105E90000135F7E700211D2000910B000A00FEF7F5
:105EA000A3FDFDF77DFAA3E72000FFF7FDFE9FE7C6
:105EB000FDF73EF803AC4A4A64210090494B2000AC
:105EC00005F0F8FD02232000237005F06BFE23008F
:105ED000020000211620FFF7C9FA89E700243D4A95
:105EE000E300D558002D27D06B689E00701DFFF78A
:105EF00027FA2B0000253200083321000120FFF78C
:105F0000B5FA2F00FEF774FC2E00002818D1002FE0
:105F100004D03A0001212000FFF726FA002D04D01A
:105F20002A0002212000FFF71FFA002E04D03200C1
:105F300000212000FFF718FA0134FF2CCFD157E7DA
:105F4000FF2103681A120A40A24209D11A140A401A
:105F50000B2A08D10B400CD0012B0CD0022B0CD0FB
:105F6000FEF73AFBD1E7132AFAD100252F002E00C5
:105F7000F6E70600F4E70700F2E70500F0E7002483
:105F8000FFF7A8FA2200210000942300DA20FEF790
:105F90002BFDFF222100D2000E4805F079FA80E7A0
:105FA000012C02D1FEF742FB22E7022C02D1FEF7C0
:105FB00017FD1DE70120FFF707FE19E70023210069
:105FC0001A001A2087E7C046CC1A0020CC16002001
:105FD000BC1200208C25002030DB0000842D002026
:105FE00047DB000042DB0000FB2B00D0CBE6226841
:105FF000042A00DCC3E62E79E878574B36020643C4
:106000009E4200DDBFE6331D9A4200DCB7E6EB5C42
:10601000FE2B00D0B7E66B78AC78771E1B2B61D0D7
:1060200019D8072B47D0082B1CD0012B18D1FF2CD7
:1060300016D02000FFF784FB6D79484AB31E00920A
:1060400021002A000A20FEF7CFFC454BE400E05077
:106050001B191D7104E01D2B56D048D31E2B6AD08E
:10606000701D91E6632CFBD86A79022A13D0032AAB
:106070001BD0012AF4D1E979AB79090219432B7AB3
:10608000A4001B0419436B7A1B060B435B001343EC
:10609000344AA350E4E7002FE2DDB11E2F48FDF79C
:1060A000F3FB304BA400E050DAE7AB79A4005A1EB2
:1060B00093419B00ECE7632FD2DC03AD3A002A4901
:1060C000280005F0C9F900232800EB55FFF708FE6A
:1060D0000028C5DB234B8000C25821001520FFF7A4
:1060E0003BFABDE739002048FFF75EFCB8E7FF2C1C
:1060F000B6D06A79022AB3D818490B200091210042
:10610000B31EFEF771FCABE7632F00DD63270023AE
:1061100003A99F420ADCFB430022DB173B40CB185C
:106120001A70152000917B1C2100EAE7EA185279C9
:10613000CA540133EDE7012C92D1002F90DD6B7929
:10614000002B03D01C00322B00DD322464235C437F
:10615000064B1C6084E7C046F6030000D216002000
:106160008C250020842D0020D11600200400002062
:106170000122094B1A60094A1368002BFCD0032244
:10618000074B1B68D8171040C01801238010063831
:10619000400018437047C04600C0004000C10040A6
:1061A00008C500400120704710B5064C200000F0E3
:1061B000D7FD0549200000F0FBFD0122034B1A60CA
:1061C00010BDC046FC1A0020801A0600D01A00201C
:1061D00010B501210D20FCF7B1FE01210E20FCF7C6
:1061E000ADFE00210F20FCF7A9FE044C200000F0BA
:1061F000F3FC1021200000F00BFD10BDDC1A002084
:1062000010B504680D20E30703D56410FF2C03D9F3
:106210001720FBF751F810BDFFF7DAFFE1B2024893
:1062200000F018FD0020F6E7DC1A002010B5FFF79B
:10623000CFFF0021034800F00DFD4300012018436B
:1062400010BDC046DC1A002010B5034A08210348DF
:10625000FFF7C0F810BDC04674DB0000B4DB0000DF
:106260000D4B70B51B6804000E001500002B01D10A
:10627000FFF79AFFE1B2094C200000F030FEF1B2C6
:10628000200000F033FDE9B2200000F02FFD2000D7
:1062900000F090FE70BDC046D01A0020FC1A00200D
:1062A00010B501240368234205D04168214202D081
:1062B0008268224203D10D20FAF7FEFF10BD58106C
:1062C000802801D91520F7E74910FF2901D91620A8
:1062D000F2E75210FF2A01D91720EDE7FFF7C0FFC0
:1062E0000020EBE7F7B501221400904222DD0D6893
:1062F0002A421FD01D4B15411B684C68002B01D151
:10630000FFF752FFE9B201272500194E3D4030004A
:1063100000F0E5FD002D0FD03C413000E1B200F06F
:10632000E5FC300000F046FE0024A04202D023200D
:10633000FAF7C2FF2000FEBD042CF2D90F23226819
:106340001340092BEDD163685B100193019BAB42B5
:10635000E7DDAB00E3189968394204D04910C9B2AF
:10636000300000F0C3FC0135F0E7C046D01A002031
:10637000FC1A0020154B70B51B6805000E00002BA1
:1063800001D1FFF711FF124CEDB22900200000F0FF
:10639000A6FDF1B2200000F0A9FC0021200000F0D1
:1063A000A9FD002801D0404270BD72B6012229002B
:1063B000200000F08FFD62B6200000F088FC00286D
:1063C000F2D0200000F088FCEEE7C046D01A002092
:1063D000FC1A002010B501240368234202D0416852
:1063E000214203D10D20FAF767FF10BD5810802815
:1063F00001D91520F7E74910FF2901D91620F2E746
:10640000FFF7B8FF40002043EFE7000010B50D2173
:106410001D20FFF7AFFF164C5A2809D101222A216F
:1064200022703D38FFF71CFF0122124B1A6010BD8D
:106430000F211920FFF79EFF332805D102235F2289
:10644000237020211A38EDE70D211E20FFF792FF5F
:10645000C7280AD1032300222A21A9382370FFF775
:10646000FFFE1B222A211E20DCE700232370DBE72E
:106470002C000020D41A0020204B10B51B6804000B
:10648000002B01D1FFF7C2FF1D4B1B785BB2022B23
:106490000AD0032B29D0012B2CD121001D2001244F
:1064A000FFF768FF644205E0012C13D12921192070
:1064B000FFF760FF7F2801DD0138FF3803007F33DD
:1064C00001DA7F204042C8237F21584302F09CFE1E
:1064D000604310BD032C0BD12B211920FFF74AFF7D
:1064E000043CE7E72D211920D9E721001E20D6E73B
:1064F000052CF7D0012400206442E4E7D41A0020E0
:106500002C00002010B50120FFF7B6FF430001204A
:10651000184310BD10B50320FFF7AEFF4300012064
:10652000184310BD10B50520FFF7A6FF430001205A
:10653000184310BD144B70B51B68002B02D101200D
:10654000FFF79AFF114B1B785BB2013301D1FFF7C4
:106550005DFF0120FFF790FF04000320FFF78CFF91
:1065600005000520FFF788FF6D436443404364192D
:10657000201804F059FE01F023FB04F01FFE430035
:106580000120184370BDC046D41A00202C00002002
:10659000F8B501231C0098422BDD0F683B4228D040
:1065A0004E6835001D4024D1042E22D90F223168B7
:1065B0000A40092A1DD173685C10202C00DD2024BC
:1065C000144B1B68002B01D1FFF7EEFD72B67F1054
:1065D000F9B2114F2200380000F07CFC62B6A542EF
:1065E00014DA380000F073FB002804D101246D0098
:1065F0002C432000F8BD380000F06EFB0122AB00F8
:106600004000F31810439860AD18E8E764000125D6
:10661000EEE7C046D01A0020FC1A00200020704788
:10662000012070470020704700207047012070470C
:1066300000207047002070470020704700207047FE
:1066400000207047002070470020704700207047EE
:1066500000207047704770477047000010B5034A2C
:106660000E210348FEF7B6FE10BDC04604DC000054
:1066700074DC00000378013B1F2B00D97047013008
:10668000F8E710B5FFF7F6FF0378002B0BD00130C9
:10669000222B11D10378002B03D0421C222B03D1D3
:1066A0001000FFF7E7FF10BD5C2B03D14378002BF0
:1066B00000D0821C1000EDE73A2BF2D02C2BF0D04A
:1066C0007B2B0BD1FFF7D6FF0378002BE9D07D2B76
:1066D00001D10130E5E7FFF7D4FFF5E720225B2B7E
:1066E00014D1FFF7C7FF0378002BDAD05D2BF0D071
:1066F000FFF7C7FFF7E7202BD3DD2C2BD3D01900F2
:1067000091435D29CFD0222BCDD001300378002BCF
:10671000F1D1C6E7002210B5904216D0FFF7AAFFCC
:1067200003780422222B10D0023A7B2B0DD0013AA1
:106730005B2B0AD0190030390232092905D92D2BDB
:1067400005D14178303909290AD8100010BD052239
:10675000742BFAD00132662BF7D001326E2BF4D0B5
:10676000581E83415A42F0E770B5FFF783FF037864
:1067700001222D2B01D18018023A00230A2502E0C4
:106780006B430130CB1801783039CCB2092CF7D9E2
:106790005A43100070BDF8B50C001500FFF76AFFF2
:1067A0000378222B02D000232370F8BD0D236A1E2C
:1067B000210008250C260A279C4601300378222B4D
:1067C00002D100230B70F0E7002BFAD0441C5C2BA5
:1067D0000BD14378841C622B0ED0662B0ED06E2B0F
:1067E0000ED0722B0ED0742B0ED0002AE9DD0B7068
:1067F000013A01312000E1E72B00F6E73300F4E72E
:106800003B00F2E76346F0E70923EEE710B504002A
:10681000FFF737FFA04202D90378202B00D910BD23
:106820000138F7E710B5002815D00378002B13D0F6
:10683000FFF720FF2021037802008B4300205D2B0F
:1068400009D01000FFF71DFF03782C3B5A4253413B
:10685000C018FFF70FFF10BD1800FCE70300002071
:1068600070B50C0081420EDD1A785B2A0BD1581CE2
:10687000FFF700FF0125AC4205D0FFF7D3FF00284A
:1068800001D00135F7E770BD70B50C001500002987
:1068900001D000230B70002820D00378002B1ED0DD
:1068A000FFF7E8FE037806002C2B03D10130FFF739
:1068B000E1FE0600337800207D2B0FD0844204D007
:1068C0002A0021003000FFF766FF3000FFF7D9FEF5
:1068D00003783A2B02D10130FFF7CCFE70BD1800CF
:1068E000FCE7F0B50D0004009DB02E78002E35D0E9
:1068F0002E21280005F03EF9071E14D0431B0193FA
:10690000303E092E14D82800FFF72EFF010020008A
:10691000FFF7A4FF0400002C20D0002F1ED0019B05
:106920000133ED18E1E7280005F03CF90190E7E7B5
:1069300023787B2B11D1601C642203A9FFF7A4FFED
:10694000041E0BD0019A290003A805F032F9002893
:10695000E1D02000FFF795FEEEE7002420001DB0F7
:10696000F0BD70B5050000200C0081421DDD28003F
:10697000FFF7D0FE0300681C012B14D00020022B6F
:1069800013D10022681C1100FFF77EFF012C0CD0F0
:10699000FFF748FF00221100FFF776FF013CF5E703
:1069A000FFF740FF013C012CFAD170BDF8B505009E
:1069B00000200C0016001F0081420DDD2800FFF7AB
:1069C000A9FE03000020022B06D1681C3A0031000A
:1069D000FFF75AFF012C00D1F8BDFFF723FF3A0063
:1069E0003100FFF751FF013CF4E710B50024A0424D
:1069F00018D0FFF73FFE03787B2B0AD1013000222D
:106A00001100FFF741FF00280CD0FFF73AFE0134D8
:106A1000F5E75B2B06D10130FFF704FF002801D01A
:106A20000134F9E7200010BDF8B5002816DD0D6827
:106A3000EB0713D56D10013D0124FDF7D9FE0026AB
:106A4000FF27644200280CD1002E21D0300005F031
:106A5000A9F801003000FCF717FFF8BD01256D42D1
:106A6000EAE703681A143A40152A0BD11B123B407F
:106A70009C4200DA1C009D4201D106000836FDF759
:106A8000ABFDDFE71D2AFAD1012400266442F6E7B8
:106A90000120013464002043DFE7000010B50868DE
:106AA0000C00FCF7D1FCFFF71BF9002803DB626840
:106AB000024B8000C250002010BDC046842D002033
:106AC00010B50868FCF7C0FCFFF70AF9012300289D
:106AD00002DB024B8000C358180010BD842D00203B
:106AE00010B50868FCF7B0FCFFF7FAF8C043C00F18
:106AF000800010BD10B5034A04210348FEF76AFC6C
:106B000010BDC04604DD0000FDDC000010B5FCF740
:106B1000CBFBFCF76BFCFEF771FC0448FEF750FE64
:106B2000FDF7C4FFFEF726FF10BDC04653DD000091
:106B300010B5FCF7B1F810BD70B5002504AC247891
:106B40000573A94205D10A4B0A4A23210A4804F0D9
:106B500015FC01600949920052589B0002715B5874
:106B6000A40083716358856043710223C37170BDB3
:106B70006BDD0000CADD000079DD000028DE0000CA
:106B8000037B002B04D143738373036101330373CD
:106B9000704700001FB50191A02100240068C900C2
:106BA000D2B24450012A10D0A24209D0032A0AD0FE
:106BB000074A8350074B019AC250012343501FBD1F
:106BC00002221343F4E70422FBE70622F9E7C0465A
:106BD000540500002405000010B50400FFF7D0FFA5
:106BE000A1222368A179D20099506179064A200038
:106BF0009950217904329950044B19685A689B685E
:106C0000FFF7C8FF10BDC0460C050000F01A0020B9
:106C10004BB2002B0FDB80233F290FD81F290FD841
:106C20000F290FD807290FD803290FD81B06016891
:106C3000074A8B50704780239B04F8E7DB04F6E794
:106C40001B05F4E75B05F2E79B05F0E7DB05EEE7E4
:106C5000240500000368074A99501A00FC32D168E5
:106C60000029FCD0A321C90058580023C0B2D3602A
:106C70007047C0461C05000007B58022074BD205AF
:106C80001A6000229A6002321A710F230C320093AC
:106C90000349023B0348FFF74FFF07BDF01A0020EE
:106CA00000300040DC1A0020F8B505000E00170087
:106CB0000024BC4208D02B68315D1B68280098472F
:106CC000002801D00134F4E72000F8BD704710B56A
:106CD0001C3000F0A9F910BD10B51C3000F096F979
:106CE00010BD10B51C3000F0A5F910BD70B5437E85
:106CF0000D00002B01D1002070BD6430040000F0B5
:106D0000A2F90028F7D12000290000F070F9012035
:106D1000F2E70000F7B50193FA23002504009B0079
:106D200083600D4B4560083303601C300F00160074
:106D300000F052F92000643000F04EF9074A276154
:106D4000B600B35820006375019B9B009B58657685
:106D5000A576A375FEBDC04608DE000028DE000053
:106D60000123A022C375837D0E49C133FF33D205B1
:106D70009B009950437DC133FF339B009950CC2237
:106D80000169094B5204CA5005220169243BCA50CB
:106D9000827D01690833CA500269417D034BD1509D
:106DA0007047C0460C060000240500000C050000DA
:106DB000A022002310B50469D200A3500A4CA142BE
:106DC0000FD90A4C8C425B4109495B420B40CD21F3
:106DD000C9045B1804690749635005210369995088
:106DE00010BDCC235B04F5E7A086010090D0030022
:106DF000000098FD24050000F7B5040000200D00F8
:106E00000193824265D01600402A00D9402627000F
:106E10001C37380000F0F6F8B1232269DB00D550AA
:106E200080220123216992008B50A27E002A03D187
:106E300022691362226913600025731EAB4207D1D9
:106E4000019B002B04D080220221236992009950DB
:106E5000012223691A622369FC33DA68002A02D10D
:106E60009A6A002AF9D09A6A002A0BD1DA60A32321
:106E70002269DB00D1583800C9B2013500F0B7F8FB
:106E8000B542DAD3019B2269002B0FD11300FC33EA
:106E90009B6A002B0AD10133A376D3612369FC33AB
:106EA000DA6C002AFCD00022DA640AE00023012117
:106EB000A37651611A002369FC3399680029FCD03C
:106EC0009A602369FC339A6A002A01D000229A62F0
:106ED000E8B2FEBD10B50123FFF78EFF10BD030021
:106EE000AC3310B504001970643000F08BF8012346
:106EF000637610BD0023020070B5AC3243760D00FE
:106F00001178B12204000069D200815080222169E9
:106F100092008B502269013313622269936026002C
:106F20006436300000F080F8002812D0300000F005
:106F30006DF81E4B2269D0502369FC331A6A002A6F
:106F400002D19A6A002AF9D09A6A002A01D11A62FB
:106F5000E5E723690122002D0DD11900FC31896A72
:106F6000002908D1DA612369FC33DA6C002AFCD0ED
:106F70000022DA6407E05A612369FC339A68002A28
:106F8000FCD000229A6000202369FC339A6A824276
:106F90000BD098622169064A8B588B501800022B3F
:106FA00003D0181F431E9841033070BD1C0500001C
:106FB000C404000010B50121FFF79CFF10BD0000C4
:106FC00010B51323142202490248FFF7A3FE10BD97
:106FD00000400040FC1A002010B5402200210400AF
:106FE00004F056FA002320002364636410BD10B53A
:106FF0003F24026C531C2340446C9C4201D08154BA
:10700000036410BD0023036443647047436C026C47
:10701000934206D03F21C25C01330B404364100011
:10702000704701204042FBE7036C406C181A00D502
:1070300040307047436C026C934201D0C05C704793
:1070400001204042FBE73F22036C406C01331340B8
:10705000181A43425841C0B27047000003210A4841
:1070600002680A430260094802680A43026008494C
:10707000084A094B9B1A03DD043BC858D050FBDC7F
:1070800000F012F8F9F740F82405004054050040DC
:107090007CE300000000002064020020FEE7FEE721
:1070A000FEE7FEE7FEE7FEE72D4B10B51A68D2B209
:1070B000012A0FD12B4A126812070BD12A4AE02469
:1070C0001168F0220800104021422DD1274909689B
:1070D00011422CD01A68D2B2012A12D12149096872
:1070E00009070ED1F020204909680140402908D144
:1070F0001E490968014204D18020C121C005C90090
:1071000042501B68DBB2012B0DD1164B1B681B07CD
:1071100009D1154B1A68F0231A40A02A0FD1134A3F
:1071200012681A420ED010BD3028CFD0D2E7104AD4
:10713000104911608021104A09021160CAE7D02A63
:10714000F1D1ECE70D4B1A68012A04D00C4A1A6001
:107150001A68012AFCD1C0220A4B1A60E3E7C04634
:10716000E00F00F0E40F00F0E80F00F0EC0F00F08B
:1071700004050040DFFF07C0186C004000EC06402B
:107180007593000014EC06400120704710B50368A9
:107190001322DB69984710BD70470000054B026958
:1071A000D1500369FC331A6A002AFCD00022012066
:1071B0001A6270471C050000030010B55C331A7892
:1071C0001F231A401E3B19009140114AD167C22269
:1071D000042104699200A150026953600269D360DE
:1071E000A02300220169DB00CA5001230169094A7A
:1071F0005B428B500169084A8B5001690C3A8B50F5
:10720000016908328B501430FFF7FCFE10BDC046F8
:1072100004E100E00C0500001405000010B5143076
:10722000FFF702FF10BD10B51430FFF703FF10BDCC
:1072300010B51430FFF7EAFE10BD0000030070B572
:107240005E331A780469724BE25003005D331A789A
:107250000469704BE250030061331C7802696E4B85
:10726000012C00D09EE005005F352E78A225ED00B0
:107270005651020060321578A1220669D200B5503D
:107280000269D4509623DB00994200D88CE0962303
:107290001B01994200D88AE096235B01994200D8ED
:1072A00088E096239B01994200D885E0E1239B0169
:1072B000994200D882E09623DB01994200D880E011
:1072C000E123DB01994200D87DE096231B0299421D
:1072D00000D87AE0E1231B02994200D877E0962398
:1072E0005B02994200D874E0E1235B02994200D826
:1072F00071E0E1239B02994200D86EE0474B99422E
:1073000000D86CE0E123DB02994200D86AE0E12278
:10731000002312038A425B41414A5B4213408022B0
:1073200052059B1801693F4A8B50A0230422016932
:10733000DB00CA5000210369FC33D9600369FC33C8
:107340001962012301690B6001698B60C121046925
:10735000890062501F215C3002780A4093406231FC
:10736000314AFF3153500021415600293CDA0F23A6
:107370000B40083B2D4C9B089B001B19032421400C
:10738000A140FC348C40DD69A5432C00C0258D4014
:1073900029002143D9611F23017819401E3B8B40EE
:1073A000136070BD00246CE79E23DB02BAE79D23C7
:1073B0001B03B7E71E4BB5E71E4BB3E7EC239B035C
:1073C000B0E71D4BAEE71D4BACE71D4BAAE71D4BCD
:1073D000A8E71D4BA6E71D4BA4E71D4BA2E78023A2
:1073E000DB049FE71B4B9DE78C080F4BA400E418C0
:1073F00003230B40FF21C025DB009940AD006659F7
:107400008E433100C0269E4033000B436351C2E7D8
:107410000C050000140500006C05000090D003006E
:1074200000D0BEFE2405000000E100E000ED00E019
:1074300000B013000050270000A04E0000F07500BF
:1074400000509D0000F0EB0000903A0100E0D701F1
:1074500000B0AF0300705F07F7B5009308AB1B786F
:1074600000250193FA2304009B0083600E4B4560C6
:107470000833036014300F001600FFF7ADFD230042
:107480005C3327611E70009B084A9B0099582300BB
:107490005D331970019B20009B009A5823005E33D6
:1074A000DD701A70FEBDC046ACDE000028DE0000B4
:1074B000036910B51A00FC32D2680400002A0AD011
:1074C000A322D20099581430C9B2FFF790FD0022D0
:1074D0002369FC33DA6010BD10B50248FFF7E8FFFE
:1074E00010BDC046B41B0020162307B5022200932E
:1074F0000249013B0248FFF7AFFF07BD00200040F3
:10750000B41B002010B5002801D004F07DFA10BD96
:107510007047000010B500F011F8FFF7F9FF0120E7
:1075200000F000FAFFF7F2FAFFF702FB024B002B24
:10753000FAD000E000BFF7E700000000C420114BC4
:1075400080001A5810491140C02212020A431A50F2
:10755000C0218022490092025A501A608023A3223F
:107560000021DB05D20099500122F9309A60074BC7
:10757000FF301950C120023180001950403019509D
:107580001A60704700E100E0FF00FFFF00100140BB
:10759000014B18607047C04678000020F7B5002303
:1075A00020285AD8384B8000C258042A5BD007D80C
:1075B000022A54D055D80423012A09D000234CE0D4
:1075C000062A54D051D31A2A53D002231B2AF5D1AC
:1075D0002E4A116808294ED909294FD00A240226BB
:1075E000A02001252A4AC00015502A482A4D0768C4
:1075F0001C20BF0007402948019700685759009098
:1076000027481B0207401F43C02300989B020340EA
:10761000FF2057515759000207401F43019B1F434A
:10762000009B58016023184007433E4356510125F3
:107630001C4B156058680028FCD000205860A1231E
:107640000125DB00D3585560A025ED0050511BB239
:10765000A14202D015D2611ACB401800FEBD08230A
:10766000B6E71023B4E72023B2E74023B0E7802336
:10767000AEE70123ACE708240026B1E70C000126A1
:10768000AEE7091B8B40E8E728DE0000740000200D
:10769000007000403000002004050000340000208D
:1076A000FF00FFFFFC700040F0B520285BD8364B90
:1076B0008000C258354B1E68002E30D1C227344B93
:1076C000BF00D859334C03250440C020000220439A
:1076D000D851C02480206400800018512E4F1860BB
:1076E0002E4B803CD859FF3CA043D8510437D85981
:1076F000A8432043D8510837D8590C35A8438446AD
:10770000072065462843D851A820C0001E50C1203C
:107710008026800076021E501C601C4B1C601425C5
:1077200000202B001E4C2E0046433659771C1BD1DF
:107730004343E250A0230325C132FF329200DB0510
:10774000D550184B1A68082A14D114234343E31860
:107750009A6812485132FF32920059601150DA682B
:10776000C1239B00C250F0BD9642E1D001300328F6
:10777000D9D1F8E7082A02D9083AD140E5E7082329
:107780009A1A9140E1E7C04628DE0000181C00204C
:1077900000E100E0FF00FFFF040500000090004052
:1077A00038000020780000202149F0B54A6C2148BB
:1077B000002A14D0A025A12600230124ED05F600FF
:1077C000C258571C06D0C7187F68002F02D0270068
:1077D0009740AF5114333C2BF2D100234B64A023CC
:1077E0000121DB0500260F009C4614234B43C318E0
:1077F0001A1F1268104C0E4D920014195219526C37
:10780000002A10D01A00143A1268551C09D0103BF7
:107810001B68FF2B05D03B00934065461A00074BC1
:10782000EA50FC34666401310429DED1F0BDC04663
:10783000FC90004038000020009000400C05000043
:1078400000B5202810D80C4A8000835803290BD893
:10785000A0220800C133FF33D2059B0001F036FCA3
:10786000020905070021D15000BD0C21FBE70421CE
:10787000F9E70321F7E7C04628DE000020280AD8F0
:10788000074B8000C25801239340A022D205002953
:1078900002D1044953507047A121C900FAE7C046FC
:1078A00028DE00000C05000003000020202B0AD871
:1078B000A021A222C905D2008858034A9B009B58E8
:1078C000D84001231840704728DE0000F7B50600B5
:1078D0000D000C008B180193019B671B9C4207D085
:1078E000336821781B683000984701340028F3D1B1
:1078F0003800FEBD0849094A094B10B51B68885875
:10790000FA22190A1B0618439200002301F0B4FD65
:107910004904C00B084310BD0010014004050000DD
:107920001C1C002070B5041E09D0FFF7E3FF050002
:1079300000F014F8FFF7DEFF401BA042F8D370BD43
:107940000022044B9A60044A13680133DBB21360CF
:107950007047C046FC1001401C1C0020704700000E
:10796000F0B5C64600B5CB0F9846404A4B005B0DBC
:107970009A1882B00D000400132A2FDC002A49DB7C
:107980003B4F17413E000E40064323D07F0839008D
:1079900029400C430AD03749BD438C4663445C42BE
:1079A0005C418023DB021341E4071D434146CE00C6
:1079B00031492B008E192200346875682000290097
:1079C00001F000FF009001910098019922002B0026
:1079D00003F090F802B004BC9046F0BD332A08DDF5
:1079E0008023DB009A42F5D102000B0001F0EAFE91
:1079F000F0E7224A9446012263445242DA400242AE
:107A0000E8D052080242D1D094438022D2051A41D4
:107A10001443CBE74B005B080343DBD00B031B0B8A
:107A20001C436342234380244D0C24031B0B23403F
:107A30006D042B4319004346DA000F4B9B181C685A
:107A40005D6802000B002000290001F0BBFE0090E1
:107A500001910098019922002B0003F04BF8424657
:107A60004B005B08D60733431900B3E701FCFFFF67
:107A7000FFFF0F00EEFBFFFFE0DE0000EDFBFFFF6E
:107A8000F8B5274A4B005B0D9A180C000700132A23
:107A900010DC002A36DB234B13410B423AD0802402
:107AA00024031441002064189C4306002500300084
:107AB0002900F8BD332A0EDD80230600DB000D000F
:107AC0009A42F4D102000B003800210001F07AFE46
:107AD00006000D00EBE7144D0600AC46012563449B
:107AE0006D42DD40AC4663460D000342DFD03323D8
:107AF0009A1A323B93401818874200D94C1C6346AF
:107B00009843D2E7C90FCC070020531CCDD1074BB7
:107B10001C43CAE706000D000028C0D1C7E7C046D5
:107B200001FCFFFFFFFF0F00EDFBFFFF0000F03F38
:107B300030B5214A4B0087B05B0893421EDD1F4AD7
:107B4000934205DD02000B0002F0D4FF07B030BD08
:107B500002AA00F095F803231840049A059B012817
:107B600013D002281DD0002814D00298039900F0E9
:107B70006FFB80231B069C466144E7E7002300223D
:107B80000093002301F0DEF8E0E70298039900F08B
:107B90005FFBDBE7012402980399009401F0D2F81F
:107BA000D4E7012402980399009401F0CBF88023D4
:107BB0001B069C466144C9E7FB21E93FFFFFEF7FBD
:107BC000F0B54746CE4680B58DB004000D0000F0FC
:107BD00067FA294B06001B780F005BB29846013309
:107BE00010D022002B002000290003F0CBFA8146A0
:107BF000002807D1002200232000290001F014FCF6
:107C0000002806D1300039000DB00CBC90469946D2
:107C1000F0BD01230293194B0694079503934B463D
:107C20000A93434604940595002B15D000230022A7
:107C30001900100002F0E2F8434608900991022B67
:107C40000ED103F0B9FB212303600A9B0193002BA3
:107C50000CD1089E099FD5E70023002408930994BE
:107C600002A801F0C1F90028EFD1EAE703F0A4FB74
:107C70000A9B01930360ECE77C000020F0DE00002B
:107C8000F0B54E464546DE465746E0B5E14B4C0062
:107C90008FB09046894664089C4200DC87E0DE4B4A
:107CA0009C4222DCDD4A002900DC92E0DC4B02F041
:107CB00021FFDB4B06000F009C4200D17EE1D94A38
:107CC000D94B02F017FF02000B00414630000A605A
:107CD0004B60390002F00EFFD34BD24A02F00AFF8C
:107CE000434601259860D9606BE0D04B9C4200DC94
:107CF0008FE0CF4B9C4200DD55E1CE4A23159246E2
:107D00009A4451460905631A19001D00040003F046
:107D100055FA03F089FA02000B00200029000892AE
:107D2000099302F0E7FE0022C34B02F071FC0F0042
:107D3000060003F043FA03F077FA04000D00020096
:107D40000B00300039000A940B9502F0D3FE00229C
:107D5000B94B02F05DFC002200230C900D9101F064
:107D60005DFB002800D192E10023002220002900C1
:107D700001F054FB434243410133B04A4146019272
:107D8000022208A80092524600F07CFB4B460500F8
:107D9000002B16DA802243461206944642465B6860
:107DA000454263445360D3686344D36009E00B00E9
:107DB000020041460A604B600022002300258A60D1
:107DC000CB6028000FB03CBC90469946A246AB461B
:107DD000F0BD934B01F0F6FC914B06000F009C4266
:107DE00000D13DE18F4A904B01F0ECFC02000B000A
:107DF000414630000A604B60390002F07BFE894A40
:107E0000894B01F0DFFC012543466D429860D96043
:107E1000D7E701F049F88A4A8A4B06000F0002F0C2
:107E2000F7FB0022884B01F0CDFC03F0C7F90500F9
:107E300003F0FAF9794A7A4B0490059102F0E8FBD5
:107E400002000B003000390002F054FE754A0600B3
:107E50000F0004980599744B02F0DAFB029003912D
:107E60001F2D00DCC7E0029A039B3000390002F0AE
:107E700041FE83468A4653465B0024155B0DE31A98
:107E8000102B6CDD04980599D322674B520502F044
:107E9000BFFB02000B00300039000292039302F096
:107EA00029FE0A0001001300069107920200390022
:107EB000300002F01FFE029A039B02F01BFE060038
:107EC0000F0004980599614A614B02F0A1FB320052
:107ED0003B0002F00FFE069E079F0B0002003900D8
:107EE00030000292039302F005FE4B005B0D8346C7
:107EF0008A46E41A312C32DD04980599B822544B95
:107F0000920502F085FB03000C000200029303942B
:107F10000B000698079902F0EDFD02000B00060029
:107F20000F000698079902F0E5FD029A039B02F004
:107F3000E1FD484A0290039104980599464B02F0EE
:107F400067FB029A039B02F0D5FD02000B00300094
:107F500039000292039302F0CDFD83468A465A46C9
:107F60005346414630000A604B60390002F0C2FDC2
:107F7000029A039B02F0BEFD44460B000200A26081
:107F8000E3604B46002B00DB1BE75B46236080234E
:107F90001B065344636080231B069C466144A0601B
:107FA000E1606D420DE70B00020002F0A3FD4346C5
:107FB00000259860D9601860596002E7D3221A4BF7
:107FC000520502F097FD214A214B0D00040002F0FA
:107FD00091FD02000B00414620000A604B60290021
:107FE00002F088FD1A4B194A02F084FD4346012530
:107FF0009860D960E5E602000B003000390002F01D
:1080000079FD6B1E154A9B009B5883468A46A34206
:10801000A5D130E7FB21E93F7BD902400000405465
:10802000FB21F93F3163621A61B4D03DFB21394134
:10803000FFFFEF7FEAFBFFFF0000704178DF0000E9
:1080400083C8C96D305FE43F0000E03F7370032ECA
:108050008A19A33BC14920259A837B39F8DE0000A9
:10806000D3220C4B520501F0ADFB0B4A0B4B040025
:108070000D0001F0A7FB02000B00414620000A6042
:108080004B60290002F036FD034A044BB9E6032396
:1080900073E6C04661B4D03D7370032E8A19A33BCA
:1080A000F8B54746CE46674B80B50A000F00190069
:1080B00005003940994200D19BE004000100002FE7
:1080C00069DD3F1500D1B4E05F4B12039C4680236D
:1080D000120B5B0313435B00CA0F67449B184A00F3
:1080E000F80703D5D20F5B009B188A0079108C46E5
:1080F000002180201624894680030D189D4202DC51
:1081000029185B1B8144D50F5B00013C5B195200B1
:108110004008002CF1D10020804680202025002737
:10812000000609E08B425CD0D40F5B00013DE318F0
:1081300052004008002D16D0C4198B42F2DD2718DA
:108140000E00002C49DB5B1AA242894149425B1AAE
:10815000121BD40F5B00013D80443100E318520034
:108160004008002DE8D113434ED143465B08374900
:108170004A468846494652104244C90702D58021E2
:1081800009060B4361460F05BD18180029000CBCF9
:1081900090469946F8BD7B005B0803433900002BED
:1081A000F5D0002F3CD1E30A153A6405002BFAD034
:1081B0008020400303423FD1002700E00F005B0016
:1081C000791C0342FAD0250020208D40401A290056
:1081D000D71B2200C2401A4376E7FE43F60F8E19E2
:1081E000B1E79442A0D82718002CF6DB1E0000232C
:1081F000AEE702003B002800390002F009FA2A002D
:108200003B0001F0DFFAC2E74346013303D04346A7
:1082100001335B08ABE7012398460023C144A6E77E
:108220003B00020002F066FC02000B0001F0E6FDDC
:10823000ADE713000022BBE70127210020207F4289
:10824000C6E7C0460000F07F01FCFFFF0000E03FF2
:10825000F0B54746CE4680B587B000920193754B86
:108260004F00814688467F089F4263DC02F0A6FFEC
:10827000002800D1D4E04A4643464846414602F031
:10828000C7F904000D006C4A6C4B02F0C1F96C4A4E
:108290006C4B01F097FA22002B0002F0B9F96A4A00
:1082A0006A4B02F027FC22002B0002F0B1F9684A69
:1082B000684B01F087FA22002B0002F0A9F9664A08
:1082C000664B02F017FC22002B0002F0A1F9644A71
:1082D000644B01F077FA22002B0002F099F902902A
:1082E00003910022604B2000290002F091F9029ACC
:1082F000039B06000F002000290002F089F9009A74
:10830000019B04000D004846414602F081F902003D
:108310000B002000290002F0EDFB02000B003000F2
:10832000390002F0E7FB02000B0000204F4902F089
:10833000E1FB70E002000B0002F06AF904000D009E
:108340003D4A3E4B02F064F93D4A3E4B01F03AFA99
:1083500022002B0002F05CF93B4A3C4B02F0CAFBC6
:1083600022002B0002F054F9394A3A4B01F02AFA64
:1083700022002B0002F04CF9374A384B02F0BAFBCE
:1083800022002B0002F044F9354A364B01F01AFA6C
:108390002B00220002F03CF9354B029003919F42E2
:1083A0009FDD344B00229F423DDC334900207B1887
:1083B0002E4916001F0002F09DFB0490059100223B
:1083C000294B2000290002F023F932003B0002F083
:1083D00091FB029A039B06000F002000290002F087
:1083E00017F9009A019B04000D004846414602F02F
:1083F0000FF902000B002000290002F07BFB0200B5
:108400000B003000390002F075FB02000B000498ED
:10841000059902F06FFB07B00CBC90469946F0BD81
:1084200000201249F7E7154B002604920593144FDC
:10843000C5E7C046FFFF3F3ED43888BEE9FAA8BD75
:10844000C4B1B4BD9EEE213EAD529C804F7E923EA3
:108450009015CB19A001FA3E7751C1166CC1563F59
:108460004C5555555555A53F0000E03F0000F03FE5
:108470003233D33F0000E93F0000E0FF0000E73F58
:108480000000D23FF0B5DE464E4645465746E0B5C1
:10849000DC4CA5440D9114001900A49A0993DA4B01
:1084A0009200D6584D1E03901821E01E06960295A4
:1084B00000F0AAFEC3430100DB1719404B1C9A00D1
:1084C0009B1ADB001B190B9105934C1B771918D4D1
:1084D000A59BA5009C463F1922AE6544013707E0E5
:1084E000286802F0A1FE013403C60435BC4208D05E
:1084F000002CF5DA00200021013403C60435BC420B
:10850000F6D1069B002B01DA00F0FDFB069B0399D8
:108510000133DB009A46099BDA0094460092002260
:10852000914672AA0492B94A6144934688469AAB2E
:1085300063449B44029B002B00DABCE15D460026AD
:108540000027039C4D442A686B6803CC02F060F856
:1085500002000B003000390001F034F9083D06003C
:108560000F004445EFD1049B4B441E605F6008231D
:108570009C46E144D145DDD10EA804218446494200
:1085800061448C46069A93009C44614684460A9155
:108590000399083B63448C460C93009B0092634410
:1085A0009B46009A0498D10003008C4663440891CE
:1085B0001E685F68002A33DD954980468C46624418
:1085C000D300984470AB9A460EAB99460022914B6B
:1085D0003000390002F01CF802F0F0FD02F024FE39
:1085E00000228D4B04000D0002F012F802000B0077
:1085F0003000390002F07EFA02F0E0FD4B4601C384
:108600009946434620001A685B68290001F0DAF8B1
:1086100008235B429C46E04406000F00D045D5D1BC
:10862000059B30001A003900984600F0DFFCFF235C
:1086300000229B0504000D0001F0EAFF00F038FC69
:108640000022764B01F0E4FF02000B00200029001D
:1086500002F050FA0D00040002F0B0FD814602F075
:10866000E3FD02000B002000290002F043FA06009F
:1086700040460F00002800DCEEE0009B18215A1E47
:1086800092000EAB9B58091A1D000D41A9448D4064
:108690005D1B0EAB9D5017231B1A1D41002D2DDDB8
:1086A00001239C46009BE144002B00DC1CE20E9C55
:1086B0000123002C00D0B5E0009A012A09D09900CE
:1086C0000EAA54580133002C00D0ACE0009A9A4214
:1086D000F5D1059B002B0EDD012B00D1A8E1022B6B
:1086E00009D1009B0EA95A1E92000EAB9B5807930E
:1086F0009B029B0A8B50022D00D1C1E00023002277
:108700003000390000F08AFE009B002800D194E27E
:10871000069A591E8A4210DC414A0A9894460EAACB
:108720006344944600229B0063441C68043B22433C
:108730008342FAD1002A00D0C0E0069B0EAA013B7A
:108740009B00D358002B00D0B3E001220C9B043BCC
:10875000596801320029FAD0009B9C4662441100FE
:1087600007921A0001338B4246DC0B986346804621
:10877000A59C4344A046099C9B00A1464A449844BA
:10878000D30022AA9146049A99449446089BA59A3C
:1087900063448446614494469A468B006344009344
:1087A0004346586802F040FD4B4618605960029BF2
:1087B000002B24DB4D46039C0026002701E028689F
:1087C00069680CCC01F024FF02000B003000390076
:1087D00000F0F8FF083D06000F005C45EFD153465E
:1087E0009E60DF6004239C460433E0449C46009B6B
:1087F000E144E2449845D3D1079B0093D1E600269B
:108800000027ECE794FDFFFFC0E0000018FEFFFF2B
:10881000FFFFFF1F0000703E00007041000020407D
:10882000FFFFFF3F002180225204141B0EAA545068
:10883000009999420EDD0EA884469B000EAA89007D
:10884000D25861446344CF4800E01A68821A04C3D6
:108850008B42FAD101243CE7059B002B06D1009BFB
:108860000EAA013B9B00D558ED1517E70022C64B19
:10887000300000F0F7FD002800D024E100253DE79E
:1088800032003B000020C14902F034F906000F001D
:10889000002C00D132E7059A0020BC4900F0A6FB6D
:1088A00002000B003000390002F024F906000F002E
:1088B00024E7012250E70026002754E64B46059A9C
:1088C000079388468B000EA9CB58183A0895059255
:1088D000002B0DD18C464146AD4B43449B00634475
:1088E000043B58680139183A0028F9D088460592A7
:1088F000059A0020A54900F079FB434604000D00CD
:10890000002B00DA05E29E000EAB9C464346DB00DE
:1089100066449C46059370AB9946049F6744009754
:10892000306802F081FC22002B0001F071FE002271
:1089300038607960974B2000290001F069FE083FFC
:1089400004000D00043EB945EAD14AAB03939B46AF
:1089500000239A46069B42469946434601320292BC
:1089600004934B46002B00DAAAE080208A4B009D3E
:108970009846C005894900260027002408E00823FE
:108980009C460835E044544511DC43461868596854
:108990002A686B6801F03CFE02000B0030003900D1
:1089A00000F010FF013406000F00A145E7DA5B4636
:1089B000C0C39B4601239C46009BE244083B0093B6
:1089C000029B9A45CDD1049B9846A49B022B00DDC7
:1089D0008EE0002B37DC1FD1059B00271D00039B79
:1089E00000249C461E006544083E2A686B683800D7
:1089F000210000F0E7FE083D07000C00AE42F4D174
:108A0000089B002B03D080231B069C4664443A003D
:108A100023000D990A604B600720079B18409B2399
:108A20009B009D443CBC90469946A246AB46F0BD97
:108A3000009B0EA95A1E92000EAB9B5807935B0237
:108A40005B0A8B5057E64346002B00DA70E10020AA
:108A50000021DB004AAAD61848AF32687368083E86
:108A600000F0B0FEB742F8D1089B002B00D025E102
:108A70000B0002004A984B990D9C2260636002F043
:108A800039F8434607000C00002B13DD01254CAEDE
:108A9000B14638002E0021004C4601360CCC00F0C7
:108AA00091FEA146B045F7DA089B07000C00002BA9
:108AB00000D015E13A0023000D998A60CB60ABE746
:108AC0000026002773E701239C46009BE144022512
:108AD000002B00DDEBE532003B0000202B4902F0CB
:108AE00009F806000F0009E60024F2E54AAB0393FB
:108AF000A49B032B00D08FE74346002B00DC14E13E
:108B0000039ADB009B46130091465B441E685F6836
:108B1000234B43440293DB00994448AB9A464B46AF
:108B20005C681B681800210032003B000090019136
:108B300000F048FE04000D0002000B0000980199AF
:108B400001F0D8FF3B00320000F03CFE4B4698603D
:108B5000D9601C605D6008235B429C46E1442600AE
:108B60002F00CA45DBD14346012B00DCE3E0039A2A
:108B700013005B441E685F68029BDB0099464A4411
:108B8000904610E0FFFFFF000000E03F0000F03FD4
:108B9000FFFFFF3F0000703E80E00000FB21F93F37
:108BA000FFFFFF1F984643465C681B6818002100C2
:108BB00032003B000090019100F004FE04000D0023
:108BC00002000B000098019901F094FF32003B0075
:108BD00000F0F8FD4346039A9860D9601C605D6020
:108BE000083B26002F009A42DCD14D4694460026D1
:108BF00000244746083565442A686B683000210028
:108C000000F0E0FD083D06000C00AF42F4D1039BEC
:108C10004A9F5D689968D868089B002B65D08022C0
:108C2000120694460D9B6544604464441F605D6079
:108C30009960D8601E615C61EEE69A464B460793E8
:108C4000059B30005A423900089500F0CFF9002208
:108C50003A4B06000F0000F005FC002824D0384BEA
:108C600000223000390001F0D3FC02F0A7FA52468E
:108C70000400950002F0D8FA0022304B01F0C8FC45
:108C800002000B003000390001F034FF02F096FAC8
:108C90000EAA50510122059B524418339046059369
:108CA00093000EAAD45023E65346300039009C00AE
:108CB00002F084FA0EAB1851D04619E680230D9AC3
:108CC0001B06CB18106053600B0002004A984B99AA
:108CD00001F010FF434607000C00002B00DDD5E635
:108CE00080231B069C466444E4E62B003A000D9D5D
:108CF0002A606B600A000300AA60EB603200230068
:108D00002A616B6188E6099BDB00009372AB0493D8
:108D100032E4A49B022B00DDE8E6002B00DD92E6A6
:108D200000D079E6002700246AE6002600246EE7DA
:108D30000020002198E60026340068E7000070411A
:108D40000000703EF0B5CE46474680B587B0009231
:108D50000193474A4B00814688465B08934207DCF3
:108D60004146484602F02AFA4146031E484666D06C
:108D70004A4643464846414601F04AFC04000D007D
:108D800002000B004846414601F042FC394A3A4B8A
:108D900006000F002000290001F03AFC374A384B4A
:108DA00001F0A8FE22002B0001F032FC354A364BC0
:108DB00000F008FD22002B0001F02AFC334A344B5E
:108DC00001F098FE22002B0001F022FC314B324AC8
:108DD00000F0F8FC0E9B02900391002B34D0009819
:108DE000019900222D4B01F013FC029A039B049081
:108DF00005913000390001F00BFC02000B000498D3
:108E0000059901F077FE22002B0001F001FC009A89
:108E1000019B01F06FFE224A04000D00214B30003F
:108E2000390001F0F5FB02000B002000290000F0E2
:108E3000C9FC02000B004846414601F05BFE07B04A
:108E40000CBC90469946F0BD02000B0020002900A2
:108E500001F0DEFB124A134B01F04CFE32003B00E6
:108E600001F0D6FB4A46434600F0ACFCE7E7C046BB
:108E7000FFFF3F3E7CD5CF5A3AD9E53DEB9C2B8A8C
:108E8000E6E55A3E7DFEB157E31DC73ED561C119E7
:108E9000A0012A3F1111813FA6F810110000E03F08
:108EA000495555555555C53F49004B081900704760
:108EB000474AF0B54F4691464B005B0D99444646F4
:108EC000D6464A46C0B505000C000E00884607008D
:108ED000132A27DC002A4BDB3E4B13419A460B003A
:108EE00052461340034318D03B4A3C4B2800210014
:108EF00000F068FC0022002300F0AAFA002847D006
:108F0000002C04DA80234A465B031341984446460A
:108F1000534600279E43380031001CBC90469946BA
:108F2000A246F0BD332A08DD8023DB009945F4D149
:108F300002000B0000F046FCEFE7294A94460122AC
:108F400063445242DA4092460242E6D0224A234B20
:108F50002800210000F036FC0022002300F078FAFF
:108F6000002815D0002C1EDB534646469F430FE0D9
:108F7000194A1A4B2800210000F024FC002200238B
:108F800000F066FA002803D0002C04DB002700263E
:108F900038003100C1E76400640825430027002D34
:108FA000F6D0104EF4E74B46142B0BD03422D21AD5
:108FB000012393405D19BD4208D201239C462F0036
:108FC000E044D1E7133B9C46E044CDE72F00CBE7DC
:108FD00001FCFFFFFFFF0F009C7500883CE4377E1B
:108FE000EDFBFFFF0000F0BF002070474B0070B5A5
:108FF0005B0D14000A00002B1AD14B005B080343E1
:1090000015D0234B002201F003FB224B9C422DDBA9
:109010000A004B005B0D363B1F4DE318AB422ADCC8
:10902000002B0DDD1D4C1B0522401A43110070BDA5
:109030001B4DAB42F0D102000B0000F0C3FBF6E782
:109040001D00353519DA174B02009C4209DD0B0073
:109050001548164900F032F8134A144B01F0D8FABB
:10906000E5E70B001248134900F028F8104A114BAD
:1090700001F0CEFADBE70200E9E7084C3633224084
:109080001B051343190000220B4B01F0C1FACEE778
:1090900000005043B03CFFFFFE070000FFFF0F80C1
:1090A000FF07000050C300009C7500883CE4377E39
:1090B00059F3F8C21F6EA5010000903C30B54A007C
:1090C000DB0FDB0752081A43110030BD02B47146B2
:1090D00049084900095C49008E4402BC7047C046FB
:1090E00003B47146490840004900095A49008E44BA
:1090F00003BC7047002243088B4274D303098B42A0
:109100005FD3030A8B4244D3030B8B4228D3030C57
:109110008B420DD3FF22090212BA030C8B4202D3F9
:109120001212090265D0030B8B4219D300E0090A21
:10913000C30B8B4201D3CB03C01A5241830B8B422A
:1091400001D38B03C01A5241430B8B4201D34B0313
:10915000C01A5241030B8B4201D30B03C01A524178
:10916000C30A8B4201D3CB02C01A5241830A8B42FD
:1091700001D38B02C01A5241430A8B4201D34B02E6
:10918000C01A5241030A8B4201D30B02C01A52414A
:10919000CDD2C3098B4201D3CB01C01A52418309FE
:1091A0008B4201D38B01C01A524143098B4201D338
:1091B0004B01C01A524103098B4201D30B01C01A63
:1091C0005241C3088B4201D3CB00C01A52418308DD
:1091D0008B4201D38B00C01A524143088B4201D30A
:1091E0004B00C01A5241411A00D20146524110466A
:1091F0007047FFE701B5002000F0F0F802BDC0465F
:109200000029F7D076E7704703460B437FD400224E
:1092100043088B4274D303098B425FD3030A8B420A
:1092200044D3030B8B4228D3030C8B420DD3FF2274
:10923000090212BA030C8B4202D31212090265D042
:10924000030B8B4219D300E0090AC30B8B4201D3F5
:10925000CB03C01A5241830B8B4201D38B03C01A3C
:109260005241430B8B4201D34B03C01A5241030BB3
:109270008B4201D30B03C01A5241C30A8B4201D364
:10928000CB02C01A5241830A8B4201D38B02C01A0F
:109290005241430A8B4201D34B02C01A5241030A86
:1092A0008B4201D30B02C01A5241CDD2C3098B426B
:1092B00001D3CB01C01A524183098B4201D38B01E8
:1092C000C01A524143098B4201D34B01C01A52418B
:1092D00003098B4201D30B01C01A5241C3088B42D0
:1092E00001D3CB00C01A524183088B4201D38B00BB
:1092F000C01A524143088B4201D34B00C01A52415D
:10930000411A00D201465241104670475DE0CA0F33
:1093100000D04942031000D34042534000229C46F3
:1093200003098B422DD3030A8B4212D3FC228901FD
:1093300012BA030A8B420CD3890192118B4208D3D3
:10934000890192118B4204D389013AD0921100E035
:109350008909C3098B4201D3CB01C01A5241830949
:109360008B4201D38B01C01A524143098B4201D376
:109370004B01C01A524103098B4201D30B01C01AA1
:109380005241C3088B4201D3CB00C01A524183081B
:109390008B4201D38B00C01A5241D9D243088B4271
:1093A00001D34B00C01A5241411A00D20146634614
:1093B00052415B10104601D34042002B00D5494278
:1093C000704763465B1000D3404201B5002000F0B7
:1093D00005F802BD0029F8D016E770477047C0466F
:1093E000D0400B1C1141203A03D49C461341184332
:1093F00063465242934018437047C0468446101C4F
:1094000062468C46191C634600E0C0461FB501F059
:1094100097F8002801D40021C8421FBD10B500F004
:10942000EFFF4042013010BD10B501F089F800286F
:1094300001DB002010BD012010BDC04610B501F0B9
:109440007FF8002801DD002010BD012010BDC046BE
:1094500010B501F011F8002801DC002010BD01203A
:1094600010BDC04610B501F007F8002801DA002051
:1094700010BD012010BDC046F0B5CE4647461504CC
:109480002D0C2E0080B50704140C3F0C9946030CDC
:109490007E435D43674363437F19340CE4199C4664
:1094A000A54203D980235B029846C4444B464343FC
:1094B0005143250C36046544360C2404A4195B1969
:1094C000591820000CBC90469946F0BDF0B54E46A8
:1094D00057464546DE46E0B543025B0A450083B089
:1094E0000F1C99462D0EC60F002D57D0FF2D24D0EE
:1094F0008020DB00C0041843002381469A469B4627
:109500007F3D7C027A00FB0F640A120E984623D03E
:10951000FF2A4BD0E30080240020E4047F3A1C4360
:10952000AD186B1C47460193534677403A000F2B0A
:1095300048D87D499B00CB589F46002B00D085E042
:1095400008339A46063B9B467C027A00FB0FFF25B8
:10955000640A120E9846DBD1002C00D090E05246EF
:1095600001231A4392460120DBE74C465846170078
:10957000022824D0032800D1CFE0002200230128B4
:109580004DD15802D205400AFF071043384303B0BB
:109590003CBC90469946A246AB46F0BD002B5BD141
:1095A00004239A46033B00259B46AAE7FF35002C7F
:1095B00060D1524602231A4392460220B1E7FF22AD
:1095C0000023DEE74B461B0C9C464B462604360C1C
:1095D000180461463300220C6446000C43434E439A
:1095E0005043544380191A0C1218964203D9802113
:1095F00049028C4664441B041B0C1004C0188301F0
:109600005E1EB341800E1843130C1B199B010343CC
:109610001C00230179D5012362081C401443019AE0
:109620007F32002A4DDD630704D00F232340042B33
:1096300000D00434230103D53C4B019A1C408032F6
:10964000FE2ABCDCA3015B0AD2B29AE70C239A463D
:10965000093BFF259B4654E7180001F071FE4A467E
:10966000431F76259A4000236D4291462D1A9A4653
:109670009B4646E7524603231A439246032050E78F
:10968000200001F05DFE431F2D1A9C40763D002016
:1096900047E780230027DB03FF2272E7424666E7A5
:1096A0004C463200584662E780234A46DB031A42A2
:1096B00022D01C4220D123435B025B0A4746FF2293
:1096C0005FE701239A1A1B2A21DC23000199D3406A
:1096D0009E318C401A0023005C1EA34113435A079D
:1096E00004D00F221A40042A00D004335A0111D4A6
:1096F0009B015B0A002244E780234A46DB031343B5
:109700005B025B0A3700FF223BE7019587E70022F7
:10971000002336E70122002333E78023DB032343C2
:109720005B025B0AFF222CE7D0E00000FFFFFFF79F
:1097300070B500283DD0C317C5185D40C40F280080
:1097400001F0FEFD9E22121A962A07DCD2B20828EA
:1097500033DD083885406802400A23E0992A0BDD92
:10976000052329001B1AD94003001B339D402B0001
:109770005D1EAB4119430D00052801DD431F9D40CF
:109780002B000F490B406E0709D00F263540042DE2
:1097900005D004335D0102D59F220B40121A9B01B4
:1097A000580AD2B24002D205400AE40710432043CF
:1097B00070BD002400220020F4E76802400AF1E7AF
:1097C000FFFFFFFBF0B54F464646D6460C000903A7
:1097D000C0B5490A470F5E0039431F03DB0F9C46A3
:1097E00065007B0A570F1F436D0DE40F760DA146F0
:1097F000C000B846D200AB1B64457BD0002B5FDDB8
:10980000002E00D0A4E03E00164300D112E15E1EFF
:10981000002E00D09EE1871A4346B84280410125C0
:10982000C91A4042091A0B0200D431E149024E0A1A
:10983000002E00D16EE1300001F082FD0300083BF4
:109840001F2B00DD61E120223900D21A9E40D14059
:109850009F400E439D4200DD51E15D1B6B1C1F2BA1
:1098600000DD7CE12021C91A3D0030008F40884096
:10987000DD40791E8F41310007222843D940002561
:1098800007433A40002A09D00F233B40042B05D060
:109890003B1DBB42BF417F42C9191F000B0200D4D0
:1098A00026E26A1CC64B55056D0D9A4200D106E1B1
:1098B000C44AFF080A40530752023B43120B8EE092
:1098C000002B00D0B8E06B1C5B055B0D012B00DCAE
:1098D00030E1871A4346B842B641CB1A76429E1B06
:1098E000330200D54CE13B003343A1D100220024D8
:1098F000002570E0002B00DCE5E0002E00D183E0C5
:10990000AF4EB54260D0802636043743B846382B78
:1099100000DC3EE1434613431F007A1E97413F1887
:1099200087428041404209180B0200D4B0E0A44BAA
:1099300001359D4200D1C3E0A24A7B080A400121C3
:109940000F401F435108D30707221F433A4099E7AE
:109950009B4EB54238D0802636043743B846382B64
:1099600000DDDCE01F2B00DC30E11E004746203E1E
:10997000F740BC46202B04D04026F31A46469E40B2
:109980003243170063467A1E97411F43CCE0002BF9
:1099900000D104E24346134300D159E14B07C0080C
:1099A00018438023C9081B03194208D04546ED0817
:1099B0001D4204D14346D008590708432900420FED
:1099C000C9007F4D1143C0004B07CA087C49C0083D
:1099D00003438D4268D012036D05120B6D0D0021FB
:1099E00012031800130B0A0D12051A43764B2D05AE
:1099F00013402B435B00E4075B08234319001CBCA6
:109A000090469946A246F0BD3E00164312D05E1E17
:109A1000002E00D000E18718874280414144404237
:109A2000091801250B0233D5022585E7644633006A
:109A3000414610001D00C7E7002D00D0DAE00C0001
:109A40000443F3D05C1C00D19FE15D4CA64200D1E1
:109A50002FE1DB43382B00DD66E11F2B00DD83E1C6
:109A600020240500E41A0F00DD40D940A040434601
:109A7000A7405B1A441EA04198462F433843171A4B
:109A8000BA42924143465242991A64463500CAE6A8
:109A900007223A40002A00D0F6E64B07CA08484998
:109AA000FF083B438D4296D11900114300D19EE13E
:109AB000802109030A431203120B414D8FE7150061
:109AC000002200238BE7002B00D0C7E06B1C5F0552
:109AD0007F0D012F00DCF1E0394DAB4200D1B9E040
:109AE00085180A008542894142444942511807229B
:109AF000CF076D082F4349083A401D00C2E60722F0
:109B00003049ED1A31403A40BCE63E0028388640E4
:109B100000279FE6380001F013FC20308EE6434614
:109B200013431F007A1E9741C71BB8428041404231
:109B3000091A78E60E003B0006431343002D61D15D
:109B4000002E00D0F4E0002B00D11BE16446390068
:109B5000100039E71A4FBB427AD03300FFE63000DD
:109B60001F3DE840202B03D04021CB1A9E403743B5
:109B70007B1E9F41072207433A400021002589E7C9
:109B8000171A4346BA42B641591A76428E1B6446AA
:109B90004EE61F2B00DDADE020264746F61AB74003
:109BA000B9461700B246DF404E463E4337005646A0
:109BB000B240561EB24117434246DA408918AEE61B
:109BC000FF070000FFFF7FFFFFFF0F8020264746B3
:109BD000F61AB740B9461700B246DF404E463E433C
:109BE00037005646B240561EB24117434246DA404D
:109BF000891A99E77F4CA6425BD0802424045B42FB
:109C0000214327E7002E0CD1002B00D1CBE0644686
:109C100039001000774DD7E6764FBB4218D033009D
:109C200075E6002B14D04B07C00818438023C908E1
:109C30001B03194207D0FC081C4204D17907D00845
:109C40000843E14621004C46420FC9001143C000C1
:109C5000684DB9E61D0000220023C0E6002D5BD14F
:109C60000D00054300D1E2E65D1C00D1B0E0614D7E
:109C7000AE421FD0DB43382B71DC1F2B00DD96E09A
:109C800020250F00ED1AAF40B9460700AA46DF4075
:109C90004D463D432F005546A840D940451EA8419A
:109CA00088440743BF1897429241514241443500CE
:109CB0003AE6644635004146100085E60B00034352
:109CC000002D00D063E6002BF5D04346134300D1AE
:109CD0007AE68718874280410722414440420918AA
:109CE0003A400B0200D4D5E6434B01351940C9E593
:109CF000380069E61E004746203EF740BC46202B50
:109D000004D04026F31A46469E403243170063466D
:109D10007A1E97411F4302E6364DAE42CAD08025D7
:109D20002D045B422943A6E70843411E8841A6E66D
:109D3000002B00D148E6871A4346B842B641CB1AF9
:109D400076429E1B33024BD5171A4346BA429241C4
:109D5000591A5242891A072264463A4092E5014351
:109D60000F00791E8F419DE71C000F00203CE7404B
:109D7000202B03D04024E31A99400843411E884118
:109D800038437CE60022002425E6171A4346BA42EF
:109D90009241591A5242891A6446350043E54146B8
:109DA0001000144D10E680220024120380E61D00EE
:109DB0000F00203DEF40BC46202B03D04025EB1A7E
:109DC0009940084307006346781E87411F4369E7AF
:109DD000871897429B4141445B42C9183500A3E56F
:109DE0003B003343CED0072231003A4052E60023F5
:109DF0001A00F4E5FF070000FFFF7FFFF0B55746AC
:109E0000DE464E464546E0B5834607000E03480051
:109E100085B092461C00360B400DCD0F002800D1B6
:109E20009DE0954B984239D08023F6001B041E43D9
:109E3000924A7B0F33439946944603006344009350
:109E400000230026FF00029323031B0B98466300A8
:109E5000E40F52465B0D019400D1B3E086498B427A
:109E600000D19EE04246D100802212040A435146AE
:109E7000490F11438B46814952468C4600996344F1
:109E8000CB1A0021D20000932B0063409A460F2E7C
:109E900000D905E17A4BB6009B599F465B46334398
:109EA000994600D0B8E002230826002700900293CC
:109EB000CAE7CB463A0002990195019B9A460229CE
:109EC00027D0032900D180E2012944D06D49009BAD
:109ED0008C4663441C00002C38DD530700D013E28D
:109EE000D2085B46DB0109D55946674B19408B46C2
:109EF0008021C9008C46009B63441C00634B9C423C
:109F000007DC5B4664055F075B0217431B0B620DB2
:109F100002E000230027584A00211B031C0B0B0DF5
:109F20001B05234314055A4A380013401C4353466B
:109F30006400DB0764081C43210005B03CBC90466C
:109F40009946A246AB46F0BD0122524201231B1B9B
:109F5000382B00DCADE1002200230027DCE75B4664
:109F6000334399465ED0002E00D18AE1300001F0E3
:109F7000E7F903000B3B1C2B00DD7BE11D22D31A0C
:109F80005A460100DA4008398E4013005F463343D9
:109F900099468F403F4B00261B1A009300230293E3
:109FA00052E7414653460B433B499B468C46009B38
:109FB000634400935B46002B3BD1022300221E43E7
:109FC000022161E7434613439B4637D04346002BAB
:109FD00000D162E1404601F0B3F903000B3B1C2BBA
:109FE00000DD53E102004146083A914088461D21B8
:109FF000CB1A5146D9400B0041460B439B46534672
:10A0000093401A00009B25499C46604403008C46FF
:10A0100063440093002137E70323B14600900C26E8
:10A02000029311E7002300930133042600270293D3
:10A030000AE70323C3461E43032125E701331E43DA
:10A040000022012120E700239A46802300271B03DA
:10A05000094A61E7802349461B03194200D1E2E027
:10A060005946194200D0DEE00B431B0317001B0BBF
:10A07000A246014A50E7C046FF07000001FCFFFF6F
:10A0800010E10000FF030000FFFFFFFEFE070000DD
:10A09000FFFF0F800DFCFFFF01F8FFFFF30300003F
:10A0A000D94500D9CBE000D1C6E03C0048460027A6
:10A0B000009B013B00935B46160E1B021E431302DE
:10A0C000984633041B0C9946310C0191FFF798F820
:10A0D0004A4642430B04210C050019438A4207D922
:10A0E0008919013D8E4203D88A4201D9851E8919FA
:10A0F000881A0199FFF784F809048C464A4621041E
:10A1000064464243090C030021438A4204D9891959
:10A11000013B8E4200D8F1E02D041D43AB4643467F
:10A12000891A4246280C12041D0C5B46140C2200AE
:10A130001B041B0C5A4303946B434443029568432E
:10A140001B19150CEB189C4203D980246402A44609
:10A1500060441C0C15041B042D0C20185D19814251
:10A1600077D373D00C1AA24A7D1BAF42BF419446ED
:10A17000009B7F426344E01B1C00864200D1DBE071
:10A180000199FFF73DF84A4642430B04290C0700AA
:10A1900019438A4207D98919013F8E4203D88A425E
:10A1A00001D9871E8919881A0199FFF729F809042E
:10A1B0004A46894629044D464243090C0300294377
:10A1C0008A4207D98919013B8E4203D88A4201D9B4
:10A1D000831E89193F04891A3A00039F1A433800E5
:10A1E00013041B0C584381460298150C6F434343DC
:10A1F00045434846000C8446DB1963449F4203D91B
:10A20000802040028446654448461F0C00041B041D
:10A21000000C7D191818A94200D284E000D17FE01B
:10A2200001231A4357E680234A461B0313431B03AB
:10A230001B0BAA466F4A6FE6BA4200D935E74B4678
:10A24000DC0758087B081C43FF0734E70024AF42B3
:10A2500089D247444745A4415B466442A419641827
:10A26000013BA6421ED2A0426DD800D1B6E0241A0E
:10A270009B4678E703005A46283B9A4000279146C0
:10A2800088E6584601F05CF8203072E6030052463A
:10A29000283B9A4093460022B4E6504601F050F81D
:10A2A00020309AE6A642E2D1B845DCD9341A9B4662
:10A2B00059E71F2B65DC504C0099A4465C4661446D
:10A2C00008008C4011008240D940501E82410C434E
:10A2D00014435A46DA401300620709D00F22224085
:10A2E000042A05D02200141D9442894149425B187A
:10A2F0001A0262D50122002300270DE68A4200D807
:10A300000AE7831E891907E70F231340042B00D1A6
:10A31000E6E5171D9742924153429B44FA08E0E557
:10A32000002800D1D7E57118531EB14227D3A942A6
:10A3300015D358D01A0073E7002B00DC04E6012384
:10A3400000229B44CDE502234744474589415B42B7
:10A350009C46494289190C19E344241A03E74346F1
:10A360005F0047459B41B8465B429E19023A8919F6
:10A37000A94200D054E7404500D051E7ABE51A00B0
:10A38000F6E71F215F4649420C1BE740202B07D010
:10A390001A49009B8C46634418005B4683401A436D
:10A3A000501E82413A4307270023174009D00F214E
:10A3B000002311401400042995D122005F075B029D
:10A3C0001B0BD20817430022A6E5802359461B0326
:10A3D0000B431B0317001B0B064A9DE5BD42B2D879
:10A3E0009B460024BFE68045B9D31A00C3E7C046A8
:10A3F000FF030000FF0700001E0400003E040000F1
:10A40000F0B54F464646D6468446C0B58046194EFE
:10A4100018030F034D00000B5C0082463F0B6D0DCF
:10A42000C90F9146640DDB0F0120B5420AD0B4423A
:10A4300003D0A54201D157450CD01CBC904699468B
:10A44000A246F0BD66463E43F7D1AC42F5D1544634
:10A450001443F2D10120C845EFD1994207D0002D15
:10A46000EBD163461F433800471EB841E5E70020A3
:10A47000E3E7C046FF070000F0B54F464646D64624
:10A480004D00C0B50E03C90F8A462C491F035C005E
:10A490008046360B6D0D91463F0B640DDB0F8D42F0
:10A4A0001ED08C4216D0002D1ED130438446002C85
:10A4B00001D13A4323D06246002A1AD09A4529D0C6
:10A4C000514602200139084001381CBC904699468B
:10A4D000A246F0BD39001143E5D002204042F4E726
:10A4E0003043FAD1AC420FD0002C0FD13A43E7D021
:10A4F0000CE00122013B934318000130E5E763467D
:10A500000020002BE1D0DBE73A43E6D19A45D7D1D2
:10A51000A542D5DCA54205DBBE42D1D808D000203B
:10A52000BE42D2D250460123013898430130CCE7D5
:10A53000C845C5D80020C845F4D3C6E7FF070000CA
:10A54000F0B54F464646D6464D00C0B50E03C90F7E
:10A550008A462E491F035C008046360B6D0D9146DE
:10A560003F0B640DDB0F8D4218D08C4211D0002DB3
:10A5700018D130438446002C1ED13A431CD1634687
:10A580000020002B30D0514602200139084001380C
:10A590002AE039001143EAD0022025E03043FBD104
:10A5A000AC4226D0002C26D13A4324D15146022079
:10A5B00001390840013817E06246002A0FD09A4559
:10A5C000E1D1A54205DBBE42DDD819D00020BE4254
:10A5D0000AD25046012301389843013004E0012299
:10A5E000013B9343180001301CBC90469946A2469B
:10A5F000F0BD3A43D0D19A45C5D1A542C3DCE0E7CE
:10A60000C845C0D80020C845E3D3EDE7FF070000E8
:10A61000F0B55746DE464E464546E0B58346060051
:10A620000F03480087B092461D003F0B400DCC0F32
:10A63000002800D16FE0DE4B984238D08023FF0025
:10A640001B041F43730F3B430193DA4B00279946CA
:10A6500000239B46F60081442B0369001B0B5246E6
:10A660009846490DED0F002900D185E0D04B994265
:10A6700000D173E04346DA0080231B0413435246A3
:10A68000CC48520F84461343524600206144D20006
:10A6900089442100694000918C46012149448A4641
:10A6A0000F2F00D990E0C449BF00CF59BF465B4689
:10A6B0003B43019300D06AE102230827002681462C
:10A6C0009B46C9E732005846019B6146009102282B
:10A6D00000D175E0032800D1FEE1012800D02CE173
:10A6E00000230027002600253F032A0D3F0BB34817
:10A6F00012053A4302401B051343009A5B00D10741
:10A700005B080B433000190007B03CBC90469946EB
:10A71000A246AB46F0BD5B463B43019300D12FE11F
:10A72000002F00D1A5E1380000F00AFE03000B3B2A
:10A730001C2B00DD96E11D22D31A5A460100DA4097
:10A740005E4608398F4013008E403B4301939C4B7B
:10A7500000271B1A994600239B467DE74146534636
:10A760000B4393498C46E144002B00D01AE10222AE
:10A770000220174300228CE7134300D10DE143462A
:10A78000002B00D181E1404600F0DAFD02000B3AD7
:10A790001C2A00DD72E10100434608398B409846CF
:10A7A0001D239A1A5346D3401A0043461343524678
:10A7B0008A404946081A824989468144002068E750
:10A7C0007B4B002700268EE7140C1204120C11009C
:10A7D000370C3604350C794328008C462E00604334
:10A7E0006044834656432100300C804658467943E6
:10A7F00040440291844506D98846802149028C460E
:10A80000E044414602913604010C360C00048B46AC
:10A8100081191E0C1B041B0C0391190079438C46F3
:10A82000280075436544A8465843050C45447743C2
:10A83000A94203D9802149028C466744290C8C46E1
:10A8400039000004000C2D042D186144AB4405911F
:10A850005946049101990F043F0C080C39005143EB
:10A860004243904602008C46090C8B4662437C436F
:10A8700044445C44A04503D98021490288464244AF
:10A88000210C884661460904090C8C46390059435D
:10A89000434370437E430F0CF6182404BE196444EE
:10A8A00042448C46B34203D980235B02984640441D
:10A8B000029B61469846049B370443449B46AB4544
:10A8C000AD416B420D0405992D0C8C467F196744F0
:10A8D000FD18A8465D462D19A542A4419346644241
:10A8E000A446C344DC448F42BF4198459B419345F5
:10A8F0009241A445A4415B427F421F43360C524221
:10A900006442BF192243BF18624638184302D20D71
:10A91000039913436A020A43501E82416146ED0DBA
:10A920002A434E023243D90100D4B3E00126500835
:10A9300032400243DE0732435B08224C5444002C71
:10A9400062DD510709D00F201040042805D0101DEA
:10A950009042924152429B180200D90104D58024B2
:10A960001948E400034054441848844200DD27E7B6
:10A970005E075B02D2081F0B630516435B0DB2E650
:10A98000002399460133042700269B4664E60323EF
:10A99000019781460C279B465EE601220120174362
:10A9A000002276E6032303201F43434671E6C04698
:10A9B000FF07000001FCFFFF50E10000FFFF0F80D8
:10A9C0000DFCFFFFFF030000FFFFFFFEFE0700007E
:10A9D0000023802700933F030026434B83E6019B1F
:10A9E0003200A446584670E6AC466EE680270199D0
:10A9F0003F0339422DD03B422BD11F433F033F0B36
:10AA000000951600384B6EE601252D1B382D00DD14
:10AA100066E61F2D40DC35481C005044160082407D
:10AA20008440EE40501E824134431443EB406207A1
:10AA300009D00F222240042A05D02200141D94427E
:10AA4000804140421B181A023ED5012300270026F0
:10AA500049E68027019B3F031F433F033F0B0094C0
:10AA6000214B40E603005A46283B9A4000260192BB
:10AA70006DE6584600F064FC203057E6030052466D
:10AA8000283B9A401300002293E6504600F058FC01
:10AA900020307BE6CA4650E71F201E004042041BC0
:10AAA000E640202D03D0124C5444A3401A43501EBC
:10AAB0008241324307260027164009D00F20002389
:10AAC000104014000428B9D122005E075B021F0B5E
:10AAD000D2081643002306E680273F031F433F03A7
:10AAE0003F0B1600004BFEE5FF0700001E040000B0
:10AAF0003E040000F8B557464E464546DE460C007B
:10AB00000903E0B5490A460F5F0031431E03DB0F1E
:10AB1000760A9B46530F3343C84E6500C000E40FCE
:10AB2000D2006D0DA24681467F0D9C469046B742ED
:10AB300000D1B9E05B46012673409B46EE1BA3455E
:10AB400000D183E0002E63DD002F00D0B1E063462A
:10AB5000134300D123E1731E002B00D0BAE1861A03
:10AB60006346B04280410125C91A4042091A0B02CE
:10AB700000D447E149024B0A98464346002B00D1D6
:10AB800089E1404600F0DCFB0300083B1F2B00DDA1
:10AB90007CE120223000D21A4146D0409940020088
:10ABA0009E400A439D4200DD6AE15D1B6B1C1F2B2A
:10ABB00000DD94E1202110003500C91A8E40DA40F2
:10ABC0008840DD40711E8E41110007222843002578
:10ABD00006433240002A09D00F233340042B05D00E
:10ABE000331DB342B641764289191E000B0200D4D0
:10ABF0003DE26A1C914B55056D0D9A4200D119E159
:10AC00008F4AF6080A40570752023743120B9BE05F
:10AC1000002E00D0C5E06E1C7605760D012E00DCFE
:10AC200048E16746861ACB1BB042BF417F42B84617
:10AC30001F004346FF1A3B00B8461B0200D55FE1E8
:10AC400037439AD100220024002579E0002E00DC51
:10AC5000FAE0002F00D18DE0784B9D4267D0802331
:10AC600067461B041F43BC46382E00DC52E1634696
:10AC700013435A1E93411E188642804140420918D0
:10AC80000B0200D4BEE06D4B01359D4200D1D2E0F5
:10AC90006B4A73080A4001210E401E435108D30736
:10ACA00007221E43324095E71E00164300D045E7B9
:10ACB00040E7624B9D423AD0802367461B041F4306
:10ACC000BC46382E00DDEBE01F2E00DC3AE13300FD
:10ACD0006746203BDF403B00202E05D04027BF1BAE
:10ACE0006646BE40324390464646721E9641334306
:10ACF000DAE0002B00D114E26346134300D168E18F
:10AD000080234E07C008C9081B030643194208D018
:10AD10006046C008184204D163460100D2085E07AD
:10AD20001643F3009946C900720F444D11434B4638
:10AD3000DE08424B4F073743CA089D4200D16EE000
:10AD400012036D05120B6D0D00211203130B0A0D7A
:10AD500012051A433B4B2D0513402B435B00E407C0
:10AD60005B082343380019003CBC90469946A24634
:10AD7000AB46F8BD6346134311D0731E002B00D0C1
:10AD800007E1861886428041614440420918012546
:10AD90000B0237D502257BE73E0061469146350020
:10ADA000C5E75C46002D00D0E1E00B000343F3D083
:10ADB000731C00D1ACE1214B9F4200D13AE1F34337
:10ADC000382B00DD6FE11F2B00DD8CE120250E000C
:10ADD000ED1AAE40B0460600AA46DE404546354371
:10ADE0002E005546D940A8406346451EA8415B1A2F
:10ADF0009C463043161AB242924163465242991A17
:10AE00003D00B4E607223240002A00D0E4E60B4BB6
:10AE1000F6084F073743CA089D4200D090E73B0031
:10AE2000134300D1A6E180231B031A431203120B24
:10AE3000024D89E715000022002785E7FF07000083
:10AE4000FFFF7FFFFFFF0F80002E00D0C7E06B1CCD
:10AE50005E05760D012E00DCF0E0C84DAB4200D15E
:10AE6000B9E085180A008542894162444942511877
:10AE70000722CE076D082E43490832401D00A9E67F
:10AE8000BF49ED1A114007223240A3E632002838AC
:10AE90008240002686E6300000F052FA203073E649
:10AEA000634613435A1E9341C61AB0428041404242
:10AEB000091A5CE60E00674606431743002D5ED173
:10AEC000002E00D0F3E0002F00D11EE15C46614669
:10AED00091462CE7A94FBE427BD01E00F1E6100040
:10AEE0001F3DE840202B03D04021CB1A9A40164347
:10AEF000731E9E410722064332400021002583E74E
:10AF0000161A6346B2428041591A40420B1A9846BB
:10AF10005C4632E61F2E00DDABE02027BB1B9A46C5
:10AF200063465746BB40994613004F46F3401F43C4
:10AF30003B005746BA40571EBA4113436246F2409F
:10AF4000891898E62027BB1B9A4663465746BB40A4
:10AF5000994613004F46F3401F433B005746BA4003
:10AF6000571EBA4113436246F240891A9CE7834B4D
:10AF70009F425FD080252D047342294320E7002E95
:10AF80000CD1002F00D1D0E05C46614691467B4D4C
:10AF9000CDE67A4FBE421CD01E0065E6002F18D0C9
:10AFA000C0084E0706438020C9080003014208D0AC
:10AFB0006346DC08044204D12100DA46D2085E0769
:10AFC0001643F300994601245346C900720F1143FA
:10AFD0001C406A4DABE61D0000220027B4E6002DA0
:10AFE00059D10B00034300D1D6E6731C00D1B2E067
:10AFF000624B9F421ED0F343382B6FDC1F2B00DDCA
:10B0000097E020250E00ED1AAE40B0460600AA4695
:10B01000DE40454635432E005546A840D940451EE2
:10B02000A8418C440643B61896429241514261446D
:10B030003D0025E63D006146914678E60B0003435E
:10B04000002D00D055E6002BF5D06346134300D108
:10B050006DE686188642804161444042091800220C
:10B060000B0200D4D0E6464B01351940B2E5B1469B
:10B070005DE633006746203BDF403B00202E05D0D5
:10B080004027BF1B6646BE40324390464646721E6E
:10B0900096413343EFE5394B9F42CBD080252D04B9
:10B0A00073422943A8E70843411E8841A2E6002FC6
:10B0B00000D13CE66346861ACF1AB0429B415B4200
:10B0C000FB1A98461B024ED5161A6346B2429241AD
:10B0D000591A5242891A5C4600227BE501430E0050
:10B0E000711E8E419FE71D000E00203DEE40B046D0
:10B0F000202B04D04025EB1A99400843814648464E
:10B100004346411E8841184374E60022002417E696
:10B11000161A6346B2429241591A5242891A3D00A8
:10B1200025E561469146154D01E680220024120373
:10B1300079E61D000E00203DEE40B046202B04D0E5
:10B140004025EB1A9940084381464E464346711EFE
:10B150008E411E4367E7861896429B4161445B42DD
:10B16000C9183D008CE547463743CED007224146FB
:10B17000324049E600273A00E6E5C046FF070000F6
:10B18000FFFF7FFF70B50C4E0D031C0349005B00F1
:10B190002D0B490D240B5B0DB14208D00649002050
:10B1A0008B4203D114432000441EA04170BD0543CF
:10B1B0000120002DFAD1F1E7FF07000030B5144D52
:10B1C0000A034B00120B5B0DC90F0024AB4211DDCB
:10B1D000104CA34210DC8024640322430E4CE41A7A
:10B1E0001F2C0CDD0D48C31ADA4013005C42002905
:10B1F00000D11C00200030BD094BCC18FAE7094DE6
:10B20000E040AC4663449A4013000343EEE7C04677
:10B21000FE0300001D0400003304000013040000BE
:10B22000FFFFFF7FEDFBFFFF70B500282DD0C31798
:10B23000C5185D40C40F280000F082F8154B1B1A9A
:10B240005B055B0D0A2815DD0B38854000222D03B8
:10B250002D0B002110002D030A0D2D0B12052A4382
:10B260000D4D1B052A4013435B00E4075B08234395
:10B27000190070BD02002900153291400A000B210F
:10B28000081AC5402D032D0BE3E7002400230025F9
:10B290000022DEE71E040000FFFF0F804100090EC0
:10B2A0004B1C70B5DBB24602750AC40F012B14DDCE
:10B2B000E0239B006D07360BCB1800210A0D2800F8
:10B2C00012051C4D32435B052A405B0813435B00AB
:10B2D000E4075B082343190070BD002914D1002D39
:10B2E0001ED0280000F02CF80A281CDC0B232A00B2
:10B2F0001B1ADA40030015339D400F4B12031B1A33
:10B300005B05160B5B0DD8E7002D06D0320B8026AF
:10B3100036036D071643094BCFE7084B0026CCE7F1
:10B3200000230026C9E703002A000B3B9A400025B2
:10B33000E3E7C046FFFF0F8089030000FF0700001E
:10B340001C2101231B04984201D3000C10391B0A55
:10B35000984201D3000A08391B09984201D3000919
:10B36000043902A2105C40187047C0460403020270
:10B3700001010101000000000000000030B51C00C8
:10B38000094B05001B6885B0D868084B002A01D11D
:10B39000074B1A000292019300912B0022000549ED
:10B3A00000F026F800F0A6FD8000002090E10000EB
:10B3B000C4CF00009DE10000014B18687047C046F3
:10B3C00080000020084B10B50400002B02D00021A3
:10B3D00000E000BF054B1868836A002B00D0984737
:10B3E000200001F05DFBC04600000000CCE1000041
:10B3F0000EB403B5010003AB044804CB006801930D
:10B4000000F076F802B008BC03B0184780000020B6
:10B4100070B500260C4D0D4C641BA410A64209D13A
:10B42000002601F03FFB0A4D0A4C641BA410A64203
:10B4300005D170BDB300EB5898470136EEE7B30075
:10B44000EB5898470136F2E75002002050020020E6
:10B450005002002060020020002310B59A4200D163
:10B4600010BDCC5CC4540133F8E710B5884202D952
:10B470008B18984203D3002307E08B5C8354013A76
:10B48000FBD210BDCC5CC45401339A42FAD1F8E728
:10B4900003001218934200D1704719700133F9E785
:10B4A000936810B5013B9360002B04DA9469A342C2
:10B4B00007DB0A2905D01368581C106019700800B2
:10B4C00010BD00F04BFC0100F9E7F8B506000F00D5
:10B4D0001400D518AC4201D1002007E021783A00D1
:10B4E0003000FFF7DDFF0134431CF3D1F8BD00004D
:10B4F000F0B59FB002900F0016000593002805D00C
:10B5000083690493002B01D100F0F4FD7B4B9F4233
:10B510005BD1029B5F68BB891B0762D53B69002B2F
:10B520005FD0002306AC6361203363761033A376CB
:10B5300035002B78002B01D0252B5CD1AB1B04935D
:10B540000CD0320039000298FFF7BFFF431C00D136
:10B55000C4E06269049B9446634463612B78002BCA
:10B5600000D1BBE0012200235242626002A95432A2
:10B5700052186E1C2360E360A3601370A3653178DA
:10B5800005225F4800F0D4FE751C002835D12268E2
:10B59000D30604D5532302A95B1820211970130781
:10B5A00004D5532302A95B182B21197033782A2B59
:10B5B0002CD0350000210A20E3682A786E1C303A2E
:10B5C000092A64D900292ED026E04E4B9F4202D191
:10B5D000029B9F689FE74C4B9F429CD1029BDF6878
:10B5E00099E73900029800F00FFC002899D001205B
:10B5F00040421FB0F0BD01359BE7414B2268C01AA5
:10B6000001238340134323602E00B8E7059B191DD7
:10B610001B680591002B01DB099304E05B42E360AA
:10B620000223134323602B782E2B0AD16B782A2B0D
:10B6300035D1059B02351A1D1B680592002B2BDBAB
:10B640000793324E29780322300000F071FE002863
:10B6500006D04023801B83402268013513432360BA
:10B66000297806222A486E1C217600F061FE002807
:10B670003AD0284B002B25D10722059B0733934353
:10B68000083305936369039A9B18636150E743434A
:10B6900001219B18350090E701235B42D0E700238E
:10B6A0000A201A000135636029786E1C3039092997
:10B6B00003D9002BC5D00792C3E742430123521898
:10B6C0003500F1E705AB00933A00134B21000298D7
:10B6D00000E000BF0390039B0133D3D1BB895B061D
:10B6E00000D584E70B9884E705AB00933A000A4B3A
:10B6F0002100029800F080F8ECE7C04624E2000048
:10B70000D0E1000044E2000004E20000D6E10000C5
:10B71000DAE1000000000000CBB40000F7B515002E
:10B7200001938A680B6900900C00934200DA1300C1
:10B7300022002B6043321278002A01D001332B60A3
:10B7400023689B0602D52B6802332B6006272368EB
:10B750001F4027D0230043331B785A1E9341226891
:10B76000920630D42200019943320098089EB047D7
:10B77000431C25D0062320682A68E1680340002581
:10B78000042B03D18D1AEB43DB171D40A3682269FC
:10B79000934201DD9B1AED180027BD4220D1002005
:10B7A00010E00137E3682A689B1ABB42D2DD220011
:10B7B0000123193201990098089EB047431CF0D12B
:10B7C00001204042FEBD3020E118433108702100C5
:10B7D0005A1C45310978A218433202331170C1E76F
:10B7E000220001231A3201990098089EB047431C99
:10B7F000E6D00137D1E70000F0B589B004920A0025
:10B8000043320593039002920A7E0C000E9B6E2A2F
:10B8100000D186E01FD8632A33D008D8002A00D18F
:10B820008CE0582A4DD0250042352A7030E0642A39
:10B8300001D0692AF7D1196825680A1D280629D57B
:10B8400008681A60002803DA2D23029A4042137018
:10B850006B4E0A274FE0732A74D008D86F2A1FD086
:10B86000702AE0D1202209680A43226003E0752A89
:10B8700016D0782AD7D12200782145321170614E36
:10B8800022E025001A684235111D196013682B70DB
:10B89000012365E008681A606906D3D500B2D1E7D4
:10B8A00019682568081D186008682E0605D5544ECD
:10B8B00008276F2A1BD00A2719E06D06F7D580B23A
:10B8C000F5E745314E4E0A7018682268011D006880
:10B8D0001960150621D5D30702D520231A4322600B
:10B8E0001027002803D1202322689A4322602300D6
:10B8F000002243331A706368A360002B58DB0422D4
:10B90000216891432160002854D1029D002B5AD018
:10B910002500337842352B7055E05506DBD580B2D3
:10B92000D9E71A680D68101D4969186013682E065A
:10B9300001D5196002E06D06FBD519800023029D38
:10B9400023614FE01A68111D1960156800216268B3
:10B95000280000F0EDFC002801D0401B6060636807
:10B9600023610023029A13703CE023692A000499A2
:10B970000398059DA847431C3ED023689B0715D418
:10B98000079BE068984239DA180037E0220001236B
:10B99000193204990398059EB047431C2CD00135F9
:10B9A000E368079A9B1AAB42F0DCE9E70025F7E76A
:10B9B0000028ADD0029D3900FDF722FC735C013DEB
:10B9C0002B700028F7D1082F09D12368DB0706D593
:10B9D00063682269934202DC3023013D2B70029B95
:10B9E0005B1B2361059B07AA00932100049B03981E
:10B9F000FFF794FE431CB8D10120404209B0F0BDCE
:10BA0000E1E10000F2E100000D4B70B51C6805009B
:10BA1000A36B002B0FD1182000F06EFC094BA06324
:10BA20000360094B01224360084B83600B23838131
:10BA30000023026143610022A36B1D615A6170BD46
:10BA4000800000200E33CDAB34126DE6ECDE050035
:10BA5000124B10B51C68A36B002B0FD1182000F0FF
:10BA60004BFC0F4BA06303600E4B012243600E4B57
:10BA700083600B238381002302614361A46B0B4A23
:10BA8000206961690A4BFDF7F7FC01220023801849
:10BA90005941206161614800400810BD80000020CC
:10BAA0000E33CDAB34126DE6ECDE05002D7F954CE8
:10BAB0002DF451580CB430B5164B9DB00C1E1D68BA
:10BAC00008DA8B2301202B6040421DB030BC08BC3B
:10BAD00002B01847822302A99B008B8100230290A9
:10BAE00008619C4200D0631E8B604B6101235B4266
:10BAF000CB81209A21AB2800019300F055FD431C17
:10BB000001DA8B232B60002CDFD00023029A137004
:10BB1000DBE7C046800000200EB400B50B499CB0A6
:10BB20001DAB02900690079104910948094904CB86
:10BB30000591006802A9019300F036FD0023029AE6
:10BB400013701CB008BC03B01847C046FFFFFF7F4E
:10BB5000800000200802FFFF020010B51378541C7B
:10BB6000002B05D1CC5CD4540133002CFAD110BD8C
:10BB70002200F3E7C9B20378002B04D08B4200D136
:10BB800070470130F7E74B42594149420840F7E717
:10BB900002780B78002A03D0013001319A42F7D0A5
:10BBA000D01A70470023C25C0133002AFBD1581E13
:10BBB0007047002330B59A420AD0013AC45CCD5C8C
:10BBC000AC4204D1934202D00133002CF6D1631B66
:10BBD000180030BD30B50500002A00D130BD0C780A
:10BBE000013A6B1C2C700131002C05D19A189A4235
:10BBF000F4D01C700133FAE71D00EDE710B50378AF
:10BC0000002B0FD10B785A4253415B42184010BDB4
:10BC10000023CA5C002AFAD0C45C944201D10133EB
:10BC2000F7E701300378002BF2D11800EFE70000AE
:10BC3000F0B51F000E0087B00590019102920C989C
:10BC4000347800F0EAFA082200194378751C134092
:10BC500036D12D2C36D1B51C74780126002F62D038
:10BC6000102F09D1302C07D120222B789343582B49
:10BC700054D110276C7802352D4B3900F318180079
:10BC80000393FDF7BDFA049101210023494202000C
:10BC90008C4618002100303909291AD80C00A74217
:10BCA00023DD591C09D06346824206D302D1049990
:10BCB000A14202DB0123784320182C780135E9E703
:10BCC0002E00BCE72B2C01D01E00C7E7B51C7478F2
:10BCD000FAE721004139192901D8373CDFE7210073
:10BCE0006139192901D8573CD9E75A1C08D1059A5E
:10BCF00023331360029B0398002B09D107B0F0BDDA
:10BD0000002E00D04042029A002AF7D0002B01D02A
:10BD10006B1E0193029B019A1A60EFE73024002FFB
:10BD2000AAD10827A8E7302C9ED00A27A4E7C0464E
:10BD3000FFFFFF7F37B51300064A05001068046A4D
:10BD4000002C00D1044C0A0000942900FFF770FF7A
:10BD50003EBDC04680000020E4000020F8B505008C
:10BD60000E001400002804D08369002B01D100F0DC
:10BD7000C1F9224B9C422DD16C68A369A360A389B1
:10BD80001B0731D52369002B2ED023682269F7B217
:10BD9000981A6369F6B2834205DC2100280000F09E
:10BDA0003BF9002826D1A3680130013BA36023683A
:10BDB0005A1C22601F706369834204D0A389DB0789
:10BDC0001AD50A2E18D12100280000F025F90028E4
:10BDD00012D00FE00A4B9C4201D1AC68CDE7094B71
:10BDE0009C42CAD1EC68C8E72100280000F00CF89A
:10BDF0000028CAD0012676423000F8BD24E20000B7
:10BE000044E2000004E20000364B70B51D680600F5
:10BE10000C00002D05D0AB69002B02D1280000F0EA
:10BE200069F9314B9C420FD16C680C23E25E93B2EE
:10BE300019072DD4D90611D40923012033603733D3
:10BE40001343A381404270BD284B9C4201D1AC6892
:10BE5000EBE7274B9C42E8D1EC68E6E75B0713D59C
:10BE6000616B002908D023004433994202D030008E
:10BE700000F06AFA002363632422A3899343A38119
:10BE800000236360236923600823A2891343A381ED
:10BE90002369002B0BD1A0218022A3898900920065
:10BEA0000B40934203D02100300000F0E1F9012360
:10BEB000A289134011D00023A36063695B42A36190
:10BEC000002023698342BED10C23E25E1306BAD55B
:10BED00040231343A3810138B5E7920700D4636977
:10BEE000A360EDE78000002024E2000044E20000AF
:10BEF00004E2000010B5062000F090FC012000F0E4
:10BF0000CFFD0000F7B58A8905000C00130760D447
:10BF10004B68002B04DC0B6C002B01DC0020FEBD09
:10BF2000E76A002FFAD000232E682B6080235B0184
:10BF3000216A1A4034D0606DA3895B0706D5636817
:10BF4000C01A636B002B01D0236CC01A0200216A57
:10BF500000232800E76AB847A189431C06D12B6853
:10BF60001D2B30D82B4ADA40D3072CD50023636031
:10BF700023692360CB0405D5431C02D12B68002B19
:10BF800000D16065616B2E600029C7D02300443367
:10BF9000994202D0280000F0D7F900206063BEE784
:10BFA00001232800B847431CC6D12B68002BC3D0FF
:10BFB0001D2B01D0162B01D12E60AFE74023A289A3
:10BFC0001343A381ABE740230B430120A3814042ED
:10BFD000A5E70F69002FA1D00B680F60DB1B019351
:10BFE0000023920700D14B69A360019B002B00DC6A
:10BFF00094E7019B3A00216A2800A66AB04700280E
:10C0000003DC4023A2891343DFE7019B3F181B1A7F
:10C010000193EAE7010040200B6970B505000C00B0
:10C02000002B01D1002070BD002804D08369002BB3
:10C0300001D100F05FF80B4B9C4209D16C680C22D7
:10C04000A35E002BEED021002800FFF75BFFEAE79C
:10C05000054B9C4201D1AC68F1E7044B9C42EED108
:10C06000EC68ECE724E2000044E2000004E2000097
:10C07000002310B504000360436083608181436640
:10C08000C281036143618361190008225C30FFF7BC
:10C09000FFF9054B24626362044BA362044BE36225
:10C0A000044B236310BDC0465DC8000085C8000076
:10C0B000BDC80000E9C8000010B5024900F08CF8C6
:10C0C00010BDC04619C0000070B568254A1E554312
:10C0D0000E002900743100F081F9041E08D00021FF
:10C0E0002A00016046600C30A0606832FFF7D0F98A
:10C0F000200070BD836913B50400002B28D1836430
:10C10000C3640365134B144A1B688262019398420F
:10C1100001D101238361200000F020F8606020003D
:10C1200000F01CF8A060200000F018F80022E06089
:10C1300004216068FFF79CFF01220921A068FFF736
:10C1400097FF02221221E068FFF792FF0123A3610B
:10C1500013BDC046CCE10000B9C00000F8B51C4BCF
:10C1600007001E68B369002B02D13000FFF7C2FF41
:10C170004836B4687368013B04D53368002B07D098
:10C180003668F6E70C22A55E002D0DD06834F2E784
:10C1900004213800FFF798FF30600028F0D10C230D
:10C1A00004003B602000F8BD20000A4B6566256056
:10C1B0006560A560E36025616561A56108222900CD
:10C1C0005C30FFF765F96563A563A564E564E9E79D
:10C1D000CCE100000100FFFFF7B5040007000026D6
:10C1E00001914834002C01D13000FEBD6368A56880
:10C1F0000093009B013B009301D52468F2E7AB89D3
:10C20000012B08D90E22AB5E013304D0290038007F
:10C21000019B984706436835EBE7EC3000687047B0
:10C2200070B50E001D000E23C95E96B014000029E3
:10C2300007DA00232B60B3891B0611D48023DB00AF
:10C240000FE06A4600F088FB0028F2DBF022019B39
:10C2500012021340054A9B185A4253412B60EDE7E6
:10C2600040230020236016B070BDC04600E0FFFFF1
:10C27000F7B502268B8905000C00334206D0230057
:10C2800047332360236101236361F7BD01AB6A4635
:10C29000FFF7C6FF00990700280000F09FF800286C
:10C2A00008D10C22A35E9A05EFD4032293431E43C8
:10C2B000A681E4E70F4BAB628023A2892060134381
:10C2C000A381009B20616361019B002B0DD00E2395
:10C2D000E15E280000F052FB002806D00322A3896B
:10C2E00093431A0001231343A381A0893843A081FB
:10C2F000CBE7C046B9C0000010B5034B0100186879
:10C3000000F06CF810BDC0468000002082B000290B
:10C3100000D101A9101E06D0002B06D013780B60A7
:10C320001078431E984102B0704702204042FAE75D
:10C33000C9B28218904201D10020704703788B4225
:10C34000FBD00130F6E7000070B50500002910D0E1
:10C350000C1F2368002B00DAE418280000F034FBDF
:10C360001D4A1368002B05D163601460280000F09B
:10C370002CFB70BDA34209D9216860188342F3D118
:10C3800018685B6841182160EEE713005A68002ABC
:10C3900001D0A242F9D919685818A0420BD12068DF
:10C3A0000918581819608242E0D110685268411883
:10C3B00019605A60DAE7A04202D90C232B60D5E756
:10C3C00021686018824203D11068526841182160C8
:10C3D00062605C60CAE7C046201C0020032370B581
:10C3E000CD1C9D43083506000C2D1ED20C25A942FC
:10C3F0001DD8300000F0E8FA254A14682100002911
:10C4000019D1244C2368002B03D1300000F0CAF965
:10C4100020602900300000F0C5F9431C2BD10C230B
:10C420003000336000F0D1FA03E0002DDFDA0C2396
:10C430003360002070BD0B685B1B19D40B2B03D934
:10C440000B60CC18256003E04B688C420DD1136063
:10C45000300000F0BAFA200007220B30231D904371
:10C46000C31AE7D05A42E250E4E763600C00EFE7FA
:10C470000C004968C3E70323C41C9C43A042E1D0DD
:10C48000211A300000F08EF9431CDBD1C7E7C0460B
:10C49000201C0020241C0020F8B507000D00160009
:10C4A000002905D11100FFF799FF04002000F8BD15
:10C4B000002A03D1FFF748FF3400F7E700F086FABF
:10C4C0002C00B042F2D231003800FFF787FF041E83
:10C4D000ECD029003200FEF7BFFF29003800FFF73B
:10C4E00033FFE3E7F0B58E6885B007000C000392D8
:10C4F00001939E423CD890238A89DB001A4234D0B3
:10C500000325096923685B1A0293636902985D43F6
:10C51000EB0F5D19019B6D1001331B18AB4200D965
:10C520001D00530532D529003800FFF757FF061EBE
:10C5300009D10C233B6040230120A28940421343D0
:10C54000A38105B0F0BD029A2169FEF785FFA3899A
:10C55000144A1A4080231343A381029B2661F618D4
:10C5600026606561019EED1AA560019B9E4200D97F
:10C57000019E320003992068FEF777FFA368002030
:10C580009B1BA36023689E192660DAE72A00380007
:10C59000FFF782FF061EE0D121693800FFF7D4FEC5
:10C5A000C7E7C0467FFBFFFFF0B59FB00290059341
:10C5B0008B890F0016001B0611D50B69002B0ED1BD
:10C5C0004021FFF70BFF38603861002805D10C23AC
:10C5D000029A013813601FB0F0BD40237B61002335
:10C5E00006AC6361203363761033A37635002B7875
:10C5F000002B01D0252B46D1AB1B04930CD032006D
:10C6000039000298FFF76EFF431C00D1AEE062696B
:10C61000049B9446634463612B78002B00D1A5E012
:10C62000012200235242626002A9543252186E1C49
:10C630002360E360A3601370A3653178052254483A
:10C64000FFF776FE751C00281FD12268D30604D59B
:10C65000532302A95B1820211970130704D5532313
:10C6600002A95B182B21197033782A2B16D03500BC
:10C6700000210A20E3682A786E1C303A092A4ED934
:10C68000002918D010E00135B1E7414B2268C01AEB
:10C6900001238340134323602E00CEE7059B191D21
:10C6A0001B680591002B01DB099304E05B42E3600A
:10C6B0000223134323602B782E2B0AD16B782A2B6D
:10C6C00035D1059B02351A1D1B680592002B2BDB0B
:10C6D0000793304E297803223000FFF729FE002807
:10C6E00006D04023801B834022680135134323601A
:10C6F0002978062228486E1C2176FFF719FE0028AB
:10C700003CD0264B002B25D10722059B07339343B2
:10C71000083305936369039A9B18636166E7434393
:10C7200001219B183500A6E701235B42D0E70023D7
:10C730000A201A000135636029786E1C30390929F6
:10C7400003D9002BC5D00792C3E7424301235218F7
:10C750003500F1E705AB00933A00114B2100029838
:10C7600000E000BF0390039B0133D3D1BB890B983A
:10C770005B0600D42FE7012040422CE705AB009375
:10C780003A00074B21000298FFF736F8EAE7C04667
:10C79000D0E10000D6E10000DAE100000000000076
:10C7A000E5C40000002370B5064C050008002360B6
:10C7B00000F060F9431C03D12368002B00D02B60EC
:10C7C00070BDC046B42F002070B504000D001F29B5
:10C7D00004D9162303600120404270BD436C002B36
:10C7E00004D08A009B181A68002A08D1200000F0A3
:10C7F00031F82A000100200000F01AF8EDE70020CF
:10C80000012AEAD0511C03D1162301302360E4E74A
:10C81000002428001C6090472000DEE710B5034B81
:10C8200001001868FFF7D0FF10BDC046800000204F
:10C83000002370B5064C050008001100236000F0CD
:10C8400001F9431C03D12368002B00D02B6070BD7D
:10C85000B42F002010B500F0E5F810BD70B50C0045
:10C860000E25495F00F0BAF8002803DB636D1B1842
:10C87000636570BDA389024A1340A381F9E7C046EE
:10C88000FFEFFFFFF8B51F008B8905000C001600B5
:10C89000DB0505D50E23C95E0022022300F080F8D7
:10C8A000A389054A28001340A38132000E23E15ECC
:10C8B0003B0000F02BF8F8BDFFEFFFFF70B50C0058
:10C8C0000E25495F00F06CF8A389421C03D1054A8C
:10C8D0001340A38170BD802252011343A381606580
:10C8E000F8E7C046FFEFFFFF10B50E23C95E00F06A
:10C8F00021F810BD0B1E04D0FF2A04D98A2303603F
:10C900008B3B180070470A700123FAE770B50500E9
:10C91000080011000022064C22601A0000F0B8F84E
:10C92000431C03D12368002B00D02B6070BDC04690
:10C93000B42F0020002370B5064C050008002360CA
:10C9400000F060F8431C03D12368002B00D02B605B
:10C9500070BDC046B42F0020002370B5064C050002
:10C9600008001100236000F055F8431C03D1236830
:10C97000002B00D02B6070BDB42F0020002370B5B9
:10C98000064C05000800236000F054F8431C03D156
:10C990002368002B00D02B6070BDC046B42F002050
:10C9A00070B50500080011000022064C22601A0034
:10C9B00000F050F8431C03D12368002B00D02B60FB
:10C9C00070BDC046B42F0020704770470B1F1B6816
:10C9D000181F002B01DA0B58C018704770B50500FE
:10C9E000080011000022064C22601A0000F03AF8FC
:10C9F000431C03D12368002B00D02B6070BDC046C0
:10CA0000B42F002058220120014B40421A60704789
:10CA1000B42F002058220120014B40421A60704779
:10CA2000B42F002058220120014B40421A60704769
:10CA3000B42F00205822024B00201A607047C046D5
:10CA4000B42F002058220120014B40421A60704749
:10CA5000B42F002058220120014B40421A60704739
:10CA6000B42F002058220120014B40421A60704729
:10CA7000B42F0020044A1368002B00D1034B181870
:10CA8000106018007047C046281C0020B82F0020F6
:10CA900058220120014B40421A607047B42F0020F9
:10CAA000FEE7C046F8B5C046F8BC08BC9E467047D5
:10CAB000F8B5C046F8BC08BC9E4670476461746116
:10CAC0000000000040CB0000EF01000049CB000057
:10CAD000E302000051CB00000909000058CB000020
:10CAE000190A00005DCB00003105000068CB000092
:10CAF000530300006DCB0000710C000079CB0000E7
:10CB00001F02000083CB00001108000091CB000041
:10CB1000BD0600009ECB0000F104000072616E644F
:10CB20006F6D00616C6C006C6173740066616C7396
:10CB300065007472756500252E3135732E2E2E001A
:10CB40006D616B654C697374006164644C617374EE
:10CB50000064656C657465006A6F696E00636F7070
:10CB60007946726F6D546F0066696E64006A6F6912
:10CB70006E537472696E677300756E69636F646576
:10CB8000417400756E69636F6465537472696E6792
:10CB9000006E6577427974654172726179006672E0
:10CBA00065654D656D6F72790000000011CC000065
:10CBB000D910000016CC0000F710000051CB000087
:10CBC000FB1000001CCC0000DD10000026CC000093
:10CBD000FF1000002FCC00000311000039CC000032
:10CBE0000711000044CC00000B11000050CC0000E5
:10CBF000E110000059CC0000EF10000063CC0000F1
:10CC0000E51000006ECC0000F310000066696C6552
:10CC1000006F70656E00636C6F736500656E644FC6
:10CC20006646696C6500726561644C696E65007288
:10CC3000656164427974657300617070656E644CFF
:10CC4000696E6500617070656E6442797465730029
:10CC500066696C6553697A650073746172744C69B6
:10CC60007374006E657874496E4C697374007379DF
:10CC70007374656D496E666F000000003813000024
:10CC80004813000062130000E013000018140000B5
:10CC90004E14000086140000AC140000E8140000DC
:10CCA0002A15000080150000C41500003016000091
:10CCB000781600009E160000D61600001C17000013
:10CCC00042170000701700009E170000D4170000E4
:10CCD000581800002019000096190000061A0000DC
:10CCE000521A0000721A0000941A0000461B00003D
:10CCF0008C1B0000041C0000321C0000621C0000A1
:10CD0000981C0000001D0000801D0000C61D0000D2
:10CD10000E1E0000841E0000FA1E0000421F0000CC
:10CD2000881F0000BE1F0000042000004A200000F1
:10CD300092200000E6200000442100008221000033
:10CD4000EC210000222200006A220000B222000032
:10CD5000FA220000342300007C230000C4230000DA
:10CD60003025000070170000381300002C2400004C
:10CD700038130000622400008E240000C424000048
:10CD8000F0240000381300003813000038130000AE
:10CD900038130000AA250000EC250000381300001D
:10CDA000381300003226000082260000A82600006A
:10CDB000D62600003813000038130000FA260000C1
:10CDC0002A2700005A27000090270000BA270000F9
:10CDD000F02700001A280000422800006A280000FE
:10CDE0009A280000CA280000F42800004C290000FE
:10CDF0007C290000A6290000381300003813000029
:10CE0000381300003813000038130000D629000042
:10CE1000022A00002E2A00005A2A0000862A00005A
:10CE2000BC2A0000F22A0000282B00005E2B000024
:10CE30008A2B0000B62B0000EC2B000038130000FA
:10CE400038130000381300003813000038130000B6
:10CE500038130000381300003813000038130000A6
:10CE60003813000038130000381300003813000096
:10CE700038130000182C00004E2C00005B256420A5
:10CE80006974656D206C6973745D00282564206287
:10CE9000797465732900286F626A656374207479F8
:10CEA00070653A2025642900537461636B20756EA8
:10CEB000646572666C6F7700626F6F6C65616E009F
:10CEC0006E756D62657200737472696E67006C696D
:10CED0007374006279746520617272617900000078
:10CEE00007000000030000003ACF0000712D000091
:10CEF00042CF0000212E00004BCF0000CB2E0000BF
:10CF000054CF0000752D00005DCF0000CF2E000033
:10CF100065CF0000B92E00000000000001000000F5
:10CF20000200000003000000040000000A000000EE
:10CF30006D6963726F3A62697400686173546F6EF1
:10CF40006500706C6179546F6E650068617353653C
:10CF500072766F00736574536572766F00646163F7
:10CF6000496E697400646163577269746500474370
:10CF700020746F6F6B2025642075736563733B208D
:10CF80006672656520256420776F726473003C4982
:10CF90006E74656765723E003C4C6973743E003C7C
:10CFA0004F626A6563743E003C42797465417272F7
:10CFB00061793E000D0A564D2050616E69633A203A
:10CFC00025730D0A006D69736300000001D0000035
:10CFD000953B00000AD00000253B00000ED0000069
:10CFE000793A000016D000001F3A000020D000005F
:10CFF000B53900002CD00000B73800006E756C6C9D
:10D0000000686578546F496E740073696E006A73C6
:10D010006F6E476574006A736F6E436F756E740050
:10D020006A736F6E56616C75654174006A736F6EDA
:10D030004B6579417400000094D00000013C000071
:10D040009CD00000053C0000A6D00000233C00005E
:10D05000AFD000002D3C0000BAD00000373C0000EB
:10D06000C6D00000413C0000DBD000004B3C00007B
:10D07000F0D00000553C0000FCD000005F3C0000F8
:10D080000CD100000F3C000018D10000193C00003A
:10D090006E657400686173576946690073746172E4
:10D0A00074576946690073746F70576946690077F1
:10D0B000696669537461747573006D794950416490
:10D0C0006472657373006874747053657276657208
:10D0D0004765745265717565737400726573706F1E
:10D0E0006E64546F48747470526571756573740022
:10D0F00068747470436F6E6E6563740068747470E6
:10D100004973436F6E6E6563746564006874747010
:10D1100052657175657374006874747052657370CC
:10D120006F6E7365001A1B1C03040607090A1718A3
:10D1300019000000000008080800080A4A40000022
:10D140000A5FEA5FEA0ED92ED36E19324489330C96
:10D15000924C924D08080000000488080804080456
:10D16000848488000A448A4000048EC48000000041
:10D17000048800000EC0000000000800012244885E
:10D18000100C9252524C048C84848E1C824C901E43
:10D190001EC244924C06CA525FE21FF01EC13E02FC
:10D1A000448ED12E1FE24488100ED12ED12E0ED1E6
:10D1B0002EC4880008000800000480048802448807
:10D1C0000482000EC00EC008048244880ED126C01E
:10D1D000040ED135B36C0C925ED2521C925C925C00
:10D1E0000ED010100E1C9252525C1ED01C901E1EAF
:10D1F000D01C90100ED013712E12525ED2521C8889
:10D2000008081C1FE242524C12549814921010103D
:10D21000101E113B75B131113935B3710C92525258
:10D220004C1C925C90100C92524C861C925C925159
:10D230000ED00C825C1FE4848484125252524C1132
:10D2400031312A44113135BB7112524C9252112A9C
:10D250004484841EC488101E0EC808080E100804DA
:10D2600082410EC242424E048A400000000000008B
:10D270001F0804800000000ED2524F10101C925C58
:10D28000000ED0100E02424ED24E0C925C900E0652
:10D29000C81C88080ED24EC24C10101C92520800B6
:10D2A000080808024002424C10149814920808081A
:10D2B0000806001B75B131001C925252000C9252AC
:10D2C0004C001C925C90000ED24EC2000ED010108A
:10D2D0000006C8049808080EC807001252524F00F2
:10D2E00011312A4400113135BB00124C8C920011CF
:10D2F0002A4498001EC4881E06C48C848608080828
:10D30000080818080C881800000C83600000000052
:10D310000100000002000000030000000400000003
:10D3200005000000060000000700000008000000E3
:10D33000090000000A0000000B0000000C000000C3
:10D340000D0000000E0000000F00000010000000A3
:10D350001200000014000000160000001800000079
:10D360001A0000001C0000001E0000002000000049
:10D370002300000026000000290000002C0000000F
:10D380002F00000032000000360000003A000000CC
:10D390003E00000042000000460000004B0000007C
:10D3A00050000000550000005A000000610000001D
:10D3B000680000006F000000760000007D000000A3
:10D3C000840000008B000000920000009900000023
:10D3D000A0000000A7000000AE000000B5000000A3
:10D3E000BC000000C3000000CA000000D100000023
:10D3F000D8000000DF000000E6000000ED000000A3
:10D40000F4000000FB000000FF0000005CD40000FE
:10D41000813C000067D40000D141000071D40000BD
:10D420003D3E00007ED400004140000085D4000055
:10D43000914000008ED40000E14000009AD400002A
:10D44000D93F0000ABD40000AD3E0000B8D40000CE
:10D45000693F0000646973706C6179006C6967688A
:10D46000744C6576656C006D62446973706C6179AB
:10D47000006D62446973706C61794F6666006D621D
:10D48000506C6F74006D62556E706C6F74006D62DD
:10D49000447261775368617065006D6253686170B2
:10D4A00065466F724C6574746572006E656F506985
:10D4B00078656C53656E64006E656F506978656C55
:10D4C00053657450696E004E6F7420656E6F75679A
:10D4D0006820726F6F6D206576656E206166746579
:10D4E0007220636F6D70616374696F6E00436F6D5E
:10D4F00070616374656420466C61736820636F6457
:10D50000652073746F72650A25642062797465738F
:10D51000207573656420282564252529206F6620E1
:10D52000256400426164207265636F726420666FD7
:10D53000756E6420647572696E6720696E697469BE
:10D54000616C697A6174696F6E00256420256420BE
:10D5500025642028256420776F7264732900256470
:10D56000207265636F7264732C20256420776F725C
:10D5700064732C206D617849442025642C20636FEE
:10D580006D70616374696F6E206379636C6573207D
:10D59000256400526573746F72656420256420737E
:10D5A000637269707473005374617274656400729D
:10D5B0006164696F0000000048D60000994B0000CC
:10D5C00055D60000354E000065D60000B54D000070
:10D5D00073D60000C94F00007ED60000C14B00008A
:10D5E0008ED60000494C0000A2D60000314C00004D
:10D5F000B1D60000AB510000BDD60000295100009B
:10D60000C6D60000CD500000D1D600001550000055
:10D61000DCD6000051500000E5D600008550000027
:10D62000EED60000D14B0000FDD60000B14B00004B
:10D6300006D70000E14B00006E6F6E65006F7468E6
:10D64000657200706169720064697361626C655231
:10D650006164696F006D65737361676552656365C9
:10D6600069766564007061636B65745265636569B2
:10D670007665007061636B657453656E64007265F6
:10D68000636569766564496E746567657200726585
:10D690006365697665644D65737361676554797018
:10D6A00065007265636569766564537472696E6757
:10D6B0000073656E64496E74656765720073656EAC
:10D6C00064506169720073656E64537472696E6749
:10D6D000007365744368616E6E656C0073657447B2
:10D6E000726F757000736574506F7765720073693F
:10D6F000676E616C537472656E67746800646576FA
:10D700006963654944006C6173744D657373616747
:10D7100065494400556E6B6E6F776E207072696D4F
:10D720006974697665205B25733A25735D00000096
:10D7300000000000963007772C610EEEBA5109996F
:10D7400019C46D078FF46A7035A563E9A395649ECB
:10D750003288DB0EA4B8DC791EE9D5E088D9D297EF
:10D760002B4CB609BD7CB17E072DB8E7911DBF904B
:10D770006410B71DF220B06A4871B9F3DE41BE846F
:10D780007DD4DA1AEBE4DD6D51B5D4F4C785D383CB
:10D7900056986C13C0A86B647AF962FDECC9658A6F
:10D7A0004F5C0114D96C0663633D0FFAF50D088DCB
:10D7B000C8206E3B5E10694CE44160D5727167A26F
:10D7C000D1E4033C47D4044BFD850DD26BB50AA5CB
:10D7D000FAA8B5356C98B242D6C9BBDB40F9BCACEF
:10D7E000E36CD832755CDF45CF0DD6DC593DD1AB4B
:10D7F000AC30D9263A00DE518051D7C81661D0BF6F
:10D80000B5F4B42123C4B3569995BACF0FA5BDB8CA
:10D810009EB802280888055FB2D90CC624E90BB16E
:10D82000877C6F2F114C6858AB1D61C13D2D66B6CA
:10D830009041DC760671DB01BC20D2982A10D5EF2E
:10D840008985B1711FB5B606A5E4BF9F33D4B8E88A
:10D85000A2C9077834F9000F8EA8099618980EE12E
:10D86000BB0D6A7F2D3D6D08976C6491015C63E68A
:10D87000F4516B6B62616C1CD83065854E0062F2AE
:10D88000ED95066C7BA5011BC1F4088257C40FF50A
:10D89000C6D9B06550E9B712EAB8BE8B7C88B9FC2E
:10D8A000DF1DDD62492DDA15F37CD38C654CD4FB8A
:10D8B0005861B24DCE51B53A7400BCA3E230BBD42E
:10D8C00041A5DF4AD795D83D6DC4D1A4FBF4D6D38A
:10D8D0006AE96943FCD96E34468867ADD0B860DA2E
:10D8E000732D0444E51D03335F4C0AAAC97C0DDD8A
:10D8F0003C710550AA41022710100BBE86200CC9AE
:10D9000025B56857B3856F2009D466B99FE461CE09
:10D910000EF9DE5E98C9D9292298D0B0B4A8D7C72D
:10D92000173DB359810DB42E3B5CBDB7AD6CBAC089
:10D930002083B8EDB6B3BF9A0CE2B6039AD2B174A5
:10D940003947D5EAAF77D29D1526DB048316DC7301
:10D95000120B63E3843B64943E6A6D0DA85A6A7AA5
:10D960000BCF0EE49DFF099327AE000AB19E077D01
:10D9700044930FF0D2A3088768F2011EFEC2066925
:10D980005D5762F7CB67658071366C19E7066B6E81
:10D99000761BD4FEE02BD3895A7ADA10CC4ADD67A5
:10D9A0006FDFB9F9F9EFBE8E43BEB717D58EB06001
:10D9B000E8A3D6D67E93D1A1C4C2D83852F2DF4FA5
:10D9C000F167BBD16757BCA6DD06B53F4B36B24801
:10D9D000DA2B0DD84C1B0AAFF64A0336607A0441A5
:10D9E000C3EF60DF55DF67A8EF8E6E3179BE694601
:10D9F0008CB361CB1A8366BCA0D26F2536E2685225
:10DA000095770CCC03470BBBB91602222F26055580
:10DA1000BE3BBAC5280BBDB2925AB42B046AB35CA4
:10DA2000A7FFD7C231CFD0B58B9ED92C1DAEDE5B00
:10DA3000B0C2649B26F263EC9CA36A750A936D02E4
:10DA4000A906099C3F360EEB856707721357000540
:10DA5000824ABF95147AB8E2AE2BB17B381BB60C64
:10DA60009B8ED2920DBED5E5B7EFDC7C21DFDB0BC0
:10DA7000D4D2D38642E2D4F1F8B3DD686E83DA1FE4
:10DA8000CD16BE815B26B9F6E177B06F7747B71840
:10DA9000E65A0888706A0FFFCA3B06665C0B0111E4
:10DAA000FF9E658F69AE62F8D3FF6B6145CF6C1640
:10DAB00078E20AA0EED20DD75483044EC2B30339E4
:10DAC000612667A7F71660D04D476949DB776E3E40
:10DAD0004A6AD1AEDC5AD6D9660BDF40F03BD83764
:10DAE00053AEBCA9C59EBBDE7FCFB247E9FFB530C0
:10DAF0001CF2BDBD8AC2BACA3093B353A6A3B424E4
:10DB00000536D0BA9306D7CD2957DE54BF67D9233F
:10DB10002E7A66B3B84A61C4021B685D942B6F2AE3
:10DB200037BE0BB4A18E0CC31BDF055A8DEF022D3F
:10DB3000416C6C207461736B732073746F707065CB
:10DB400064007630383600202573202573004D653B
:10DB50006D6F727920636C6561726564004E6F2031
:10DB600066726565207461736B20656E7472696599
:10DB700073000000BCDB000035650000C9DB00005D
:10DB800071610000D5DB000005650000DBDB0000F3
:10DB900015650000E1DB000025650000E7DB000003
:10DBA000A5610000F1DB000091650000F9DB0000D9
:10DBB000E562000073656E736F7273006163636585
:10DBC0006C65726174696F6E0074656D7065726109
:10DBD000747572650074696C74580074696C74595A
:10DBE0000074696C745A00746F756368526561647F
:10DBF0000069326352656164006932635772697407
:10DC00006500000078DC00001D66000086DC000076
:10DC1000216600008FDC00002D66000099DC00000A
:10DC200031660000A2DC000035660000A7DC0000C1
:10DC300039660000ACDC00003D660000B8DC000086
:10DC400041660000BFDC000045660000C8DC000043
:10DC500049660000CDDC00004D660000D8DC000005
:10DC600051660000E2DC000025660000ECDC0000EC
:10DC70002966000074667400656E61626C654469B3
:10DC800073706C61790067657457696474680067C4
:10DC90006574486569676874007365745069786570
:10DCA0006C006C696E65007265637400726F756EEE
:10DCB0006465645265637400636972636C650074C3
:10DCC0007269616E676C650074657874007466745F
:10DCD000546F756368656400746674546F75636827
:10DCE0005800746674546F75636859007466745490
:10DCF0006F756368507265737375726500766172D3
:10DD00007300000024DD0000E16A00002EDD000049
:10DD1000C16A000037DD00009D6A000043DD00009D
:10DD2000296A0000766172457869737473007661C0
:10DD3000724E616D6564007365745661724E616DFB
:10DD40006564007661724E616D65466F72496E64FE
:10DD500065780057656C636F6D6520746F204D6941
:10DD600063726F426C6F636B732100705F737069D5
:10DD700020213D204E554C4C002F686F6D652F675C
:10DD800069742F2E706C6174666F726D696F2F707D
:10DD900061636B616765732F6672616D65776F7222
:10DDA0006B2D61726475696E6F6E6F726469636EFC
:10DDB0007266352F6C69627261726965732F535098
:10DDC000492F5350492E63707000535049436C6182
:10DDD00073733A3A535049436C617373284E5246F9
:10DDE0005F5350495F547970652A2C2075696E74B1
:10DDF000385F742C2075696E74385F742C207569D7
:10DE00006E74385F742900000000000000000000FC
:10DE1000ED6C0000A96C0000CF6C0000D96C000014
:10DE2000E36C0000CD6C0000030000000200000065
:10DE300001000000040000000500000011000000C7
:10DE40000C0000000B000000120000000A0000009F
:10DE5000060000001A000000140000001700000077
:10DE6000160000001500000010000000FFFFFFFF7B
:10DE7000FFFFFFFF000000001E000000190000006F
:10DE80001800000007000000080000000900000062
:10DE90000D0000000E0000000F0000001C0000003C
:10DEA0001B0000001D000000130000000000000027
:10DEB000000000009D710000CD7800001D72000080
:10DEC0003172000027720000997100008D7100000E
:10DED0003D720000B971000089710000000000006F
:10DEE000000000000000304300000000000030C3CC
:10DEF0007371727400000000FB21F93FFB2109409F
:10DF00007CD91240FB2119407A6A1F407CD92240FB
:10DF1000BBFD2540FB2129403A462C407A6A2F4020
:10DF20005C4731407CD932409C6B3440BBFD35406E
:10DF3000DB8F3740FB2139401BB43A403A463C4026
:10DF40005AD83D407A6A3F404C7E40405C47414051
:10DF50006C1042407CD942408CA243409C6B4440B0
:10DF6000AC344540BBFD4540CBC64640DB8F474007
:10DF7000EB584840FB21494083F9A200444E6E0013
:10DF8000FC291500D1572700DD34F50062DBC00005
:10DF90003C999500419043006351FE00BBDEAB000D
:10DFA000B761C5003A6E2400D24D42004906E00038
:10DFB00009EA2E001C92D100EB1DFE0029B11C00C5
:10DFC000E83EA700F535820044BB2E009CE98400A2
:10DFD000B4267000417E5F00D6913900538339002A
:10DFE0009CF439008B5F840028F9BD00F81F3B00CA
:10DFF000DEFF97000F980500112FEF000A5A8B00E3
:10E000006D1F6D00CF7E360009CB2700464FB7004D
:10E010009E663F002DEA5F00BA277500E5EBC7005A
:10E020003D7BF100F739070092528A00FB6BEA0052
:10E030001FB15F00085D8D00300356007BFC460079
:10E04000F0AB6B0020BCCF0036F49A00E3A91D00B2
:10E050005E619100081BE60085996500A0145F00D1
:10E060008D40680080D8FF0027734D000606310000
:10E07000CA561500C9A873007BE260006B8CC00013
:10E0800000000040FB21F93F000000002D44743ED9
:10E09000000000809846F83C0000006051CC783BBE
:10E0A00000000080831BF0390000004020257A38F2
:10E0B000000000802282E336000000001DF3693575
:10E0C0000200000003000000040000000600000041
:10E0D000C49500006E9500006E9500009C960000AF
:10E0E0006A9500006A950000929600009C960000D8
:10E0F0006A950000929600006A9500009C960000C8
:10E10000A0960000A0960000A0960000A89600002F
:10E11000A0A00000129F0000569F0000BA9E0000C1
:10E12000569F000046A00000569F0000BA9E0000C7
:10E13000129F0000129F000046A00000BA9E00003F
:10E14000B29E0000B29E0000B29E000054A00000EB
:10E15000C8A70000CAA60000CAA60000E8A90000DF
:10E16000C4A60000C4A60000D0A90000E8A90000D1
:10E17000C4A60000D0A90000C4A60000E8A90000C1
:10E18000DEA90000DEA90000DEA90000ECA9000065
:10E190002C2066756E6374696F6E3A20006173732C
:10E1A000657274696F6E2022257322206661696C26
:10E1B00065643A2066696C6520222573222C206CE8
:10E1C000696E65202564257325730A00840000208C
:10E1D000232D302B2000686C4C0065666745464750
:10E1E00000303132333435363738394142434445D3
:10E1F0004600303132333435363738396162636442
:10E200006566000000000000000000000000000043
:10E2100000000000000000000000000000000000FE
:10E2200000000000000000000000000000000000EE
:10E2300000000000000000000000000000000000DE
:10E2400000000000000000000000000000000000CE
:10E2500000000000000000000000000000000000BE
:10E26000000000004300504F534958000020202078
:10E270002020202020202828282828202020202076
:10E280002020202020202020202020202088101046
:10E2900010101010101010101010101010040404A2
:10E2A0000404040404040410101010101010414160
:10E2B000414141410101010101010101010101014E
:10E2C0000101010101010101101010101010424262
:10E2D000424242420202020202020202020202021E
:10E2E00002020202020202021010101020000000BE
:10E2F000000000000000000000000000000000001E
:10E30000000000000000000000000000000000000D
:10E3100000000000000000000000000000000000FD
:10E3200000000000000000000000000000000000ED
:10E3300000000000000000000000000000000000DD
:10E3400000000000000000000000000000000000CD
:10E3500000000000000000000000000000000000BD
:10E3600000000000000000000000000000000000AD
:04E3700000000000A9
:08E37400941DFF7F0100000071
:10E37C00FFFFFFFF4006000001000000E803DC0582
:10E38C00DC05DC05DC050000FFFFFFFFFFFFFFFFE6
:10E39C001800000019FCFFFFFFFFFFFFFF0000004B
:10E3AC000200000003000000FFFFFFFF0000000060
:10E3BC00010000000000020001000000FFFFFFFF51
:10E3CC000000000002000000000004000200000039
:10E3DC00FFFFFFFF0000000003000000000008002A
:10E3EC00030000000A00000008000000010000000B
:10E3FC00840000200000000024E2000044E2000041
:10E40C0004E200000000000000000000000000001A
:10E41C0000000000000000000000000000000000F0
:10E42C0000000000000000000000000000000000E0
:10E43C0000000000000000000000000000000000D0
:10E44C0000000000000000000000000000000000C0
:10E45C00000000004300000000000000000000006D
:10E46C0000000000000000000000000000000000A0
:10E47C00000000004300000000000000000000004D
:10E48C000000000000000000000000000000000080
:10E49C00000000004300000000000000000000002D
:10E4AC000000000000000000000000000000000060
:10E4BC00000000004300000000000000000000000D
:10E4CC000000000000000000000000000000000040
:10E4DC0000000000430000000000000000000000ED
:10E4EC000000000000000000000000000000000020
:10E4FC0000000000430000000000000000000000CD
:10E50C0000000000000000000000000000000000FF
:10E51C0000000000430000000000000000000000AC
:10E52C0000000000000000000000000000000000DF
:10E53C0000000000F5C800000DC300000000000042
:10E54C006CE200003ECB0000C4CF0000C4CF000042
:10E55C00C4CF0000C4CF0000C4CF0000C4CF000063
:10E56C00C4CF0000C4CF0000C4CF0000FFFFFFFFEA
:10E57C00FFFFFFFFFFFFFFFFFFFF00000100415304
:10E58C0043494900000000000000000000000000AA
:10E59C0000000000000000000000000000004153DB
:10E5AC00434949000000000000000000000000008A
:10E5BC00000000000000000000000000000000004F
:10E5CC00E9000000796C0000C16F0000E9740000E4
:04E5DC00C10000007A
:040000030000705D2C
:00000001FF
